:080000000C94980D0C94000013
:100008000C9400000C9400000C9400000C94000068
:100018000C9400000C94A7610C9400000C94000050
:100028000C94DC150C9400000C9400000C94000057
:100038000C9400000C9400000C9497150C9400008C
:100048000C945D5E0C9400000C94995E0C94000076
:100058000C9400000C9400000C9400000C94000018
:100068000C9400000C9400000C9400000C94000008
:100078000C9402600C9400000C9445610C940000F0
:100088000C940000000001000200040008001000A9
:100098002000400080000001000200040008001059
:1000A8000020004000800001020408102040800069
:1000B800B003C10B80100000B403C10B821F000005
:1000C800BE03C10B81030000C603C10B010403007A
:1000D800D003C20B01060500DA03C40B018000003F
:1000E800E603CB0B020F0000EE03C50B020F000066
:1000F800F603C70B020FD012FE03C90B0110000054
:100108000804190C011000001204CA0B00010000B9
:100118001A04CD0B010801002404CE0B03080100CA
:100128003204CF0B030700003A04E50B017F3F00C0
:100138004404E40B010400004E04D00B0304000047
:100148005604E30B01641E006204D10B0001000099
:100158006E04D20B000100007A04E20B01020000D9
:100168008604D30B000100009404D40B020F000096
:10017800A004D60B020FE703AA04180C01630000C1
:1001880008051A0C01100000B604D80B030801007A
:10019800BC04D90B03080000C204DA0B03080000F2
:1001A800C804DB0B03080000CE04DC0B03080000C6
:1001B800D404DD0B03080000DA04DE0B030800009A
:1001C800E004E60B040A2E00E804F00B040A2E00F3
:1001D800F004FA0B040A2E00F804040C040A2E009A
:1001E80000050E0C040A2E0000000000FF000000AD
:1001F800120500021A0504042005080726050C0547
:1002080026058C062C0580093405100B3C05500C7E
:10021800460540034E05140A5805180860051C01D8
:1002280000000002280060009800D000080140018A
:10023800210C58002D0B2D002B0B2B004D0A4D00C7
:10024800808182838400002188898A8B8C8D8E8F9F
:10025800310B312041424300320B322044454600E5
:10026800330B3320474849004D0A4D000000000079
:10027800340B34204A4B4C00350B35204D4E4F0083
:10028800360B3620505152002B0A2B00000000007C
:10029800370B372053545500380B38205657580021
:1002A800390B3920595A2F002D0A2D000000000063
:1002B800430C430000000000300B3020202E2C009F
:1002C8002C0A2C00000000003D0A435200000000E8
:1002D80000004A01460032002100004B004A014656
:1002E8000032004D000096004A01460032005400DA
:1002F80000E1004A01460032003D0000F000000025
:10030800320050002D0000F000500032005000472D
:100318000000F000A000320050004B0000F000F098
:1003280000320050002B00005800B40004003800D0
:100338003800213003006A6100008700C8006400AB
:1003480032003D3E03006E65696E00000800C8007B
:1003580064003200214E03004B004A01460032007F
:100368004D00000001000100E60063004D000000A0
:100378000000A0001B00007105D700A0001A0200B1
:10038800710569000000180400730569001E011951
:100398000600730550726F64756B7420000053700B
:1003A80061727465202000005F4944005F52733217
:1003B8003332494400005F526F74617465005F54C2
:1003C800617374656E5800005F54617374656E598B
:1003D80000005F44656661756C744B6579002A435B
:1003E8006F64653000002A436F64653100002A435A
:1003F8006F64653200002A4D61784D6F64756C003A
:100408005F4572774D6F64756C002A546973636831
:1004180045005F4D795465726D4E72005F4D617392
:100428007465725465726D7300005F454D6F646545
:1004380000005F4543726564577472005F52733001
:100448004D6F646500005F5634756E6435005F500B
:10045800756C736554696D6500005F41736B437219
:100468006564697400005F53656E6444656269740D
:1004780000005F4372656469744D6F6465005F4393
:1004880072656469744D6173746572002A5461629F
:100498006C655374617274002A5461626C65456EB0
:1004A80064002A4669727374426F6E5000002A4ACB
:1004B8006F6231002A4A6F6232002A4A6F62330043
:1004C8002A4A6F6234002A4A6F6235002A4A6F62EC
:1004D80036002A4A6F6237005F4572726F723100C8
:1004E8005F4572726F7232005F4572726F723300CD
:1004F8005F4572726F7234005F4572726F723500B9
:100508005F467265696761626500546173746572FC
:1005180000004C69745A00004C65697454005075A9
:100528006C73000054617374203000007365726945
:10053800656C6C0073657269656C203200005461EB
:10054800737420320000546173742070617200006B
:10055800466F6C67655400005377697463680000E0
:10056800706F7274696F6E696572656E00002E66D1
:100578006F6C67650000506F7274696F6E656E20EE
:100588007369636865726E00436865662D4D656EB4
:1005980075004B206C697374656E00004B206C6F9E
:1005A80065736368656E00004B20647275636B65E4
:1005B8006E0054206C697374656E000054206C6F73
:1005C80065736368656E00005420647275636B65BB
:1005D8006E0053797374656D0000506F7274696FA3
:1005E8006E004B726564697465004B7265642E43D6
:1005F8006C7200006D616E2E506F7274696F6E00C0
:10060800546573740000506172616D6574657200A1
:1006180050726F64756B746500004B656C6C6E6529
:10062800720056656E74696C6500436F6C6F727307
:100638000000309005319A0532A40533B00534BA6C
:100648000535C40536D00546DA0541E20543EA0515
:1006580044F2054AFC050000000030DA05370806B8
:10066800390E06381806422206452A066332060065
:1006780000004572726F72004F70742E0000496D51
:1006880070756C73000054696D656F7574007A0637
:100698002E0C000500008006310C000300008606C1
:1006A8002F0C000500008E06300C001400002E20D0
:1006B8002C304142433144454632474849334A4B3E
:1006C8004C344D4E4F35505152365354553756577A
:1006D8005838595A2F390500C11100000300D90BA9
:1006E80000000300C1110300170E0300D90B00001E
:1006F8000500E00800000A00C1110A00170E0A00F0
:10070800D90B0A00C1110A00170E2800D90B0000E6
:1007180000000000000000000000000000000000D1
:100728000000000000000000070C182022204D994E
:100738004D40114048914720222018C00700000072
:10074800070C1F3FEE3F7277727FFF7F777F783FFE
:10075800EE3F1FC007000000000000000C183DEE2F
:100768003F3FEE3F1FC80F070002000000000000D7
:1007780000000000000207080F1FCE3F1FC80F0728
:10078800000200000000000000000007080F0F88AA
:100798000F376F7F7FFF7F3260070F8000000000F8
:1007A80000000002000207080F1FCE3F3FEE3F1A6D
:1007B800C0070F80000000000000000000000000DB
:1007C8000006000F0F0006000000000000000000F7
:1007D800FFFFFFFFFFFFFFFFFFF9FFF0F0FFF9FF4B
:1007E800FFFFFFFFFFFFFFFF000000000000060003
:1007F8000910881010881009000600000000000089
:10080800FFFFFFFFFFFFF9FFF6EF77EFEF77EFF658
:10081800FFF9FFFFFFFFFFFF000000000E01006A65
:100828001E33286161886133001E0000000000004B
:10083800000000078C0C186618186C0C078003035E
:100848000C0F030003000000020003038C0302CC1A
:100858000202800202000E1E001E0C0000000000B2
:100868000C000E0B08090CC40E0B4C0938C4787820
:100878004C3103CC030180000000020202271FCC88
:1008880018306770306C181FC22702000200000081
:100898000000001000181C001E1F081F1F001E1C4F
:1008A8000018100000000000000000008801038804
:1008B800070F881F0F8807038801008000000000C9
:1008C80000000207080F1FC0020200020200021FF8
:1008D800C80F0700020000000008191988191988B4
:1008E8001919881919881919800019881900000020
:1008F800000E1F36CC6666CC6636CC1E06CC0606C5
:10090800CC0606CC0600000000081F30C0303008B6
:100918001F30CC301F8C0000CC301F80000000003E
:1009280000000000000000000000000000000000BF
:100938000E1F1FEE1F0000000200070F8C1F020091
:10094800020200020200021FC80F0700021FC000B7
:1009580000000207080F1FC0020200020200020284
:100968000002020002000000000002020002020071
:10097800020200020200021FC80F07000200000066
:1009880000000000000001080101CE3F01C801017C
:10099800000000000000000000000000000004004B
:1009A8000C1C0E3F1C000C0400000000000000009E
:1009B800000000000000000000000000400040406F
:1009C8000040400E7F000000000000000000088C7E
:1009D8001838EF7F38EC180880000000000000008D
:1009E80000000000000000000207080F1FCE3F7F34
:1009F800F000000000000000000000000000000FF0
:100A08007F3FEC1F0F80070200000000000000007D
:100A180000000000000000000000000000000000CE
:100A280000000000000000000600060F000F0F0085
:100A38000F0F000606000600000006000600000072
:100A4800000000198819198819000000000000002A
:100A580000000000000000000006060666063FFCD5
:100A68000C0CC819198C7F330033330000000000C8
:100A78000600061F8C3F3600363F8C1F06CC063F0B
:100A8800C81F060006000000000000001338387E6A
:100A98003801C80307000E1C0E3870EE6000000015
:100AA8000000070D881919801B0E001E3E063333FF
:100AB800C8313BC61E0000000E000E0E00060600E0
:100AC8000C00000000000000000000000000000012
:100AD8000380060E000C1C001C1C001C1C001C0CB7
:100AE800000E0608030000001C0006070003038828
:100AF8000303880303880303000706001C000000A3
:100B0800000000000C3636C81F0F0C3F0F081F36B8
:100B1800CC360000000000000000000000000600C5
:100B280006060C3F3FC00606000600000000000055
:100B380000000000000000000000000000000000AD
:100B4800000E0E000E06000C000000000000000061
:100B580000000C3F3FC00000000000000000000043
:100B6800000000000000000000000000000000007D
:100B7800000E0E000E00000000010000370000EC1F
:100B8800010380070E001C380070600000000000A0
:100B98000F8E3F30676060FB616333666C3378703B
:100BA80036303FE80F0000000300071F001F030056
:100BB800030300030300030300031FEE1F000000EC
:100BC8001FCE3F707360607E0001C80307000E1CD3
:100BD80000387FFF7F0000001FCE3F707360003732
:100BE800000FEC0F0063006037703FEC1F0000003F
:100BF80001CC0307CC0E1CCC3870CC607FFF7F0083
:100C0800CC0000CC000000007FFF7F600060600C1B
:100C18007F3FE7000033006037703FEC1F000000A3
:100C280003CC070E001C3800307FCE7F70736060E5
:100C380037703FEC1F0000007FFF7F00660000CC8C
:100C4800000188010300030600060C000C000000E8
:100C58000F8C1F38E630306E381FCE3F70736060DF
:100C680037703FEC1F0000001FCE3F707360603785
:100C7800703FFF1F006E0001C8031F001E00000028
:100C88000000000000000E000E0E00000000000E24
:100C9800000E0E00000000000000000000000E0022
:100CA8000E0E00000000000E000E0E000606000CDE
:100CB80000CC010380070E001C3800381C000E070A
:100CC800080301CC00000000000000000000000E36
:100CD8003F3FE000000E3F3FE00000000000000042
:100CE8003000381C000E07080301CC010380070EF2
:100CF800001C3800300000001F8C3F70E66060EC7C
:100D08000103800706000606000006000600000032
:100D18001FCE3F306B676FBB6D6DBB6D6DBE6F6770
:100D2800C0703FCC0F0000000600060F000F0F0830
:100D38001919881930CC3F3FC66060666000000012
:100D48007F087F61CC6060CC617F8C7F60E66060EB
:100D58006E607FC87F0000000F8C1F38E63060008F
:100D680060600060600060306E381FC80F000000CF
:100D78007F087F61CC606066606066606066606006
:100D8800CC617F807F0000007FEE7F6000606000A4
:100D9800607F887F6000606000607FEE7F000000F9
:100DA8007FEE7F6000606000607F887F6000606029
:100DB80000606000600000000FCE1F3860306000E7
:100DC8006063EE636066603066381FEE0F000000F7
:100DD8006066606066606066607FEE7F6066606027
:100DE80066606066600000001F881F060006060037
:100DF800060600060600060600061F881F000000FB
:100E0800006600006600006600006600006660601C
:100E18006C703FC81F000000606E6061C8636700A7
:100E28006E7C007C6E0067638C6160E66000000089
:100E3800600060600060600060600060600060608A
:100E480000607FEE7F000000606E7070EE7979E6DA
:100E58006F6F666666666060666060666000000068
:100E68006066707066786C666C66666663666361F9
:100E7800EE6060E6600000000F081F39CC30606645
:100E88006060666060666030CC391F800F000000CB
:100E98007F8C7F60E66060666060EC7F7F8060606A
:100EA80000606000600000000F081F39CC306066E9
:100EB8006060666060666333CC391FE60F0000002F
:100EC8007F8C7F60E66060666060EC7F7F80676330
:100ED8008C6160E6600000001F8C3F70E660600077
:100EE800703F8C1F00E600606E703FC81F00000056
:100EF8003FCC3F060006060006060006060006066A
:100F080000060600060000006066606066606066B5
:100F180060606660606660606C303FC81F000000FB
:100F2800606660606C3030CC3019881919800F0FFA
:100F3800000F06000600000060666060666060667C
:100F48006060666666666F79EE7070E66000000045
:100F580060666030CC3019800F0600060F08193023
:100F6800CC3060666000000060666030CC30198864
:100F7800190F000F0600060600060600060000000E
:100F88007FEE7F00CC000180030600060C001830BD
:100F980000307FEE7F0000001F881F18001818001F
:100FA800181800181800181800181F881F000000CB
:100FB80000004060007038001C0E0007038C010020
:100FC800E7000030000000001F881F018801018829
:100FD800010188010188010188011F881F000000A4
:100FE8000200070F8C1D38E7706030000000000019
:100FF80000000000000000000000000000000000E9
:10100800000000000000000000000000007FFF7FDB
:1010180000000707000706000603000000000000A4
:101028000000000000000000000000000000000CAC
:101038001F3FE6001FEE3F6066607FEE3F00000046
:1010480060006060006060086F7FCE7060666060FE
:101058006E607FC87F0000000000000000000008EC
:101068001F3FC6706000606006703FC81F00000028
:1010780000660000660000661F3FEE7160666060F3
:1010880066703FEE1F00000000000000000000082E
:101098001F3FC6707FEC7F6000703FC81F000000D4
:1010A80007880F1C00181800187F007F18001818F0
:1010B8000018180018000000000000000000000ED2
:1010C8001F3FE670606E703FE61F006E003FC83F2E
:1010D80060006060006060006F7F8C7160CC606051
:1010E800CC6060CC60000000000000060006000034
:1010F8000E0E00060600060600061F881F000000E8
:10110800000000018801000803038801018801012B
:1011180088010188191F800F3000303000303008F6
:10112800313380373E003E37083331CC3000000081
:101138000E000E0600060600060600060600060655
:1011480000061F881F0000000000000000000008C3
:10115800597FCE7F666666666666666666000000CC
:1011680000000000000000083F3FCE3030663030FD
:101178006630306630000000000000000000000803
:101188001F3FCE70606660606E703FC81F00000031
:1011980000000000000000087F7FCE60606660707D
:1011A800EC7F6F8060600060000000000000000EAF
:1011B8001F3FE67060666070EE3F1F6600006600C5
:1011C800000000000000000C373FE63830003030E7
:1011D8000030300030000000000000000000000077
:1011E8003F7F80607F083F0188017F803F000000CB
:1011F80000001818001818007F7F00181800181829
:1012080000181F880F000000000000000000000602
:1012180060606660606660606E703FE61F00000098
:10122800000000000000000660606C3030C819192A
:10123800800F0F00060000000000000000000006FC
:10124800666666666666666F6C3F39C810000000A1
:10125800000000000000000C6071C83B1F000E1F5A
:10126800083B71CC60000000000000000000000C8A
:101278003030C81919800F0F000606000C0C001832
:10128800000000000000000C7F7F800306000C189F
:1012980000307FCC7F00000003CC070E000C0C0050
:1012A8000C1C00381C000C0C000C0E0C0703C000B2
:1012B80006000606000606000600000606000606EA
:1012C80000060600060000003C003E07000303007D
:1012D80003038C0103800303000307003E3C000066
:1012E8000000001C6C366380000000000000000055
:1012F80000000000000000000000000000000600E0
:101308000F198C306066607FEE7F000000000000DF
:1013180000001E0060077E0700F01EF060F77EF7F1
:10132800FBDE1F00E007FF0700F81FF8E0FFFFFFE4
:1013380000000F00E002EF0200780F78E07AEF7A01
:10134800F7BD1F00E007FF0700F81FF8E0FFFFFFE9
:10135800230000020000100000050000FE05001830
:101368002800FE0400182400F90F00F80F00700090
:101378001F71802372802A73111574111C75151B37
:1013880076151A77181C781521050100FF00000052
:10139800013F2B0200100721000001000723001065
:1013A8000000FD3000073300113068FF0000E50041
:1013B8008000010001000102000403301004000055
:1013C8000802020900000A00000C00000D00000FCE
:1013D8000000100000110700120000130000FD506B
:1013E8000010B01B110700FD5000121E01FD500037
:1013F80013001F291F00FD5000200000210000FEDF
:1014080001002B0C00FE00002B20003000003106EC
:101418000332000235070136040437060638050191
:101428003907073C00063D070850000051EF0052FD
:101438000000533F01FE01006000A7FE00006000AD
:10144800276101006A00008000008100008200001E
:10145800830000840000850000901000920007932C
:101468000700953F03970000980000070100FD5012
:1014780000072100072300FD5000077301FD00004D
:1014880000000000007C0000000001C000C0000057
:101498000000000000000000038380000000063008
:1014A80007387FFFFC3FFFE007FFFFC00400F000A4
:1014B8000000080E0808FFFFF8FFFFFC0FFFFFF011
:1014C80008000E00FC1F1001F018FFFFF9FFFFFED7
:1014D8000FFFFFF0100001810330D0000019FFFF5B
:1014E800F3FFFFFE1FFFFFF8100000C100C0D0008F
:1014F8000039FFFFE7FFFFFE1FFFFFF81000006243
:101508000000C80000300FFC07FE0FFE1FF81FF890
:10151800200000320000C80000601FFC07FE0FFC1E
:101528003FF83FF8200000340000C80000601FFCAE
:101538000FFC1FFC3FF03FF820000034000188003A
:1015480000C01FF80FFC1FFC3FF03FF030000064A4
:101558000001880000C03FF80FFFFFF87FFFFFF091
:10156800100003E40001880001803FF81FFFFFF826
:101578007FFFFFE01C000F840003080001803FF09C
:101588001FFFFFF87FFFFFC004003C0400031000AA
:1015980001807FF01FFFFFF07FFFFF000200700453
:1015A8000006100003007FF03FFFFFF0FFFFFC0084
:1015B800020060040006200003007FE03FF07FF097
:1015C800FFE0000002006004000C20000300FFE0C0
:1015D8003FE07FE0FFC000000200C004000C4000B4
:1015E8000300FFE07FE0FFE1FFC000000200C0044D
:1015F800001880000100FFC07FE0FFE1FFC000008D
:1016080001018002003080000181FFC07FC0FFC15E
:10161800FF80000001018002007100000181FFC00D
:10162800FFC1FFC3FF800000010300020063000048
:101638000181FF80FFC1FFC3FF8000000103000399
:1016480000C2001E0183FF80FF81FF83FF000000AE
:10165800018600010381807F0303FF81FF83FF87E9
:10166800FF00000000CE0001C70080E18703FF01F2
:10167800FF83FF87FF000000007C00007E00F780EA
:10168800EE07FF01FF03FF07FE0000000030000027
:1016980038003F007C07FF03FF07FF0FFE00000034
:1016A80000000000000000000007FE03FE07FF0F17
:1016B800FE0000000000000000000000000FFE0017
:1016C8000007FE000000000000000000000000000D
:1016D800000FFE00000FFE000000000000000000E8
:1016E80000000000000FFE00000FFE0000000000D8
:1016F8000000000000000000001FFF00000FFC00B9
:10170800000000000000000000000000001FFFFFB4
:10171800FFFFFFFFFFFF00000000000000000000C7
:10172800001FFFFFFFFFFFFFFFFF0000000000009A
:1017380000000000003FFFFFFFFFFFFFFFFF00006A
:101748000000000000000000003FFFFFFFFFFFFF58
:10175800FFFF00000000000000000000003FFFFF46
:10176800FFFFFFFFFFFE0000000000000000000078
:10177800007FFFFFFFFFFFFFFFFE000000000000EB
:1017880000000000007FFFFFFFFFFFFFFFFE0000DB
:101798000000000000000000007FFFFFFFFFFFFFC8
:1017A800FFFC0000000000000000000000FFFFFF39
:1017B800FFFFFFFFFFFC000000000000000000002A
:1017C80000FFFFFFFFFFFFFFFFFC0000000000001D
:1017D8000000000000FFFFFFFFFFFFFFFFF8000011
:1017E8000000000000000000007FFFFFFFFFFFFF78
:1017F800FFF800000000000000000000007FFFFF6D
:10180800FFFFFFFFFFF800002564002B003E3E00AD
:101818006B65696E204B726564697400436F6C6F09
:1018280072546F75636820567320312E343700491F
:10183800443D00202047433D0020203531326B00D5
:101848004B653A00496E3A0043616C696272617493
:10185800696F6E004F4B00546F74616C20002D2D22
:101868002D2D0054696E79200054696E79206261CB
:1018780064006B65696E20454570726F6D004D4F51
:1018880044554C2053544F50004461746120006902
:101898006E697400533F000066616C73636865721B
:1018A8002054697363682000546973636820766FF5
:1018B8006E204B20004665686C6572200056656E88
:1018C80074696C20616B7469760054696D656F7515
:1018D8007400435349204E722000436F6465200012
:1018E8006B65696E204B72656469740066616C7320
:1018F8006368657220546973636800546973636828
:1019080020766F6E204B0058313939313030005015
:101918004C5520203A00436F6465203A005469739F
:101928006368203A004D42005053004B656C6C6E62
:10193800657220004D31004F310053500043500074
:1019480044590062757379004D50002067657370C3
:1019580065727274002564004162726563686E7511
:101968006E67004B656C6C6E65722000546F746115
:101978006C004D6F64756C2000202000433F00739D
:10198800656300496D7000504C553A2000537061F2
:101998007274653A20005072313A20005072323A1F
:1019A800200046756E6374203A20005479703A20FE
:1019B800003A20563A2020302B2030003A003A20B6
:1019C800544F3A20003A2050733A200053703A009E
:1019D8004B204D6F6465204A6F62204A6F62466CE7
:1019E800616773004B20004D6F646520004A6F6289
:1019F800202000562020204572722050676C204914
:101A08006D7020544F005620005061757365004B6F
:101A1800656C6C6E65723A004D49004D42004D434D
:101A2800004D50004D4C0074657374202E2E004FED
:101A38004E00253032580025303458002533642EA6
:101A480025303264002535640025640025326400A1
:101A580025336400444400004B23004253004221D4
:101A680000424600542300544F004952004D5A008A
:101A78004251004252004353005653005643004916
:101A88004C00426600004B230054230042450043AB
:101A98004500424100445300434200235022415331
:101AA8004349492D492F4F222C22312E3030222CE8
:101AB800323030382D30312D30313B00234822452B
:101AC800636F222C22312E3030222C323030382DC8
:101AD80030312D30313B0023532245636F222C22B5
:101AE800312E3030222C323030382D30312D3031FB
:101AF8003B00504F00504632333B505500256400A0
:101B08002B302B303B0025640025303258002564EB
:101B18002E253264004F4E0001002D4E414E00002C
:101B28000100DC0E201B0000F894EE27ECBBF1E06E
:101B3800F5BFE5BFE0936C00F8E1F1BDE1BD8DE0D4
:101B4800A2E0BB27ED938A95E9F780E090E1A0E059
:101B5800B1E0ED930197E9F7E8E2FBE18591959112
:101B6800009761F0A591B59105901590BF01F0011E
:101B780005900D920197E1F7FB01F0CFEFEFEDBF74
:101B8800E0E1EEBFC0E0D3E00C9449170A9902C027
:101B9800E1E00895E0E008951A931FEFE2E00E9463
:101BA8003B6CE3EFE1BB85E38A95F1F7E0EFE1BB3E
:101BB800E4E4E09374000E94446C0E94EB66E03019
:101BC80091F4E981EE0FE0520E94496C41F4EDB7BF
:101BD800FEB7FA93EA931F930E944E6C1F910E94DE
:101BE800FC660E94526CE0E0E09371000E94526C27
:101BF800E12F70C30E94576C10E01430F0F400E03D
:101C08000430C8F4A12FECE30E945B6C0E945F6C67
:101C18000E94646CE15BFF4FFA93EA930E94696C3F
:101C28000E94696CE02FEE0FEE0FE10FEA930E941D
:101C3800264C0F5FE5CF1F5FE0CFECE0E0930F0489
:101C4800E0E0E09310040E946E6C0E94BF490E947D
:101C5800746C0E947243E030D9F40E947B6C0E943D
:101C68007B6CE6E9F0E00E94806C0E947B6C0E942D
:101C78007B6C0E9410470E948A6C0E94DB410E9484
:101C8800916C0E94DB41EEE1F0E00E94986CE1CF9C
:101C98000E9475433FC4E881E03011F01C9A01C0EE
:101CA8001C9832C00E947B6C0E947B6C0E949C6CCA
:101CB800EFE3F0E00E94A16C08951A93A091040349
:101CC800A43081F4E0910F04E093100410E0183080
:101CD80048F4ABE01A9FF001E852FD4F0E94A76C50
:101CE8001F5FF5CF42C0A0910403A43039F4E88106
:101CF800E0931004E0E0E0930F0406C0E881E0936D
:101D08000F04E0E0E0931004219608951A93A0913F
:101D18000403A43031F110E0143018F50E94AB6CC4
:101D28003196E491EA93DFDFE0E0E09310040E944B
:101D3800B46C3896FA93EA93EBE0F1E00E94B76C42
:101D48000E94B76CFA93EA930E94AB6CE491EA9311
:101D58000E94AB6C32960E94BC6C0E9433441F5F99
:101D6800DBCF0E94BF6C0E94C46C199108952A971A
:101D78000E94A67D30E010E000E047ED50E028E04A
:101D8800E091190CE03019F020E149E650E03217F3
:101D9800F0F50E94C86CE13098F10E94C86CE038F8
:101DA80070F0EEE00E94CE6CE0E1F8E1FA93EA937D
:101DB8000E94C86CEF70EF5F0E94D66C07C0ECE021
:101DC800EA9391DFE8E5EE83E0E0EF830E94B46CEC
:101DD80038960E945F6CE7E3F0E00E94207BE40FF6
:101DE800F51F0E94B76CFA93EA93EDE2F0E0FA93DC
:101DF800EA930E94C86CEA930E947B6C0E94E06C94
:101E08001F5F143011F410E00F5F3F5FC0CF0E94D6
:101E1800BF6C0E94BF490E94AD7D619608950E94E3
:101E2800E66CECE0EA935FDF0E946E6CEBE0EA930D
:101E38005ADF0E94EA6C0E94EF6CEAEAF0E00E9426
:101E4800F46CE091390CF0913A0CE491EA93E0914A
:101E5800390CF0913A0C31960E94FB6C0E94334485
:101E680001E00E94FE6C0E94016D11F00F5FF9CF36
:101E78000E940F6D031718F4E0E0E093C0050E947C
:101E88000F6D11E00E94166D0E94016D11F0153062
:101E980008F021C00E94EA6C0E94196DE0E4F0E0AD
:101EA8000E94207B3496FA93EA93E2EEF0E00E94D7
:101EB800F46C0E94166D0E941C6DE491EA930E94D6
:101EC800166D0E941C6D31960E94FB6C0E94334473
:101ED8003F5F1F5FD7CF0E94C46C0E94AF7D29C4AB
:101EE80027970E94A67D22E354E0A0910403A43022
:101EF80011F426E453E010E0143010F00C94CF0FE6
:101F080000E0051710F00C94CD0FE12FEE0FEE0F47
:101F1800E00F3E2F0E94166D0E94286D3196E491C5
:101F28000E94CE6C0E94166D0E94286D3296FA931C
:101F3800EA930E943A69ED85E03039F4AF81A13225
:101F480010F4E0E0EF83E0E0E887A02FBB27E22F62
:101F5800E85FF0E00E94207B3896FA93EA930E94AB
:101F6800196DEAE3F0E00E94207BE55BFF4F0E94D9
:101F78002D6D0E94B76CFA93EA930E94166D0E9429
:101F8800286DE491EA930E947B6C0E94E06C0F5FDD
:101F9800B8CF1F5FB1CF0E94C46C0E94AD7D2E9652
:101FA800089522970E94326DA13059F40E94376D2E
:101FB800ABE2B1E00E944B7B2E2F57E1E2ECF0E060
:101FC80008C00E94376D0E943B6D2E2F53E0E7EE4C
:101FD800F0E0EE83FF830E94406DA0911908A130C4
:101FE80081F4E9ECF0E00E94576D0E945E6D0E945A
:101FF800636DEBE2EA93E3E1F8E10E94BC6C0E94B6
:102008003344E3E0F0E00E94576DEA85FB850E94C7
:10201800696D0E946C6D0E94706D3F5FE091C10B0D
:10202800AFEE0E942A7BF0E0EE83FF8311E0E0919F
:10203800C20B1E17B0F500E0E091C10B0E1778F542
:102048000E94766D49F10E947D6DE09310040E9414
:10205800FE6CAE81BF810E94207B33960E942D6D5D
:102068000E94196D0E94207BDF010E94876D0E94EB
:102078008A6DEA85FB8534970E94696D0E946C6DB4
:102088000E94706D3A930E947B21EF3F29F0ADE0EA
:102098005A9FF0010E948F6D3F5F0F5FCDCF1F5F8A
:1020A800C6CF0E94BF6C0E94C46CC6C022970E9413
:1020B800A67DE2E5F7E0EE83FF8340E0443190F44B
:1020C800AE81BF8111960E94976D1396EFEFEC9346
:1020D800AE81BF81EC93EE81FF813496EE83FF835E
:1020E8004F5FECCFE091C10BA0EF0E942A7B2E2F0F
:1020F8000E94376DA0E4B1E00E944B7B5E2F0E94E6
:10210800406D21FE21C00E949C6D0E949C6DEFEAEB
:10211800F0E0FA93EA930E94A16D0E946C6D0E9410
:10212800706D0E94746CE6EBF0E00E94A76D0E944F
:102138005E6D0E94A16DEFE7EA93E5E1F8E1FA939D
:10214800EA93E0E0F0E011C00E949C6D0E949C6D53
:10215800E8EEF0E0FA93EA93E52F0E94AA6DFA936D
:10216800EA930E946C6DEAE8FBE0FA93EA930E9416
:1021780033443F5F11E0E091C20B1E1710F00C943E
:102188001A1100E0E091C10B0E1710F00C94181111
:102198000E94766D11F40C941511A0919A0BE0E849
:1021A800EA23E03821F0A091E20BA23019F40E9452
:1021B8007D6D0AC00E94AD6DE03011F4E0E001C011
:1021C800E8E0E0930F04E7E0E0931004A02FBB27BA
:1021D800E22FF0E00E94207B3396FA93EA930E9464
:1021E800876D0E94196D0E94207B33960E94696D4D
:1021F8000E94A16D0E946C6D0E94706D4E2FA0917F
:102208001E08E32F0E94B26DEA0FFB1F43833A9327
:102218000E947B21EF3F29F0ADE04A9FF0010E9428
:102228008F6D3F5F0F5FAECF1F5FA5CF0E94BF6C62
:102238000E94C46C0E9478360E94AD7D289608954D
:10224800E1E0E0930D04E2E0E0930E04E0E0E093C7
:102258001004ECE0E0930F04E4E5F3E00E94A76CBF
:10226800EAE0E0930F04E2E4F3E00E94A76C0E9426
:10227800BF4908951A93A981A43029F4A0E021FC4C
:10228800A1E0A03009F426C0E9810E94B96D04904C
:10229800E9810E94BF6DE491A02DAE1BA2501A2FB8
:1022A8000E94746CE4EBF0E0FA93EA93EB810E94ED
:1022B800BF6D0E94D37B3296FA93EA93EAE3F0E08B
:1022C8000E94C76DEFE7EA93E5E1F8E10E94BC6C74
:1022D8000E9433441881229608950E94576CE0E0CA
:1022E800EA930E94A8190E94AD6D0E2FECE2F2E06D
:1022F8000E94D37B33971E2F0E947B6C0E947B6CBD
:102308000E949C6C0E94CE6D0A930E94264C0E94EB
:10231800696C0E94D36D0E942B47E2E0E0930E04A3
:10232800E091980BEF70E09310040E94D86DEFE0F5
:10233800E0931004AA81A13051F40E94E06D0E943C
:10234800EF6C0E941047E8E1F8E10E94E56D21FE7C
:102358000DC0E4E0EA938EDFE4E3F2E00E94E96D69
:10236800E6E3F2E00E94E96D0E94DA49A6DC80C04B
:10237800E8810E94BF6D0E94E96DEA810E94B96DF3
:102388000E94E96D0E946847E881EA9373DFBFC144
:102398001A930A93EC81EA93EBDF1AEEEC810E9420
:1023A800B96D0490EC810E94BF6DE491A02DAE1B25
:1023B800A2500A2FAC81A43029F4A0E021FCA1E0AE
:1023C800A03009F409C01EEAAA81BB811B96E0E08F
:1023D800EC93EC81EA934EDF0E947D6DE09310044C
:1023E800EC810E94EE6DFF93EF930E949C6DEE814D
:1023F8000E94BF6D0E94D37B31960E94C76D0E94D8
:10240800FE6CFA93EA93EC85E058EA930E947B6CA1
:102418000E94F46D0E943344AF91BF91EC93EC811C
:102428000E94BF6D0E94E96DEE810E94B96D0E9405
:10243800E96D0E94DA4919810881259608950E945C
:10244800F96D0E943B6D8F010E947B6C0E947B6C32
:102458000E949C6C0E94FC6D0E94E06D0E941047D7
:10246800EA81EA930E94A8190E94D86D0E94036E1F
:1024780019810881239608950E94F96D0E943B6D89
:102488008F010E947B6C0E947B6C0E949C6C0E9456
:10249800FC6D0E94E06D0E941047EC81FD810E9456
:1024A800E56DAA81BB810E949C7D24F4A030E0E107
:1024B800BE070CF006C0EA81FB81FA93EA930E94FA
:1024C800E241AA81BB81A130E0E1BE0724F0A0303F
:1024D800E1E1BE070CF00AC0A6EEBBE0EA81FB8191
:1024E800E150F0410E940D6E0E94156E0E94036E2D
:1024F80019810881269608950E94F96D0E943B6D06
:102508008F010E947B6C1A930A930E94DA49E0E0DB
:10251800E0933B0C099119910895E881EA930E9490
:10252800A8190E945720E03051F10E941B6E0E94AA
:102538007B6C0E941F6E0E94D86D0E94236EE881FA
:10254800EA930E94C221E8830E94276E3B9734F0E9
:102558000E94276E0E94326EE9E40BC0A6E0B7E045
:102568000E94366E0E94396E0E943E6E0E94436E33
:10257800E3E7EA930E94AE46E2E0E0930E04C7C0A8
:102588000E94EB68E0E0E0930F04A0910403A430FC
:1025980019F4E0E6F3E002C0ECE6F3E0FA93EA931C
:1025A8000E94134408950E9437470E94EB680E94D6
:1025B800FE68E1E0E0930D040E941B6EE6E0F0E0A7
:1025C8000E94476EE4E2F8E10E94E56D0E947B6C90
:1025D800E7E0F0E00E94476EE7E3F8E10E94E56D6E
:1025E8000E944B6EEA930E94ED41EBE3F8E10E94F2
:1025F800E56DE0910403EA930E94ED41E1E4F8E11E
:102608000E94E56D08952A971A930A930E947B6C9D
:102618000E947B6C0E949C6CE4E6F0E00E94A16C36
:1026280000E010E01530B0F4053020F40E94506E40
:10263800E03009F40DC00E947B6C0E94FE6C0E9481
:10264800476E0E94576E0E94506E0E945C6E0F5F2C
:102658001F5FE8CF0E945E6E0E941047E8E4F8E131
:102668000E94E56DE0913108EA930E94ED410E94D5
:10267800EA6C0E94E06D0E941047ECE4F8E10E94C9
:10268800E56DE0912306EA93E5E0EA930E94BD41F7
:10269800E091190CE03079F10E94EA6C0E94D36D48
:1026A8000E941047E09128060E94616E0E949C6D6E
:1026B8000E941047E0912806E295EF70E695E695AE
:1026C800AE2FE0912906EE0FEE0FEA0F0E94616E21
:1026D8000E94EF6C0E941047E0912906E295EF7086
:1026E800AE2FE0912A06E295E07FEA0FEA93E6E052
:1026F800EA930E94BD411981088181C1E881E064A3
:10270800E7B9369A349BFECF349AE4B1F5B12196F5
:102718000895E881F981AA81BB81AE17BF071CF42F
:10272800EA1BFB0B06C0A881B981EA81FB81EA1B81
:10273800FB0B2496089528970E94A87DEFE0E0936C
:102748006100E1E0E09362000E94446CE5E0E09300
:1027580061000E94446C0E94676EE0936F05F093DD
:102768007005E0917B05F0917C05E0936D05F09391
:102778006E05E1E0EA93C2DFE0937B05F0937C0508
:10278800EFE0E0936100E8E0E09362000E94446CAF
:10279800EAE0E09361000E94446C0E946C6EE09352
:1027A8006B05F0936C05E0917905F0917A05E0935B
:1027B8006905F0936A05E0E0EA93A0DFE093790504
:1027C800F0937A050E946C6EA0916B05B0916C0530
:1027D800EA0FFB1FA0917905B0917A050E94716EEE
:1027E8008F010E94676EA0916F05B0917005EA0F86
:1027F800FB1FA0917B05B0917C050E94716E9F0123
:10280800E0916B05F0916C050E94786EFF93EF9351
:102818000E946C6E0E94786EAF91BF91EA0FFB1F09
:10282800FF93EF93E0917905F0917A050E94786E15
:10283800AF91BF91EA0FFB1FE0937505F093760502
:10284800E0916F05F09170050E947E6EFF93EF9303
:102858000E94676E0E947E6EAF91BF91EA0FFB1FC8
:10286800FF93EF93E0917B05F0917C050E947E6ECB
:10287800AF91BF91EA0FFB1FE0937705F0937805BE
:10288800A0917505B0917605E4E1F0E00E94F27A36
:102898000E2EA0917705B0917805E4E1F0E00E9452
:1028A800F27AE02919F00E94E345A7C00093710568
:1028B800109372052093730530937405A0916405F5
:1028C800A63428F4E0916405EF5FE09364050E9464
:1028D800846E989724F40E94896E98970CF00EC025
:1028E800A0916405AA3019F4E1E0E0936105A09194
:1028F8006405A83219F4E2E0E09361050E94846E51
:10290800999724F00E94896E99970CF476C0E0910B
:102918006705EF5FE09367050E948E6E0E94846EE4
:102928000E94936E0E949A6E0E949F6E0E94257B61
:102938007F936F93FF93EF93A2E0B0E00E94EE7B4A
:102948000F010E948E6EDF01F001EA1BFB0BAF91B5
:10295800BF918F919F910E94A86E0E949A6E0E94CB
:10296800AD6E0E94896E0E94936EEC83FD836E8328
:102978007F83AC81BD818E819F81EFE3F1E060E0D0
:1029880070E00E94257B7F936F93FF93EF93A6E0FF
:10299800B0E00E94EE7B0F010E94AD6EDF01F001F6
:1029A800EA1BFB0BAF91BF918F919F910E94A86E7C
:1029B800EC83FD836E837F83E0911204E03049F459
:1029C800E885F985E0935905F0935A05EC81FD8176
:1029D8000AC0EC81FD81E0935905F0935A050E94E5
:1029E8009F6E0E94BA7AE0935B05F0935C050E94A3
:1029F8008A6C0E94916C0E946B450E94AF7D2C9658
:102A080008951A930E943747E2E0E0930E04E2E348
:102A1800F0E00E94B76C0E94B26EE0E5F8E10E9417
:102A2800E56DE4E1EA930E946641E0E9F1E00E9485
:102A3800B66EE4E1EA930E946641A0916705A13071
:102A480010F0A895FACF10E0143010F00C9484150B
:102A5800E2E0E0930D040E94BA6EDF010E94E96D86
:102A6800FD0132960E94E96D0E942B470E94BA6EC2
:102A78003496E491EA930E94AE46E1E0E0930D04B7
:102A8800A0916705AF3110F4A895FACFEAE0EA9370
:102A98000E9466410E94BA6EDF0135960E94D37B80
:102AA800BF01FD010E94C06EDB010E94FE7BE2E3D4
:102AB800F0E0FA93EA930E94196DE8E2F0E00E94D0
:102AC800207BE65AFF4F0E94B26E0E94BA6E0E94A7
:102AD800C06E0E94326EA0916705AE3110F0A895C5
:102AE800FACF0E94BA6EDF010E94E96DFD013296AD
:102AF8000E94E96DE8E1F0E00E94806C1F5FA4CFBE
:102B0800E2E3F0E0FA93EA93EAEFF0E00E94B26EB3
:102B1800ECE5F8E10E94E56DE0EDF7E00E94B66EA5
:102B28000E9437474DC10E94C76E0A93E4E6E2BF90
:102B380078940E942D45FFDDE6B3AFEFEA27E093D6
:102B48003108A2E6BBE00E94D66EE091620BE77006
:102B580031F4A0910A04E0E4EA27E0930A04E09142
:102B6800620BEF7131F4A0910A04E3E8EA27E093DD
:102B78000A040E94B9660E946322E2B3EF700E2E27
:102B8800A0911408B0911508EFE0F0E0AE27BF2738
:102B9800EA23FB230E94D37AE029E2BBE0911408E0
:102BA800E07111F41D9A01C01D980991199115C081
:102BB8000E94C76EE6E0E4BDE0B1E295EF70AE2F8B
:102BC800E0916300E071E15FEA231E2F0E94CE6D61
:102BD8000E943A220E9493661991E991EFBFF991F8
:102BE800E991B991A9919991899179916991F9900E
:102BF8001990099018950E94BD650E9443660E942D
:102C080075510E94931F08951A93A8950E944443F2
:102C1800E13011F00C946916E091C605E1501E2FC1
:102C2800A091C505A13021F40E94DC6EE03009F4C2
:102C38000CC0ADE01A9FF001E15FFC4FBF01E081DD
:102C4800E260DB01EC930E94E36EA091C505A2301F
:102C580011F0A43089F40E94DC6EE093DB050E9439
:102C6800E86E31F0FD01E15FFC4FE081E27009F4AC
:102C780003C01A930E94F16EA091C505A33019F400
:102C88001A930E941428A091C505A53029F4E09153
:102C9800C605EA930E944B28A091C505A830A9F45F
:102CA800E0E0EA93E091C605EF77EA930E947B198A
:102CB8001E2F1F3F51F0E0E0EA930E946641E12F8A
:102CC800E058E093DB05E0932D06E0910A04E078F4
:102CD800D1F0E0910A04EF77E0930A040E94034AD6
:102CE800E0910A04E07131F0E0910A04E270EA939D
:102CF8000E941546A0913208A13328F0E2E0EA9339
:102D08000E94D00D1E2FA0913B0CA13039F4E09108
:102D18003C0CF0913D0C0E94F56E09F401C0ECDB0F
:102D28006ADF4EC01A930E943747E1E0F0E00E9444
:102D3800BC6C0E94104710E00E94FF6E0E947B6CE2
:102D48000E94CE6D0E941047E0912108E03049F4BE
:102D5800EFE5F8E10E94E56D0E94056F0E94436E61
:102D68001E5FA0912108A130F0F0E0912108E15008
:102D7800EA930E94D719A091B30BAD3229F40E94AF
:102D88000E6F0E94987D79F0E3EBFBE00E94156ED0
:102D9800E6E0F0E0FA93EA930E941B6F0E940E6F40
:102DA8000E94436E1E5FE0912108EF5FE0932108C7
:102DB8001C3020F4A0912108AB3008F001C0BECF30
:102DC800199108951A930E943747E981E03019F460
:102DD800E0E0E0931E08A981A230A9F410E0A091D8
:102DE8001E08A13010F01C3008F00DC0E0911E083C
:102DF800E150E0931E080E941F6F19F40E942D6F86
:102E080009F01F5FECCF0E94FF6E10E00E947B6C00
:102E18000E94CE6D0E941047A0911E08A33608F5A7
:102E2800E0911E08EA930E94A8190E941F6F19F4E6
:102E38000E942D6FA9F00E94D86D0E947B6C0E94A1
:102E48001B6F0E94386F0E94326EE8E7EA930E9477
:102E5800AE460E94236E0E943D6F0E94436E1E5F25
:102E680005C0E6E6F8E10E94E56D1E5FE0911E08E8
:102E7800EF5FE0931E081C3020F4A0911E08A436D2
:102E880008F001C0C3CF0C94D81BE0E0E5BFE09385
:102E98006D00E0936C00EBBBEFEFEABBE0E0E8BB52
:102EA800E7BBE5BBEFEFE4BBE0EFE2BBE1BBE0E291
:102EB800E3B9ECEBE2B9E0E0E0936200E093610093
:102EC800EFE0E0936500E0936400E0E0E0BFE7E056
:102ED800E3BFE4E6E2BFE0E0E1BFEFBDEEBDEDBD7C
:102EE800ECBDE7BDE6BDEBBDEABDE9BDE8BDE093DD
:102EF8007900E0937800E3E0E5BDE6E0E4BDE0E0DA
:102F0800E3BDE0938B00EAE0E0938A00E0E0E09321
:102F18008900E0938800E0938100E0938000E2E17B
:102F2800E0938700E4E3E0938600E0E0E093850027
:102F3800E0938400E0938300E0938200E0936A00CA
:102F4800E0E3EABFE0E4E9BFE8BFE1E4E7BFE0E0CF
:102F5800E0937D00EBB9E8EDEAB9E6E0E09395008F
:102F6800E0E0E0939000E7E6E9B9E0E0E0939B0059
:102F7800E8EDE0939A00E6E0E0939D00E0E0E0935E
:102F88009800E3E3E0939900E0E8E8B9E0E0E0BD09
:102F9800E0E4E7B9E7E8E6B9E0B5EF7EE0BDE0E2F6
:102FA800E0937000E0E0E0937200E4E4E0937400E2
:102FB800EFE1E1BDEFE0E1BD0E943A5E78940E9446
:102FC800C24B0E940646E1E0EA930E944F0E0E941F
:102FD8004B6EE53128F0A9E0B0E0E0E00E94067C05
:102FE800E2DA21E030E0E0E0EA930E94D00DE093DD
:102FF8003208EAE0F0E00E94B66E3F5FA091320826
:10300800A43511F03A3008F001C0EDCF0E94E06D10
:103018000E94EA6C0E941047A0913208A43581F4FE
:10302800E1E0EA930E94D00DE0933208EBE6F8E184
:103038000E94E56DE0913208EA930E94AE4607C00F
:10304800E0E0E0933208E1E7F8E10E94E56D94D012
:10305800E03059F40E94E06DE9E0F0E00E94476E2C
:10306800EAE7F8E10E94E56D20E00E948E6E0F010C
:10307800A2E0B0E00E94EE7B0E161F0654F40E94F8
:10308800AD6E0F01A6E0B0E00E94EE7B0E161F06A3
:103098000CF0B7DC203071F40E94E06DEAE0F0E05B
:1030A8000E94476EE6E8F8E10E94E56DA8950E9447
:1030B800466FFCCF0E945F370E94E06DE9E0F0E0C8
:1030C8000E94476EE1E9F8E10E94E56D0E941D1C2F
:1030D800E03019F0E7E9F8E102C0ECE5F8E1FA932D
:1030E800EA930E94C5460E94CB66E1E0EA930E94FB
:1030F800664100E010E00436E0E01E0724F40E9478
:103108004366E03009F007C0EAE0F0E00E94B66EDE
:103118000F5F1F4FF0CF0436E0E01E072CF0A091A0
:103128006705AF3108F06DDC6FDD0E94BC320E948C
:103138004F1EFACFFFCF0E94496F17FD02C0103013
:1031480011F4E0E031C3E12F2FC30E94496F17FD4E
:1031580010E01A3008F41F5F0E94566F25C30E94C2
:10316800496F17FD02C0103011F4E0E01DC3115083
:103178000E94566FE1E018C31A930A9310E0E4E640
:10318800F0E00E94B66EA8950E94EB66E03021F44C
:10319800E0EA0E94616F09F002C001E001C000E0AE
:1031A8000E94FC661F5F003011F4153008F001C062
:1031B800E6CFE02F0991199108950E94666F11C416
:1031C8000E94666F0E94736F0895A881B9810E945A
:1031D8009C7D24F4A83EE3E0BE070CF005C00E94E5
:1031E800796F0E945E67E1C2E0E0DFC2A881B98121
:1031F8000E949C7D24F4A83EE3E0BE070CF005C0C5
:10320800EA81E03011F4EFEFEA830E94796FED81F3
:10321800EA930E948A6760C10E94A87D20E030E09E
:10322800283EE3E03E077CF4A8953A932A93CDDF45
:103238001E2F1F3F29F0EFEFEA933A932A93D6DF28
:103248002F5F3F4FEDCF0E94AF7D4FC01A930A9377
:10325800E0E0F0E0E0933E0CF0933F0CAA81A33647
:1032680068F40E94826FE55FFD4E8F010E94896FAE
:103278001A930A93EEE3FCE00E948C6FE0913E0CF7
:10328800F0913F0C27C11A931FEF1F5F1A93DEDFDF
:10329800A981BA81EA17FB0711F0143608F001C0BA
:1032A800F4CFE12F188118C11A930A93A091C10B8A
:1032B800E091C20BEA9FF001A0911E08EA0F0E2FC1
:1032C800043608F002E610911E08101758F41A93F5
:1032D800BDDFAA81BB81EA17FB0711F4E12F03C008
:1032E8001F5FF3CFEFEF19810881249608950E949C
:1032F800A67D10E0133618F50E94196DE8E2F0E09B
:103308000E94207BE050FE4EAF01E0EAEA93FA010A
:1033180070960E94906FEC713E2FE0EAEA93FA01F2
:103328003F960E94906F0E2FEF81E31719F4EE81FC
:10333800E01709F002C0E12F03C01F5FDBCFEFEFFA
:103348000E94AD7D289608951A930A93E091890BFF
:10335800AA81EA17C1F0A33668F40E94826FE05090
:10336800FE4E8F010E94946F0E948C6FEA81E09359
:10337800890B09C0EFEFE093890B0E949F6F0E94B1
:10338800A46FE093940BA6C01A930A930E94826FCD
:10339800E050FE4E8F01AA81A33620F40E94946F5C
:1033A8000E94736F97C01A930A93E091B20BAA8197
:1033B800EA17A1F00E94AE6F40F40E94BA6F0E9413
:1033C8008C6FEA81E093B20B09C0EFEFE093B20B88
:1033D8000E94C56F0E94A46FE093BD0B7BC01A9337
:1033E8000A930E94AE6F20F40E94BA6F0E94736F16
:1033F80071C01A930A93E091320CAA81EA1761F11D
:103408000E94CA6F18F50E94896F1A930A93E3E322
:10341800FCE00E948C6FEA81E093320CE0E0E093DC
:103428002B06A091340CA13020F0A091340CA830C8
:1034380008F00BC0A8EDBBE0E091340C0E94D46FFB
:10344800AE0FBF1FEC91E0932B0606C0EFEFE093A1
:10345800320CE0E0E093330C3DC01A930A930E94CB
:10346800CA6F40F40E94896F1A930A93E3E3FCE061
:103478000E94736F2FC01A930A93E0912D0CAA81B2
:10348800EA17C1F00E94D76F70F4E0EAEA930E944D
:10349800EF6C1A930A93EEE2FCE00E948C6FEA81CB
:1034A800E0932D0C07C0EFEFE0932D0C0E94E16F25
:1034B8000E940F690FC01A930A930E94D76F50F4A5
:1034C800E0EAEA930E94EF6C1A930A93EEE2FCE0BA
:1034D8000E94736F19810881239608950E94E16FF5
:1034E8000E940F69E881EF5FE0932F0CA0C1249739
:1034F8000E94A67D0E94E86F0E940F69AB85A130EB
:1035080010F0A13208F009C0EB850E94D46FA3E641
:10351800B0E00E94EF6F0E940070EB85E03059F533
:10352800E0E0EE83EF83E887E98740E050E020E0C1
:1035380030E02032E0E03E07B4F4D901E3E6F0E001
:103548000E94EF6F0E9400700E94386F4E0F5F1F3D
:103558000E943D6F0E9405700E94B57A0E940A7011
:103568002F5F3F4FE6CF40931D0C50931E0C0E94D7
:103578000F700E9414700E94AD7D2C9608951A93C6
:103588000A93AB81A13010F0A13208F01CC0EB8186
:103598000E94D46FA3E6B0E00E94207BDF01EA819D
:1035A8000E941D70E8E0F0E00E94207BE050F04DA2
:1035B8008F01E0EAEA930E94EA6C1A930A93EBE11E
:1035C800FCE00E94736F198108810C94911F0E947E
:1035D800A87DEC810E942170E83109F453C00E9453
:1035E8002670309729F00E9426700E942B70EC8379
:1035F8000E944B200E2F10E0101710F00C94461B61
:103608000E942F7074DFADE1BCE00E94D66EA091DD
:103618001F0CB091200C8091210C9091220C0E94DB
:1036280034700E94B57A0E9414700E942F70A7DF30
:10363800E0EAEA93EE810E94D46FEE0FFF1FE0509C
:10364800F04F0E94906FE270D9F4ED81E093230C63
:103658000E942670309751F40E944B6E0E943B7076
:10366800EF5EF84DDF010E94417002C00E94267093
:10367800E093240CF093250C0E9446700E944B7036
:103688001F5FBACF0E94AF7D269608951A930A93BA
:103698000E945170ECE2F0E00E9458700E945C7049
:1036A8000E94617010E01336D8F41A934DDEE09151
:1036B8002208EA931A931BDF0E946A70EA0FFB1F25
:1036C8000F010E946A700E947270DF01CB010E9494
:1036D8003D6F0E94B57AD0010E94CE7B1F5FE3CF79
:1036E800A0911908A330B9F500E00031A0F50E94B7
:1036F800FE6C0E94777069F510E01A3050F5E02FE3
:10370800E05DEA93ECE9F8E10E947C70E12FE05D6E
:103718000E948370E1F40E9488700E948F70EA0F03
:10372800FB1FFF93EF930E948F700E9472707F932C
:103738006F93FF93EF930E947E62AF91BF918F9139
:103748009F910E94B57AAF91BF910E94CE7B1F5F77
:10375800D4CF0F5FCACF10E01A3090F40E948F7058
:103768000E947270A0912908B0912A0880912B08B4
:1037780090912C080E94B57A0E9461701F5FECCF6F
:103788000C94D91F1A93A895A981A13268F40E94B4
:10379800E86F0E940F6910E0133630F4E981EA936C
:1037A8001A93EDDE1F5FF8CF1881229608951A93B9
:1037B80011E0113220F41A93E5DF1F5FFACF67C3D7
:1037C800E1E0E093330CE093340C31C0A8950E94FB
:1037D800C56FE6EAF3E0FA93EA930E94EA6C0E9466
:1037E8009670E093BB0B0E949F70E093BC0BE0E0E7
:1037F800E093BD0B1CC0A895E9E8FBE00E94A67009
:10380800E9E2F0E00E9458700E949F6FECE9F3E053
:10381800FA93EA930E94EA6C0E949670E093920BE6
:103828000E949F70E093930BE0EBE093980B219636
:1038380008950E94A67D0E94AB70E03228F0AAE0AD
:10384800B0E0E0E00E94067C00E0B7DCA091BE0B8F
:10385800B091BF0BA633E2E1BE0741F110E01A3088
:1038680030F41A93B3DF1A93BADD1F5FF8CF10E074
:10387800133630F41A93BFDF1A9386DD1F5FF8CF33
:1038880010E0103830F41A939BDF1A93E6DD1F5FBF
:10389800F8CF8DDFA9E0B0E0E0E00E94067CE6E327
:1038A800F2E1E093BE0BF093BF0B01E010E017329A
:1038B80010F00C94B01C0E94B0709F010E94B07070
:1038C800AF010E94BA703496E491E03011F0E13013
:1038D80069F4D901AC910E94BA703596E491EA175F
:1038E80020F40E94BA700E94C17034C0E23091F492
:1038F800DA010E94C47BE031A7E2FA0714F4FF233F
:1039080042F40E94BA7036960E94D37BDA01ED9396
:10391800FC9320C0E33049F4D901AC91AF3F21F4C6
:103928000E94BA700E94C17015C0E43099F4D901A0
:10393800AC91AF3F79F400E00E94BA703596E491FB
:103948000E1740F40E94BA700E94C1702F5F3F4F5B
:103958000F5FF2CF1F5FABCF33DC10E0153060F4A0
:103968001A9389DDA0912E0CA63020F01A93B6DDAB
:103978001A93A1DD1F5FF2CFE02F0C946121E8813B
:10398800EF5FE883A881A43610F0E0E0E883E881DF
:103998000C94DA210E94366EA5E0B0E00E94207BEC
:1039A80030960C94DA21A091360CBB27E091350CA7
:1039B800A6C0F9DF329774F00E94C670E091350C0A
:1039C8000E94CD700E94736FE091350CEA93D7DFA7
:1039D800E093350C08950E94C670E091360C0E9461
:1039E800CD70FA93EA930E94AB670895E3E2FCE096
:1039F8000E94D5700E94C670E091360C0E94CD706E
:103A08000E94736FE091360CEA93B9DFE093360CAD
:103A180008950E94A87DE0E0E093350CE093360C11
:103A280010E030E0343680F5A8950E94C6703A93CD
:103A3800B1DFFA93EA93E3E2FCE00E948C6F00E0C6
:103A4800A091230CA13010F0A03808F001C001E0CB
:103A5800E12FE03041F4013029F43093360C3093F3
:103A6800350C11E00FC0E13031F4003019F4309317
:103A7800350C12E007C0E23029F4013019F4309314
:103A8800360C13E03F5FCECF46C21A93A091CF0BFE
:103A9800A870B9F010E0E981FA810E94196DAE179B
:103AA800BF077CF4ED81E093230CEB81FC81E851A6
:103AB800FC4F0E94DC70E0E0F0E00E944B701F5F5A
:103AC800EACF18810C946321E881EF5FE883A8812D
:103AD800A43610F0E0E0E883E8810C94DA21E8816C
:103AE800E150E883A881A43610F0E3E6E883E88192
:103AF8000C94DA21A091380CBB27E091370CF0E048
:103B080031960E94E170EC59FF4FDF01E4E6F0E0E6
:103B18000E947D7B08950E94366EA5E0B0E00E9469
:103B2800207BE050FE4F0C94DA21E8E2FCE00E9492
:103B3800D570E881EA93BBD10C94DA211A936CDB37
:103B4800E1E0E093860BA3C1A89510E0143680F459
:103B58001A93A6D1A091280CAF3F31F40E94E670C9
:103B6800AF3FEFEFBE0711F01A93DFDF1F5FEECF15
:103B78000E94EB70689420F88AC10E94A87D109179
:103B8800380CAD81AA23CAF5E091370CE11719F07A
:103B9800AD81AA230AF030C01A9382D10E94E67040
:103BA800EE81FF81EA17FB0729F4E885A091280C2C
:103BB800EA1709F01EC00E94F170EC81FD810E9495
:103BC800BF7AEA17FB0744F40E94F6700E94FF7060
:103BD800E0E0EC83ED830BC00E94F670EC83FD837C
:103BE800E0E0F0E00E94FF70E0E0E093280C1A9318
:103BF8005ED10E940471C8CF46C0E091370CE1172E
:103C080029F0AC81BD810E949C7D0CF01BC01A93E9
:103C180047D10E94E670EE81FF81EA17FB0729F47D
:103C2800E885A091280CEA1709F009C00E94F670EF
:103C38000E94FF701A933BD1E0E0EC83ED830E9471
:103C48000471DBCFAC81BD810E949C7D1CF452DFE6
:103C580033970CF418C0E885E093280CEE81FF81B7
:103C68000E940971EC81FD810E94FF70E091370C80
:103C7800EA931DD1E091370CEA9326DFE093370CE5
:103C8800E0E0EC83ED83689420F8EC81FD810E94EC
:103C9800AF7D299608951A93A091400CA03059F44D
:103CA800E091430CF091440CFA93EA93E8EBFBE0C3
:103CB8000E940E7109F40BC0E1E0E093400CE09122
:103CC800370CE093420CE091370CE093410CA09143
:103CD800400CA13011F00C94CD1EE091380CA0914D
:103CE800420CEA1711F40C94BE1EE091420CEA93C0
:103CF800F6DEE093420CEA93D3D0A091280CA130D1
:103D080010F0A03808F035C0E091410CEA93E7DEE6
:103D1800E093410CA091420CEA1759F1EA93C7D0FD
:103D2800E091E20BE030E9F410E01530D0F4ABE0BC
:103D38001A9FF001DF01E352FA4FE081E03049F0C9
:103D4800FD01E452FA4FE081AE2FE091420CEA17F0
:103D580009F005C00E941471A091410CA0831F5F57
:103D6800E4CFE8E2FCE00E94D570E091420CEA93CF
:103D78009ED00FC0E091410CE093380CE0E0E09356
:103D8800400C689420F80E94C568E093430CF093B7
:103D9800440C7DC01A93A8951091380CE091370C0B
:103DA800E117C1F00E941A710E949C7D64F4EB81B6
:103DB800A091280CEA1739F40E94E670E981FA818B
:103DC800EA17FB0709F003C0E12F1881A6C00E947B
:103DD8000471E4CFEFEF1881A0C00E94F1700E9437
:103DE8009C7D84F4E0912B06E87031F4E0912F0873
:103DF800A091280CEA1731F40E941E710E942B70C2
:103E0800E33608F001C05CC10C943822A895E09113
:103E1800370CA881EA1761F0E8810E94237119F034
:103E2800E8810C94DA21E881EA934EDEE883EFCF4B
:103E3800EFEF0C94DA211A93A8951091380CE091C1
:103E4800370CE117E1F00E941A710E949C7D8CF4F6
:103E5800E0912B06E87031F4E0912F08A091280C2E
:103E6800EA1739F40E94E670E981FA81EA17FB073C
:103E780009F002C00C941F220E940471E0CFEFEFFA
:103E88000C9420221A931091380C1A93BFDF1991C1
:103E98000895E881EA9318DEE883EA93B7DF86C2DB
:103EA8000E94C6700E942A710E948C6F7FC20E9475
:103EB800C6700E942A710E94736F78C20E94A87D02
:103EC8000E94EB7010E030E0343628F5A8953A935C
:103ED800E7DF00E0A091280CA03808F401E0E12F0A
:103EE800E03041F4013029F43093380C3093370C2A
:103EF80011E00FC0E13031F4003019F43093370C81
:103F080012E007C0E23029F4013019F43093380C7C
:103F180013E03F5FD9CF0E94AF7D249608951A938E
:103F28000A93A0911908A43009F43FC010912F08F2
:103F380000914F0CE0913108E03059F0E0932F08E0
:103F4800689424F80E943371E0E0E0933008E0E5DB
:103F580020C0E0913008E03021F0E0932F08E2E53E
:103F680018C0E0E0E0932F08E0934F0CE091C40BF9
:103F7800E03031F0E091C40BE150EA930E94FD1962
:103F8800A091330CA17039F0E091C40BE0932F0895
:103F9800E4E4E0934F0CA0912F081A1721F4A091A4
:103FA8004F0C0A1711F0689423F809911991089594
:103FB8000E943971EBE0EC93EC81D8011696EC93F2
:103FC800EB81D8011796EC93D8011896E0E0F0E061
:103FD800ED93FC93D80112960E944671D80114966D
:103FE8000E9446710E944B71F2C00E943971ECE048
:103FF800EC930E944B7121C21A9318E0113108F515
:10400800E0911408F0911508A981BA81EA27FB27E5
:10401800BF010E945771E623F723309781F00E9471
:104028005771A981BA81EA23FB23309731F01A939B
:10403800E0E0EA931A93BCDF02C01A93D6DF1F5F51
:10404800DDCFFAC1A0911A0CA93030F0E091570CDD
:10405800A091560CEA1709F414C0E091570CE0300F
:1040680021F4E3E6EA93C1DF08C0E0911A0CEA9371
:10407800E0E0EA93E3E6EA939BDFE091570CE093F4
:10408800560C0895A0919A0BECE1EA230895A091AB
:104098009A0BA07411F0E2E00895A0919A0BA07811
:1040A80009F0E2C10DC0A091890BAF3F09F4DCC152
:1040B800E9DFE43009F4D8C1E5DFE03109F4D4C11F
:1040C800E1E008950895A881AF3F11F4E0E06EC1E2
:1040D800D9DFE43011F4E1E069C1E0E067C1A8810B
:1040E800A23019F4CFDFE83011F0E1E05FC1E0E081
:1040F8005DC1E881A3E2EA9FF001ED55F94FE08147
:10410800E13010F0E43108F002C0E1E04FC1E0E036
:104118004DC1A881A13118F0E881E051E883E88118
:104128000E9462710E946C71A091D00BA13018F0AE
:10413800A881A43009F006C0E6E9F0E00E94D37B2C
:104148000E946C7133C1A881A13010F0A63008F02C
:1041580006C0E8810E947771E15CF94F26C1E0E072
:1041680025C1A881A13010F0A63008F006C0E8816A
:104178000E947771EC5BF94F18C1E0E017C10E940B
:10418800A87DEC81EA93EDDFEF731E2F1030E1F08C
:10419800EC81EA93E6DFE0743E2FE12FE150A1E0E5
:1041A8000E94CB7AA0912306EA230E2F303011F417
:1041B800003009F002C0E1E008C0303011F00030F2
:1041C80009F402C0E1E001C0E0E00E94AF7D25965D
:1041D80008950E94A67D00E00530A0F50A930E948C
:1041E8003F1A0E947C71A7E10A9FF001EE5CF94F2B
:1041F8000E94A670E4E1F0E00E945870E0912F0C54
:10420800DA015096EC93A0912E0CEFE3EA23AE2F3F
:10421800E091310CE295E07FEE0FEE0FEA0FDA0144
:104228005596EC93E0912F0CE1503E2F3F3F41F023
:10423800E091300C0E943B70DA015196ED93FC93AB
:104248000F5FCACF10E01336C0F51A930E94A81961
:104258001A9339DFE13079F5E0919D0BEA9373DF2A
:10426800E1500E2F0F3F39F10E947C71E12FDA01E6
:104278001396EC93E0919D0BDA011496EC93E09180
:10428800A30BF091A40BDA011696ED93FC930E9410
:104298003470A4E6B0E080E090E00E94257BDF0166
:1042A800CB01E091A30BF091A40B0E94A86EDA0158
:1042B8001A96ED93FC931F5FC6CF0E94AD7D26969C
:1042C8000895A0911908A23031F0A83021F0A73044
:1042D80011F0A53009F40AC00E945170EFEFF0E028
:1042E8000E94587076DFE0E0E093A20608951A93E2
:1042F800E981E058E98310E01530C0F4A3E21A9F81
:10430800F001EB55F94FE081AE2FE981EA1749F446
:10431800F001EC55F94FE081AE2FE0912F08EA1734
:1043280009F002C0E12F03C01F5FE6CFEFEF18814D
:10433800229608950E94A87DED81EA93D8DF1E2F6A
:104348001F3FC1F00E9483719F01D9011296EC9121
:10435800EF77EC93EC81D9010E948971EF5EFC4FF5
:10436800BF01E081EF77DB010E948971E15FFC4FBB
:10437800A1E0A083E12F0E94AF7DE4C40E94366EC5
:10438800ED55F94FE081E03061F4E091490CEF5FC1
:10439800E093490C0E94366EED55F94FA091490CF7
:1043A800A0830E94366EED55F94FE081219608955D
:1043B8001A931FEFE091D40BF091D50BA981BA8124
:1043C800AE17BF073CF0E091D60BF091D70BEA1778
:1043D800FB070CF412C00E9490710E94E9181E2F6E
:1043E800103031F01F3F21F0E0912F08E11729F438
:1043F800E1E0E093570CE0E01FC0E0E0E093570CE9
:104408001AC01A930E949071D3DF1E2F103099F0B2
:104418001F3F39F4E0EAF8E1FA93EA93EB81FC8173
:1044280006C0E0EBF8E1FA93EA930E949571FA93DB
:10443800EA930E944012E12F188123960895E09193
:104448006505E03009F00895E0912C06E03009F0A8
:1044580008950AC0E0916605E03009F00895E091FA
:104468002D06E03009F00895E0E008950E94A87D47
:10447800E0912606F0912706AC81BD81EA27FB274B
:104488009F0110E0153090F4F901E17049F0A7E1BF
:104498001A9FF001EF5CF94FDF01EC91EF5FEC93AD
:1044A800D9010E9498719F011F5FECCFEC81FD81BB
:1044B800E0932606F09327060E94AF7D43C4289711
:1044C8000E94A67D3091260610E01530B8F5A7E1C8
:1044D8001A9FF001EB5BF94F0081E12FA1E00E94E8
:1044E800CB7A2E2FE22FE32391F0003810F0003C16
:1044F80008F001C00F5F003C31F4E22FA0912306C1
:10450800EA2BE0932306003808F400E80FC00034D3
:1045180008F40F5F003439F4EFEFE227A091230687
:10452800EA23E0932306003808F000E0A7E11A9F89
:10453800F001EB5BF94F00831F5FC7CFE0E0E0932A
:104548002C06E0E0F0E0E0931608F0931708E091FD
:10455800570CE03021F0E0911A0CEA93DADDE09193
:104568001D08EF5FE0931D08E091E30BA0911D0883
:10457800EA1751F4E091E30BF0E0A0E0B1E00E940B
:10458800E77BEA1BE0931D08A0911908A13019F0F8
:10459800A93009F096C0A091620BB091630BE4E1D9
:1045A800F0E00E947D7B309719F4E1E0E0931F086A
:1045B80046DFE03019F04EDFE07809F462C04ADFE8
:1045C800EF775E2F5A930E94A8190E94876DED55C8
:1045D800F94F5081503011F40C94452364DDE130DB
:1045E80031F4E0911A08EA937ADDE03009F449C021
:1045F8000E949D710E941D70EC91EC71EC3021F4C9
:10460800E0911D08E07851F40E94A271EC91EA93C0
:1046180080DD0E94A771EC91EA937BDD0E94A27174
:10462800AC91A63070F5A6E0B7E00E94876D0E94B5
:10463800396E0E94D66E0E94A271EC91EA9383DDD6
:104648001E2F1130F0F00E94AC710E94AF71CF01A3
:104658000E94AC710E94396E6D917C91E12F0E948D
:104668007771EF5CF94F0E94B471E60FF71FDC0118
:10467800ED93FC93E12F0E947771EF5CF94FA0E076
:10468800A08310E01530E8F40E94B77113965C918E
:104698005F3FA9F05A9372DE5E2F0E94C1710E949B
:1046A800AC710E94AF71BF010E94AC710E94396E5B
:1046B8000E94C771AE81BF811296E0E0EC931F5F44
:1046C800E1CFA0911908A23039F0A83029F0A5301F
:1046D80019F0A73009F0E6C1E0E0E093200800E017
:1046E800053010F00C945625A3E20A9FF001ED5511
:1046F800F94FEA87FB87AA85BB85AC91A03019F0F2
:10470800A281A07809F0CCC1E0912008EF5FE09386
:104718002008AA85BB8513960E94C47B309771F048
:10472800AA85BB8513960E94D4710E94DA7129F478
:10473800AA85BB8513960E944671B2C180DEE0301F
:1047480021F00E94DA7109F4ABC120E030E0333087
:1047580010F00C9403250E94E271DF010E94166D8F
:104768000E940D6EE887F987A181A27021F4A481C7
:10477800B581109709F40CC1E885F985A181A47069
:1047880011F40C942724A181A87021F40E943C34D0
:10479800E03009F457C00E94E871EBE0EC93A8857B
:1047A800B9850E94F571A885B9851396EC91AC85F9
:1047B800BD851796EC93EC85FD8538960F01E88545
:1047C800F985A181E1E0EA230E94FC71ED93FC9355
:1047D800A885B98514960E94C47BAC85BD851296C0
:1047E800ED93FC930E94FF71AC85BD851496ED9303
:1047F800FC93A02FEAE0EA9FF001E30FEF5F0E942D
:104808000572E885F985A085B185E2E0F0E00E94AF
:10481800207BA885B9851896ED93FC930E94FF71BB
:10482800309739F4A885B9851896E8EEF3E0ED934A
:10483800FC93E885F985A181E8E0EA2BA885B9858C
:104848001196EC936CC0E885F985A181A17031F4CB
:10485800A885B98514960E94D47141C00E940E7231
:1048680072DCE1501E2F0E94B7711296EC91E03075
:10487800F1F4AE81BF8153960E94D66EEE81FF811E
:10488800A189B289109751F003881488AE81BF813D
:1048980051960E94C47BE015F1050CF007C00E94F8
:1048A800137211F00E9418720E9420720EC0E885DF
:1048B800F98534960E9428720E94FC710E94E1706A
:1048C8000E94307253960E944671E885F985A58149
:1048D800AA232AF4A885B98514960E944671A8854A
:1048E800B985EC91EC71EC3021F4E0911D08E07889
:1048F800B1F4E885F985A481B5815E971CF4A1819E
:10490800A07209F404C0E885F985A28106C00E9456
:104918000E72FFDBE885F985A381AA93FADB0E9472
:10492800FF71309781F0A885B98518960E94D471D7
:104938000E94FF71309739F40E94137211F00E949F
:1049480018720E9420720E940E7219DCE03001F188
:104958000E94137259F00E941872AA85BB85EC91C7
:10496800E150ADE0EA9FF0010E948F6DAA85BB85FA
:104978001296EC91E058AA85BB851296EC93E3E079
:10498800E09324060E940E72ECDBEF73E093250699
:10499800A885B98514960E94C47B309771F52F5F5E
:1049A800323058F5A885B98516960E94C47B309791
:1049B80099F0E885F985A681B781E4E6F0E00E94E0
:1049C800207BAA85BB851396ED93FC93A885B985B2
:1049D80016960E94467111C00E94E271DF01E32F12
:1049E800EF5FF0E00E940D6EE887F987A181EDEF97
:1049F800EA23A885B9851196EC933F5FA8CE2330AA
:104A080011F00C9454250E94137211F00E94187230
:104A18000E943C34E03069F00E94E871E8E0EC93D1
:104A2800AA85BB850E94F571AA85BB85EC910E9479
:104A38000572AA85BB85E0E0EC93EA85FB85A58134
:104A4800ECE1EA23E83061F50E944B6EAE2FEA856F
:104A5800FB85E38DEA1741F4EA85FB85E48DE15097
:104A6800EA930E94A9181CC00E943C34E030C1F0AF
:104A78000E94E871E3E0EC93AC85BD85EFEFEC9321
:104A88001896EA85FB85E38D0E943772AC85BD8553
:104A98001296EA85FB85E48D0E9437720E943B726C
:104AA8000F5F1ECE0E94417249F4A0911908A230EE
:104AB80021F0A83011F0A53009F401C050C010E071
:104AC800153010F00C94B3250E94B77113965C91C1
:104AD8005F3F11F40C94B1250E94C171AE81BF8172
:104AE800BD010E94C771EE81FF8138960E9428722D
:104AF8000E9447720E9430720E94C47BDF010E94AC
:104B08009C7DB4F4EE81FF81A681B7810E949C7DD3
:104B18007CF4AE81BF810D901C90AE81BF8116964A
:104B28000E94C47BD001AE1BBF0B0E949C7D0CF081
:104B380014C0AE81BF81BD010D901C90EE81FF8134
:104B4800A681B781F001EA1BFB0BDB01ED93FC9317
:104B58005A93E5E0EA930E9462431F5FB1CFE09168
:104B68001C08E03041F4E0911608F0911708E09332
:104B78001408F09315080E94AD7D2E9608950E94A2
:104B8800A87DA091C10BE091C20BE150EA9FF00112
:104B9800EF5F1E2F2FE330E000911E08A091180C44
:104BA800A13080F0E091180CE150A0911E08AE17DA
:104BB80028F0E091180CE1503E2F04C0E091180C49
:104BC800E2502E2FEC81E03049F1EF3F51F4A091F3
:104BD8001E08A11BA31720F0E0911E08E11B0E2F51
:104BE8001DC0EE3F59F4E12FA0911E08AE0FA21789
:104BF80020F4A0911E08EA0F0E2F10C0EC3F49F4D4
:104C0800A091180CA13020F0E091180CE1500E2F63
:104C180005C0AC81A1501A9FF0010E2FE0911E082B
:104C2800E01751F00A930E94A819A0918A0BAD329F
:104C380009F4032F00931E080E943747A091190812
:104C4800A83019F40E945A1002C00E94D50F0E9481
:104C5800AF7D259608950E94A67D14DAE03111F4FF
:104C68000C94A32620E030E040E050E010E0133040
:104C780060F50E944B720E94396E0E94C47B309787
:104C880011F10E944E720E9462712E2B3F2B0E94DE
:104C98004E72EA9374DAE03029F0E3E0E0932406F8
:104CA800E0E04EC00E9455720E9462712E2B3F2B8D
:104CB8000E945572EA9363DAE03029F0E3E0E0936A
:104CC8002406E0E03DC01F5FD2CF00E0053068F564
:104CD800A3E20A9FF001ED55F94FE081E03019F1A8
:104CE80010E0133000F50E94E271DF010E94957117
:104CF8000E945C72AE0FBF1F1296EC910E94627107
:104D08004E2B5F2B0E94E271DF010E9495710E9479
:104D18005C72AE0FBF1F1396EC910E9462714E2B0E
:104D28005F2B1F5FDECF0F5FD1CFF901E423F5239F
:104D3800309729F0E1E0E0932406E0E001C0E1E0EB
:104D48000E94AD7D269608951A93E0914D0CE030AF
:104D580011F40C94EF26E091E40BE13059F4A091A2
:104D68004D0CA13311F4EFE001C0E0E0EA930E949A
:104D7800D25E31C0E23059F4A0914D0CA13311F448
:104D8800E6E001C0E5E1EA930E94D25E24C0E33088
:104D9800B1F410E0173040F40E949571E05CF64FD2
:104DA8000E9463721F5FF6CFA0914D0CA13311F4DE
:104DB800E1E301C0E0E3EA930E94D25E0CC00E94E6
:104DC8006772E9E4EA930E943A63E0914D0C0E940D
:104DD8006E720E94737284C422970E94A67D30E08E
:104DE800A0911908A23029F0A83019F0A53009F0CF
:104DF80013C1A985A33610F00C940F28E0912F0851
:104E0800E03009F409C1E9850E942170E03129F4F4
:104E1800E1E3E0934D0CE1E0FFC045D9E03009F44F
:104E2800FBC010E0153058F40E948371E081AE2F6A
:104E3800E885EA1711F4E0E0EFC01F5FF3CF0BDF5E
:104E4800E03011F40C940F2810E00E948371EE8377
:104E5800FF83AE81BF81EC91E03011F00C940828FB
:104E680013960E94467100E0033010F00C94D82786
:104E7800A3E21A9FF001E855F94FDF010E94FE6C8A
:104E88000E940D6EAF01DA0116960E9446710E94CB
:104E98007872DA011296EC930E947F72DA01139607
:104EA800EC93A0919A0BEEEFEA23DA01EC930E94BF
:104EB8008672DA011196EC93E5D8E43139F0FA01FB
:104EC800A181E2E0EA2BDA011196EC930A9307D963
:104ED800E03011F40C94BA27FA01A281AA9333D9CD
:104EE800E1502E2F2F3F81F0A7E12A9FF001EF5CC0
:104EF800F94FA0E0A083A7E12A9FF001EE5BF94FEC
:104F0800A0E0B0E0A083B1830E948E720E94396E47
:104F18000E94C47BDA011496ED93FC93013040F0B3
:104F28000E948E720E94396E0E94C47B309709F0ED
:104F38000EC0AE81BF811596E02F0E94D46F0E94EB
:104F48005C72AE0FBF1F1196EC91E062EC93AE81DC
:104F5800BF815A96EC91E062EC93023030F40E94E3
:104F68009172DA0116960E94377204C0DA0114961B
:104F78000E94467187D8EC3019F4E0E0E0931D08F0
:104F88000E9498720E943B70DA011896ED93FC9388
:104F9800FA01A281A63030F0A181E4E0EA2BDA011F
:104FA8001196EC930F5F60CFA0911908A23011F011
:104FB800A53019F4A885AF3F08F007C0E0912F0885
:104FC800EA93EA85EA930E94EB1AE885AE81BF81ED
:104FD800EC93E0912F08AE81BF811196EC93E9859F
:104FE800AE81BF811296EC93A885A43130F4E88590
:104FF800E1500E949F72A1E0A083AE81BF81169606
:10500800EC91ED7FEC9331E01F5F303011F41530F7
:1050180008F001C01ACFE32F0E94AD7D2A960895AB
:105028001A930A93A0911908A23011F0A53049F4F7
:10503800EA810E949F72A0E0A083EA81EA930E941D
:10504800F16EA0911908A830F1F4EA810E949F72CC
:10505800A0E0A083EA81EA93E1E0EA930E949947FD
:10506800E091E20BE03069F4EA810E94A572E081E8
:10507800EF771E2FABE01A9FF001EA51FA4FA0E03C
:10508800A083689420F8198108812396089564976D
:105098000E94326DA23039F4E0912F08EA93EB8D2B
:1050A800EA930E94EB1AA0911908A83011F00C9409
:1050B800C1280FEF20E0253050F4A7E12A9FF00126
:1050C800EE5CF94FE081AE2FEA8DEA1709F402C0D1
:1050D8002F5FF1CFA7E12A9FF001E15DF94FAF0102
:1050E800DA0115960C910F3F11F40C94C1280E9417
:1050F800AB7210810E941A710E949C7DECF4ABE2A5
:10510800BCE00E94D4710E94B1720E94F170A08329
:10511800B1831A930E945B1FABE00A9FF001E25231
:10512800FA4F30810A93FE0137960E94B7723A937C
:10513800FE0137960E94BB720E94C172F1F40E9470
:10514800AB72AFEFA083DA011396EFEFEC93DA01BD
:105158001596EC930E94B1720E94C772E0E0F0E0ED
:105168000E94FF70E0E0E093280C1A930E945B1FF6
:105178000A930E94BC11689420F80E94AD7D6B963A
:1051880008951A9310E01031B0F4A7E11A9FF001C6
:10519800EC5BF94FE081EF73AE2FE981EA1729F450
:1051A8001A930E94C320E03009F403C0E1E018819B
:1051B800E0C01F5FE8CFE0E01881DBC01A93E09100
:1051C800500CF091510CFA93EA93E4EFF1E00E944D
:1051D8000E71F9F00E94CC7210E01530D0F4A09155
:1051E800540CAF5FE5E00E947A7BE093540CEF5FCC
:1051F800EA93C7DFE03059F0E3E0E0932406E0915A
:10520800540CF0E0EF5FFF4EE093250669C21F5F84
:10521800E4CF66C21A93E0912306E0934C0CE8E7CA
:10522800F0E0FA93EA93ECEDF0E0FA93EA930E9447
:10523800684710E01530D8F4E12FEF5FEA93A1DF5B
:10524800E03099F00E947B6CE12FEA5FF0E00E9469
:10525800476EEDEBF8E10E94E56DA6EEBBE00E941B
:1052680095710E940D6E0E94156E1F5FE3CF38C2C4
:10527800A5DFE0912406E13029F4E5ECF8E10E948D
:10528800D3723CC0E23029F4E2EDF8E10E94D37217
:1052980035C0E33051F4EDEBF8E1FA93EA93E0918D
:1052A8002506F0E0E050F04F29C0E43019F4EAEDAB
:1052B800F8E11FC0E53031F4E0912506EA930E9439
:1052C800231220C0E63019F4E2EEF8E112C0E7300C
:1052D80029F4E8EEF8E10E94D37210C0E83029F40E
:1052E800E4EFF8E10E94D37209C0E93059F4E3E031
:1052F800F9E1FA93EA93E0912506F0E0FA93EA934C
:105308000E944012E0E0E09324060895A881B98144
:105318001196E1E0EC930E941E71A881B981129662
:10532800ED93FC930E944B20A881B9811796EC93CA
:105338000E944B6EA881B98118960E943772E0913D
:10534800C605A881B981EC93E091280CA881B981A0
:105358001696EC93E091890BA881B9811A96EC9383
:10536800E091AC0BF091AD0BA881B9811496ED9347
:10537800FC932296089564970E94A87DA091E20B61
:10538800A230E1F4EB8DEA930E94A8190E944B2009
:10539800ABE2BCE00E943772A9E2BCE0EB8D0E9450
:1053A8003772E0912F08E093280C0E9426703097FE
:1053B80021F00E9426700E94097114C0AA8DAF3F87
:1053C80009F4CAC0EA8DEA930E94541FAB8DAF3F1F
:1053D80029F40E941E710E942B70EB8FEB8DEA93CB
:1053E8000E94A8190E944B200E2FA98DAF3F21F0D3
:1053F8000E945720E03009F001C0AEC00E94F17051
:105408000E94FE6CAE17BF071CF025DCE13009F0E6
:10541800A3C0A091D10BA03021F4A091E20BA2303F
:1054280011F50E944B6EE13041F00E943C34E030AF
:1054380021F00E945234E03009F002C00E94D87274
:105448000E944B6EE13021F40E944234E03009F4AE
:1054580009C00E94E472EE55F84FFA93EA9356DFBA
:105468000E94EA7277C0EB8DEA93EA8DEA93B4DC86
:105478001E2F113011F00C94AE2AA091D30BA1303D
:1054880059F4E0912F08EA930E941E71FA93EA9367
:10549800EFEFFFEF0E94F0720E94F1700E94FE6C25
:1054A8000E94E1700E94FF70689420F8A091E20BBE
:1054B800A03019F4A88DAF3F09F437C00E94F472E8
:1054C800EE51FA4F0E94F170A083B183E88D0E94DB
:1054D800EE6D3081E88DEA93FE0135960E94B77231
:1054E800E88D0E94EE6DE081EA93FE0135960E94F8
:1054F800BB720E944620E03131F00E94F472EA51FA
:10550800FA4FA1E005C00E94F472EA51FA4FA2E0F6
:10551800A0830E94F472EC51FA4FFF93EF930E941C
:10552800C568AF91BF91ED93FC930E94C17219F4C5
:10553800E0E0E093280CEA8DEA930E945B1FE0917B
:105548002F08EA930E9426700E94F972FA93EA9350
:105558000E94491DE1E001C0E0E00E94AF7D6C9629
:10556800089579DBE13041F40E943C34E03021F0C9
:105578000E945234E03009F007C00E9426700E9451
:1055880009710E94D87226C32EC30E94A87D0E946A
:10559800FC721F3F11F40C94202BE0914D0CE0306D
:1055A80011F00C941F2B1A930E94A819E5E0E093C0
:1055B800240610932506A0911908A23031F40E9400
:1055C80005730E940522E03009F010C0A0914E0C2E
:1055D800A13331F4E0912F08EA931A930E94EB1A51
:1055E800E1E3E0934D0C0E94AF7DE2C2A09119085F
:1055F800A830A1F40E9426700E9409730E2F0A9306
:105608000E94B2343E2F1A930A93EFEFEA933A932B
:10561800B2DEE03019F00E94AF7DCAC2A09119082D
:10562800A53031F49EDFE03019F00E94AF7DC0C292
:10563800E0E3E0934D0C06C0E0E3E0934D0CE4E0BA
:10564800E09324060E94AF7DB3C2E09140090E9416
:105658000D7308951A93E6E0EA930E94D25E0E94C1
:105668006772A0914009A83539F4EFE0F9E10E948A
:105678001973E0E00E947372A0914009A33509F5FF
:1056880010E0A0911908A83021F0A23011F0A5303F
:1056980009F411E3E3E5EA930E943A631A930E943E
:1056A8003A63E0E8EA930E943A63E0E8EA930E94EA
:1056B8003A63E0E80E946E72E0934D0CE0E00E94CD
:1056C8007372A0914009A93459F40E941D73E093A4
:1056D80025060E942773EC91E0934E0C56DF34DBCD
:1056E800199108950E94A87DA0913F09A53411F051
:1056F8000C94BD2B0E942C73E2E3F0E0E093470C7E
:10570800F093480CA0914009A73741F4E4E4F9E08C
:105718000E9433730E9438730E940D73A091400950
:10572800A03310F0AA3308F023C020912708309145
:105738002808E0E4F9E00E943373E2E0EA930E946B
:10574800C8620E2F0E943873E09325060E943873B2
:105758000E943C730E94FC720A931A930E94EB1AEF
:105768002093270830932808E2E5EA930E94D25E46
:105778001CC0E091450CF091460CFA93EA93E09135
:10578800470CF091480C0E940E7179F0E0E0E0932C
:105798003A09E5E4EA930E94D25E0E942C73E8EC91
:1057A800F0E0E093470CF093480C0E94AF7D00C2F4
:1057B8000E9441730E9447730E947B6C0E947B6C1D
:1057C8000E941047A0911B08A23021F4E7E1F9E1FB
:1057D8000E94E56DA0911B08A13021F4EEE1F9E1EA
:1057E8000E94E56DE0911B08E03021F4E5E2F9E163
:1057F8000E94E56D0E9451730E94BC6C0E94104784
:105808000E9454730E945973FA93EA93E0915F05DA
:10581800F09160050E945F730895E1E003C0E0E045
:1058280001C0E2E0E0931B08C3DF08950E94462010
:10583800EC3109F0D8C1E091990BE33631F4A0912D
:105848001908A23009F4EBDF17C0E23631F4A09151
:105858001908A23009F4E5DF0FC0A091C505A230F0
:1058680011F0A63021F4E091990BEA9388D9A09120
:10587800C505A43009F4D1DFADC10E941B6E0E949A
:105888007B6C0E941F6E0E947B6C0E947B6C0E9446
:105898001047E8E6F5E00E94E56DE0911A080E94DD
:1058A8006373E6E7F5E00E94E56DE2E0E0930E043D
:1058B80008950E945170E3EEF0E00E945870E8816C
:1058C800E03009F406C0A0911A08AF5FE3E00E9437
:1058D8007A7BE0931A08E1E0E093490C0E94ED20FE
:1058E80072C20E94A87D10E0133610F00C94C22CEE
:1058F8000E949571ED55F94F30813F3FE9F11A93B8
:105908000E94A81900E00E9467730E94396E0E94E5
:10591800C47B3B9794F00E946A730F010E946773DF
:105928000E94396E0E9470730E9476730E941D70E7
:10593800EC91EE7FD001EC9301E00E947B730E9412
:10594800396E0E94C47B759794F00E946A730F01A8
:105958000E947B730E94396E0E9470730E94767356
:105968000E941D70EC91E160D001EC9301E00130E0
:1059780019F41A930E94C8191F5FB6CF0E94AF7D11
:1059880017C11A930A9323FE03C00E947E7344D75B
:105998000E947243E030C1F1E0E00E948573103844
:1059A80020F5113219F40E947E7336D71D3439F46C
:1059B8000E948C730E946964E3E0E09318081B322C
:1059C80071F40E949173EAE2EA93E0E3F9E1FA9351
:1059D800EA93E0911A08E05DEA930E9469641F3235
:1059E80019F4E1E0EA93CBD848DF103868F00E9458
:1059F80097731A930E94C22119DFE03011F4103214
:105A080008F002C0E0EFF6E20E942E220E2F0038C6
:105A1800C8F10F770336A8F5E0911F08E03031F0A0
:105A28000A930E949112E0E0E0931F08E091550C60
:105A3800E01739F10A930E94A8190E94A271AC914B
:105A4800A83028F40E94A771AC91A830A8F0E02FE4
:105A5800EF5FE093A2060A930E94C2210E94A271FE
:105A6800EC91EA930E94A771EC91EA93E091A20667
:105A7800EA930E94DC1F03C0E0E0E093A2060093D3
:105A8800550C0EC0A091550CAF3F51F0E091A20605
:105A9800E03019F0EA930E94F91FEFEFE093550CFC
:105AA800099119910895A881A03310F0AA3308F03C
:105AB8001DC00E949B730E94A073AAE0B0E00E94E0
:105AC800207BDF01E8810E94A573EA0FFB1FE093AA
:105AD8002508F0932608E2E0E0930E040E94517333
:105AE8000E94BC6C0E941F6E0E945473A881A3344C
:105AF80051F40E9447730E9451730E94BC6C0E942B
:105B08001F6E0E9454735FC11A930A93A0E023FC8E
:105B1800A1E0A03019F0AA81A03009F016C0E894DD
:105B280023F8E7E0E09318080E945746A09131084F
:105B3800A03019F40E94A87309F407C0E7E0EA93BB
:105B48000E94AD7369D6E89424F824FE24C00E940C
:105B5800B073EAE5F0E00E94B77319F0AA81A130AA
:105B6800C9F486D6E030B1F00E94BD730FEF1FEF85
:105B78000E9405730E94DC21E03021F4009127087F
:105B880010912808EB81EA93E0912F08EA931A9381
:105B98000A9342D60BC00E94B073ECE2F1E00E9477
:105BA800B77321F40E94C473E09330081981088107
:105BB80024960895E091C70BF091C80B0E94C87312
:105BC80011F4E2E00895E091C50BF091C60B0E9434
:105BD800C87311F4E1E00895E091CB0BF091CC0B80
:105BE8000E94C87311F4E0E00895EFEF0895A091C2
:105BF8001908A23021F40E9437470E94D50FA091BE
:105C08001908A83009F467D6A0911908A53009F435
:105C180049D1D9C0E2E0EA930E946641E2E0E0930C
:105C28000E04E881EA933FDFA881AF3721F4E091C1
:105C38002B06E37009F403C0E2E0E0931808A8819A
:105C4800A13239F0A33421F40E949B73109709F014
:105C580004C0A0911908A23009F011C0A0911B0836
:105C6800A33009F4DEDDA0911B08A23019F4E1E0AD
:105C7800EA93BDDFE0911B08E03009F4D0DDA8818C
:105C8800AD3311F00C94A32E0E945746E0911B08E7
:105C9800E030B1F4E0912508F0912608FA93EA93F0
:105CA8000E940522E03051F4E0912508F091260881
:105CB8000E943C73E0E0EA939ADF01C0B0DD3FC088
:105CC800E13079F477DFEF3F41F0E3E00E94CC73F5
:105CD8000E948C730E94D27303C0E1E0EA9387DFCD
:105CE8002EC0E230F1F40E949B73A336E0E0BE07B9
:105CF800B4F4E0912508EA930E94D973E2E0E093B6
:105D08000E040E947B6C0E947B6C0E9410470E94CC
:105D1800D86D0E942411E3E0E0931B0801C081DDE7
:105D28000EC0E33061F4E0912508EA930E94A819B7
:105D3800E0912508EA93EEEFEA934ED872DDA88148
:105D4800AD3409F46ADDA881A43521F4A0911908BD
:105D5800A23009F001C063DDA881AB3221F4EEEF77
:105D6800EA930E94C325A881AD3221F4EFEFEA93AC
:105D78000E94C325A881A73421F4E1E0EA930E9498
:105D8800C325A881AB3421F4ECEFEA930E94C32524
:105D98001AC00E9465210E943747E0E0E0931B0883
:105DA800A881A13039F40E94A87321F0A091CA0BF0
:105DB800A03009F402C033DD06C00E94D50F0E944E
:105DC80005730E94DC21219608951A930A930E9474
:105DD800DD730E9426200E947243E03091F10E94F8
:105DE800E67378F10E94977321DDE03051F50E9447
:105DF800EE730E949E21EF3F09F00BC50E940573C8
:105E08000E940522E03021F40E945720E13009F079
:105E180018C00E944620E83119F40E94F37309F073
:105E280001C0F7C40E94EE730E94F0260E2F0130C5
:105E380021F4A091990BA03009F403C01A930E9491
:105E48002312A0912E06AF3F61F110912E06EFEFBD
:105E5800E0932E061A930E94A8190E9405730E94C7
:105E68000522E03021F40E945720E13009F019C0E2
:105E78000E944620E83119F40E94F37309F001C02A
:105E8800C8C41A93EEEFEA930E94F0260E2F013051
:105E980021F4A091990BA03009F403C01A930E9431
:105EA8002312B7C40E9465210E94ED20E89421F8CE
:105EB800E0E0E0931E080E94FA730E9437470E94B0
:105EC8007B6C0E947B6C0E941047E09132060E9416
:105ED8005C6EE09133060E945C6E0E947B6C0E94AF
:105EE800E06D0E941047E0913F060E945C6EE091D1
:105EF8003906F0913A060E94326E08950E94A87DF4
:105F08000E94DD730E947243E03049F00E94E673FC
:105F180030F00E9497738ADCE03009F422DBE091CC
:105F2800520CF091530C0E94F56E11F40C94FC2F56
:105F38000E94FA730E947B6C0E94D36D0E941F6EB0
:105F4800E0913706F09138060E94326EE0913B06E8
:105F5800F0913C060E94326E00E0053010F00C947F
:105F6800FC2FA7E10A9FF001E15DF94F9F01F901BC
:105F7800A381AF3FD9F1D9011A960E943E6E7F9353
:105F88006F93FF93EF930E940174AF91BF918F912C
:105F98009F910E94E27A0E94257BDF01CB010E943B
:105FA8000674D9011C96ED93FC93F90104841584B9
:105FB800D9011E960E94C47BE015F105B9F0F901DC
:105FC80004841584A685B785F001EA1BFB0BE093D2
:105FD800AC0BF093AD0BC5DAE13041F4D9011C9656
:105FE8000E94C47BD9011E96ED93FC930F5FB5CF39
:105FF8000E94AF7D2FC40E94A87D0E94DD730E947D
:1060080026200E947243E03011F40C9495300E94CF
:1060180075430E2F0A93FEDD003820F0A091C605C7
:10602800A03808F429C00F770A930E940D740E94C3
:1060380009731E2FA091E20BA03011F41F3F09F441
:1060480016C030E0353098F4ABE03A9FF001E452E6
:10605800FA4FE081E11749F43A9FF001E252FA4F12
:10606800E081EF5FE093C605232F3F5FEBCF0A93F4
:106078000E94EE732A9354C0A091E20BA03021F441
:10608800003810F0053808F00AC00F770E94AB728C
:106098001081EFEFEA930E94EE730A936CD9A091F6
:1060A800E20BA03011F0003808F43BC00F770A93D8
:1060B8000E94A819BBDBE030A1F50E9410740E9471
:1060C8009E21EF3F19F00E94AF7DC4C30E94572064
:1060D800E13039F50E944B20E03049F40E941074F9
:1060E8000E94F026E03011F00E9415741AC00E9438
:1060F8004620E83141F40E94F37321F00E941074A5
:106108000E94F0260EC0A0911E08E02F0E94B26DDA
:10611800AE0FBF1F1C910A930E94EE73EFEFEA9334
:106128002AD9A0912E06AF3FF9F000912E06EFEF85
:10613800E0932E060A930E940D740E9409731E2F85
:106148000A931A93EEEFEA93EFEFEA9314D91F3FFD
:1061580041F4A0919D0BA03021F4A091A00BA03098
:1061680009F002C00E94157420FE0AC0E89420F8C5
:10617800E091E20BE03019F404D455D501C0B4D550
:1061880030E0353080F5ABE03A9FF001DF01EA51AD
:10619800FA4FE081E03049F0AC51BA4F0E941B74CD
:1061A800E8EEF3E00E940E7199F4ABE03A9FF0013B
:1061B800EA51FA4FE081E23051F43A9FF001EC5194
:1061C800FA4FDF010E94C47B0E94F56E09F409C0F2
:1061D800ABE03A9FF001EA51FA4FA0E0A08368943F
:1061E80020F83F5FCECF0E94AF7D34C30E94326D4E
:1061F800A33011F40C94B832E0913A08ED3411F060
:106208000C94DC31E0913B08EA3511F00C949131A3
:1062180024FC83C0E0913C08E0532E2FE0913D0818
:10622800E0533E2FEEE3F8E00E9433730E94277399
:10623800AC91AB3429F40E9420740E9456620E2F50
:106248000E942773AC91A43529F40E9420740E94FF
:106258005662AF01E091CD0BE31731F5E0E0E09332
:106268004B0C0E94BD734093270850932808A091B7
:1062780030080A1759F0E7E0E0931808009330084F
:1062880020934A0CE0E0E0932F080DC0A0914A0C3F
:106298002A1721F0A0912E08A03009F004C02093FD
:1062A800180820934A0C35C0A0913008A03049F452
:1062B800A091CE0B0E94166DE255FF4FE491EA23A0
:1062C80009F40CC0E7E0E093180820934A0CE0E0DA
:1062D800E0932F08E0913908E0934B0CE0913908DE
:1062E800A0914B0CEA17A9F440932708509328086B
:1062F800009330080E94BD73A0914A0C2A1721F020
:10630800A0912E08A03009F004C02093180820930B
:106318004A0C273011F40E943371E0913B08E934AC
:1063280039F4E7E00E94CC730E94C473E0932F080D
:10633800E0913B08E23439F4E4E00E94CC730E9417
:10634800C473E0932F08E0913B08E03519F4E1E0CD
:10635800E0931808E0913B08EC3449F4E4E0E0935A
:106368001808E0913C08E053EA930E94E616E09191
:106378003B08E334E9F4A0913C08A13320F0A09154
:106388003C08A93308F014C00E942374E091220845
:10639800EA930E94C61BE0913908EA93ECE3F9E11D
:1063A800FA93EA930E945C700E94D77B0E945C6417
:1063B800E0913A08E03521F4A0911908A13009F0DC
:1063C80003C00E94917359DAE0913A08EF3459F406
:1063D800E0913B08EE3439F4E0913908EA93EFE3B1
:1063E800F9E10E942974E0913A08E33571F5E091EA
:1063F8003B08EF3351F5A0913C08A03360F0A09121
:106408003C08A93340F4A0913D08A03320F0A091A6
:106418003D08AA3308F019C00E942374E0913D0892
:10642800E0531E2F103011F40E944A1BE0913908E6
:10643800EA93E2E4F9E1FA93EA930E948F700E94EA
:1064480072700E94D77B0E945C64E0913A08E33442
:1064580011F00C947D32E0913B08EF3311F00C946D
:106468007D32E0913D08E03319F4EFEFE093230823
:10647800A0913C08A03320F0A0913C08A93308F073
:106488001BC00E942374E0912308EF5FE093230868
:10649800E0912208EA93E0912308EA930E947B1A8C
:1064A800A0911D0CB0911E0C109721F4A091230807
:1064B800A33608F001C0E7CFE0912308EA930E94D1
:1064C800A8190E942F74E5E4F9E10E9419730E944B
:1064D800386F0E9434740E9439740E943D6F0E9484
:1064E800D77B0E9439740E949F6F0E94C8630E94E4
:1064F8002C64E0913A08E434B9F5E0913B08E434BF
:1065080099F514E0E1E0E0933909103538F40E9478
:106518009571E85CF74FE081E03208F41AC00E94F8
:106528009571E85CF74FE081E33259F40E94957168
:10653800E75CF74FE081E053EA930E94D25E1F5F69
:1065480006C00E949571E85CF74F0E9463721F5F56
:10655800DCCFE0913808EA930E941164E8E4F9E19D
:106568000E9419730E942C640E94AD7D269608959E
:106578001A930A930E94417211F40C943833E0E0A4
:10658800E093570CE0911808EF770E2F0093180846
:106598000E9437470E94E06DE4E0F0E0FA93EA9346
:1065A8000E941047013021F0A0911908A13009F08C
:1065B8000BC0EEE7F5E00E94E56D93D9E4EFF1E05A
:1065C8000E94986C0E943747073049F40E94652161
:1065D800E0E0E0931B080E94C4120E940E290430D8
:1065E80031F4EBE4F9E10E94E56D0E948A0E08306F
:1065F80019F40E943F746FD1053019F40E943F745A
:1066080051DC013051F4E89423F8E0E0EA9351D9E1
:106618000093190832D90E94D50F093071F4E0E0CF
:10662800EA9347D9E0E0E0931E08E89423F80E9433
:10663800D50F0E944974E093570C023069F4E0E0EA
:10664800E0931E08E0E0F0E00E943C73E89423F831
:106658000E944974EA939DDB033011F40E941841AB
:10666800009319080E942620A0911908A73011F05C
:106678000C94E633E091500CF091510C0E94F56EA9
:1066880021F0A0911B08A03009F00AC00E94CC722A
:10669800E0914C0CA0912306EA1711F00E940E29F4
:1066A8000E947243E030E9F0E2E00E9485731A9399
:1066B800FAD91D3409F4B1D81D3399F40E9457460C
:1066C80079DAEF3F41F0E3E0E09318080E948C7319
:1066D8000E94D27306C0E7E8E0931808E0E0E09370
:1066E8001B08A0912F08A03031F0E0912F08A0914D
:1066F8002E08EA1709F457C0E0912F08E150EA93F1
:106708000E94FD19A091330CE1E0EA23E13021F465
:10671800E0912B06EF7C09F429C0E0E0E0932E0815
:10672800E0914A0CE03019F0E09318081EC012E01E
:10673800E0912B06EC7009F018E0E091C40BA091F1
:106748002F08EA1781F0E0912B06E07439F011E088
:10675800EAE2EA93E0E5F9E10E942974E0912B0668
:10676800E07809F019E0109318081DC00E94374717
:106778000E94C4120E94E06DE4E0F0E0FA93EA930C
:106788000E941047EBE4EA930E94AE46E0912F087E
:10679800EA930E94ED41E3E5F9E10E94E56DE0919D
:1067A8002F08E0932E08A0912F08A03021F4A09183
:1067B8002E08A03009F406C0E0E0E0932E08E7E8D0
:1067C800E0931808A0911908A33011F40E94153F0E
:1067D800A0911908A13009F4D4D8A0911908A230C1
:1067E80009F4F3DAA0911908A83009F404DCA0919F
:1067F8001908A53009F482DBA0911908A93049F4D9
:10680800E0E0E0932008E0911908EA93E0E0EA93D9
:106818007BD90991199108950E945074E652F84F56
:10682800A6E0A0830E945074E752F84FAB81A08382
:106838000E945074E152F84FAA81A0830E945074BC
:10684800E552F84FA881B981A083B1830E943B72B9
:106858000E947551249608950E945674A881B981A2
:10686800AC91A53020F0A881B981E0E0EC9387C015
:10687800A0911308BB27E091120805C0A091110848
:10688800BB27E0911008F0E031960E94E170359640
:10689800DF01E5E0F0E00E947D7B08951A931091F6
:1068A8001308E0911208E117A1F0ABE01A9FF0017C
:1068B800E652F84FE081E13011F0E23011F4E1E006
:1068C8004BC0EDB7FEB7FA93EA931F93C5DF1F914C
:1068D800E8CFE0E041C01A930E946521ECEDF5E0B5
:1068E8000E94A6700E945E6D0E940F6910E015302C
:1068F80068F40E941471AFEFA083ABE01A9FF00117
:10690800EE51FA4F0E94C7721F5FF1CF10E01530A9
:1069180048F4A7E11A9FF001EC5CF94FAFEFA083B0
:106928001F5FF5CFE0912B06E37019F00E94A87362
:1069380009F402C0689401C0E89421F8EFEFE093ED
:106948002D08E091E20BE03029F41BD06CD1E894DB
:1069580020F802C00E945A10199108951A9310E065
:10696800153058F40E941471E081AE2FE981EA17BE
:1069780011F4E12F03C01F5FF3CFEFEF18812296C8
:10698800089522970E94A67D00E0053058F40E94E1
:106998005C74A0E00E946274E152FA4FA0E0A08308
:1069A8000F5FF3CF00E00530C0F50E94AB72E081C5
:1069B800EF3F89F10E94AB72E0810E942371B9F028
:1069C8000E94B172DF010E94C47B0E94F170EA1735
:1069D800FB0751F00E94B1720E94F170A083B1834D
:1069E8000E946774A1E0A0830E945C7412C0ABE0AF
:1069F8000A9FF001EA51FA4FE081E03061F40E9409
:106A0800AB72AFEFA0830E94B1720E94C7720E945E
:106A18006774A1E0A0830F5FC6CF0E94461F1E2F98
:106A28001F3F11F0E1E001C0E0E0E093570C1F3F89
:106A380011F40C94713550E000E0053048F40E94E0
:106A4800AB72E0811E1711F451E002C00F5FF5CF61
:106A58005030E1F500E00530C8F50E94AB72E081E6
:106A6800EF3F91F50E94AB7210830E94B1720E94B1
:106A7800F170A083B183ABE00A9FF001E052FA4FB6
:106A8800A091280C0E946274EF51FA4FFF93EF9384
:106A98000E941E710E942B70AF91BF91EC930E94CF
:106AA8006774A1E0A0830E945C74A1E00E946274F4
:106AB800EC51FA4FFF93EF930E94C568AF91BF91D5
:106AC800ED93FC9351E002C00F5FC5CF503029F021
:106AD8001A930E944D1F1E2FAACF30E0353010F0B8
:106AE8000C94B735A7E13A9FF001E15DF94FEE83C9
:106AF800FF8350E000E0053048F5503029F5ABE061
:106B08000A9FF001EF51FA4F20812A930E94A81999
:106B18000E945C74E081E13059F42A930E94672056
:106B2800E13031F4A32FAF5FE0919D0BEA1709F034
:106B38000BC0E22FAE81BF811396EC93E02FAE819C
:106B4800BF811596EC9351E00F5FD5CF503049F4D3
:106B5800AE81BF811396EFEFEC93AE81BF8115969E
:106B6800EC933F5FBBCF0E94AD7D289608950E94AD
:106B7800A87DAC81BD81EBE4EC93EC81FD8131967D
:106B8800FA93EA930E946D74E052FA4FE0810E94F2
:106B9800D66C00E00E947674EC91E03011F00F5F43
:106BA800F9CF0E947674E0E2EC930F5F0E947C7448
:106BB8000E948A6D0E946D74EE51FA4FDF010E94A7
:106BC8003E6E0E948174EE81ABE0EA9FF001EF51C6
:106BD800FA4F10811A930E94A81900E00E94767457
:106BE800EC91E03011F00F5FF9CF0E947674E8E77E
:106BF800EC930F5F0E947674E0E2EC930F5F30E055
:106C08003A3060F40E947C74EA0FFB1F0F01AAE877
:106C1800BBE00E9488740F5F3F5FF2CF0E947674DA
:106C2800EC930C94A73864970E94A87D00E010E0CC
:106C3800153040F40E941471E081EF3F09F40F5FB2
:106C48001F5FF6CF053021F0A0912D08A03009F480
:106C580006C0E0E0E0932D08EA930E94711110E06D
:106C6800153088F5ABE01A9FF001E152FA4FE08148
:106C7800E03039F11A9FF001E352FA4FE081E03039
:106C8800B1F01A93FE0135960E94B772ABE01A9FD5
:106C9800F001EF51FA4F30813A930E94A8191A93E4
:106CA800FE013596FA93EA930E94CC110AC01A9312
:106CB8000E94BC11ABE01A9FF001E152FA4FA0E02C
:106CC800A0831F5FCDCF053021F4A0912D08A130FE
:106CD80009F406C0E1E0E0932D08EA930E947111DF
:106CE8000E94AF7D689608950E94A67DA091E20B50
:106CF800A23011F40C94413A30E0343168F40E9427
:106D08008F740E949274DA011296E0E0EC93DA0133
:106D1800EFEFEC933F5FF1CF0E94461F0E2F0F3F1E
:106D280011F0E1E001C0E0E0E093570C0F3FA1F162
:106D38000E941E71FA93EA930E9458191E2F1F3F52
:106D480031F1A0911E08E12FEA1B3E2F3431F8F4EF
:106D58000E948F740E949274FA0132960F01E081AA
:106D6800AE2F0E949874B0E0EA0FFB1FD001EC939D
:106D7800FA01A281A43620F0DA011296E3E6EC9338
:106D8800DA01AC91AF3F19F4E02FDA01EC930A93E2
:106D98000E944D1F0E2FCACF0E94FF1530E03431DC
:106DA80010F00C945D370E948F740E949274FA015F
:106DB800A381AF3F11F40C945B370E949D740E942D
:106DC8002170E83139F40E949D74EA930E949F185B
:106DD800E03009F408C00E949D74EA930E949F184D
:106DE800DA011296EC93A0919A0BA07839F4FA0183
:106DF8000280DA011196EC91E01509F458C0DA0125
:106E080013962C91ADE02A9FF001EF5EFC4F0F0125
:106E1800DA011296EC91D001EC930E949D74EA93EA
:106E28000E947B21EF3F29F0ADE02A9FF0010E94EC
:106E38008F6DDA011296EC91E03089F00E94A2740D
:106E4800DF010E94AD6DEC93ADE02A9FF001E25F97
:106E5800FC4FDF01E091980BEF70EC9313C00E9498
:106E6800AD6DE03021F40E94A274A0E003C00E943E
:106E7800A274A8E0A083ADE02A9FF001E25FFC4F76
:106E8800A7E0A0830E949D74EA930E947B21EF3FB4
:106E980019F0ECE0E0930F04DA011296EC91DA01B4
:106EA8001196EC932A93E1E0EA930E9499473F5F99
:106EB80076CF0C94413AE7E0E09318080E94E11875
:106EC800A8950E940D1DA8950E94621FA895EFEF36
:106ED800E093B20BE093890BE093320CE0932D0C16
:106EE800E0932E060E94A874EC7F29F0A8E0B0E099
:106EF800E0E00E94067C089568970E94A87D0E94A1
:106F08009942E0E6F9E10E94A6700E9419430E94A6
:106F1800C142E0912208E03061F0EBE6F9E10E941D
:106F2800A6700E941943E09122080E94AD740E9445
:106F3800B1740E94C1420E944A1B00E00A30A0F4CA
:106F48000A930E94D7190E94C56FEFE0EA930E9446
:106F5800F342E02FA3EAB6E00E94B5740E94727073
:106F68000E94B9740F5FEACF0E94D342E4E7F9E1C7
:106F7800FA93EA93EFE0EA930E9419430E94056F9F
:106F88000E94B9740E94D5420E94C14210E010319B
:106F980010F00C945E380E944B6EE117E1F5EAE7B9
:106FA800F9E10E94A6700E9419430E94CE6D0E94CA
:106FB800B174E0E0E0931E08A0911E08A33648F5DE
:106FC800E0912208EA93E0911E08EA930E947B1A56
:106FD8000E94386F3097B9F0E0911E08EA930E943A
:106FE800A8190E94386FFA93EA930E94BF740E940E
:106FF80019430E949F6FEAE0EA930E94F3420E94BD
:107008003D6F0E94B974E0911E08EF5FE0931E087F
:10701800D3CF0E94C4740E9495710E94777011F0BA
:107028000C945C38EAE7F9E10E94A6700E941943C3
:107038000E94CE6D0E94B1740E94C874E0E30E9461
:10704800837029F40E9488700E9456629F01022E64
:10705800032A61F10E9420740E947E62E88FF98FF2
:107068006A8F7B8F0E9420740E94D0743A932A936F
:107078000E94BF740E941943FE013496FA93EA9362
:10708800EAE0EA930E94F342E88DF98D6A8D7B8DE0
:107098000E94B9740E94C874E1E30E94837029F4C5
:1070A8000E9488700E9456629F01D1CF0E94C474CA
:1070B8001F5F6DCF0E949A420E94AF7D6C96089523
:1070C8000E94A87DAD81BE812C910E94D4740E943B
:1070D800CE6D0E94FE6C0E94476EECE3EA930E941C
:1070E800AE46EC81EA930E9402472A93ED81EA9327
:1070F8000E94A741EEE3EA930E94AE460E945973AC
:107108000E94F9720E945F730E94D974333409F4A3
:1071180031E2313320F0EC81E05DE31708F407C079
:10712800E32F0E94A573E255FF4FE4912E273D33CC
:1071380011F0313209F401C0CACF3D3319F4AD81E1
:10714800BE812C93E32F0E94AF7D279608950E945D
:10715800A67D20E0AF81B8855C910E94D4740E941E
:10716800CE6D0E94FE6C0E94476EE2E0EA930E9498
:1071780002475A930E94ED410E9459730E94F97286
:107188000E945F730E94D974303310F03A3308F0CC
:107198000EC0203009F450E021E0A52FEAE00E945B
:1071A8007A7BAAE0EA9FF001E30FE0535E2F3B32BF
:1071B80011F4533608F001C05F5F3D3211F45130CD
:1071C80008F401C05150333429F4203009F431E275
:1071D80050E020E03D3319F4EE81E51708F005C0D2
:1071E800AF81B8855C9130E020E03D3311F0313259
:1071F80009F401C0B4CF3D3319F4AF81B8855C936D
:10720800D0C00E94A67D20E0AF81B8854D915C91E9
:107218000E94D4740E94CE6D0E94FE6C0E94476E3C
:10722800AE81A23051F4E6E0EA930E940247FA01E7
:107238000E94E27A0E94436E08C0E5E0EA930E9449
:1072480002475A934A930E94DB410E9459730E9455
:10725800F9720E945F730E94D974303310F03A3388
:1072680008F01EC0203011F440E050E021E0403129
:10727800E7E25E0734F0DA01E0E1F7E20E947D7BA5
:10728800AF01493BEBE05E0724F0DA010E94A073EE
:10729800AF01DA010E94DE740E94E374D097AD0159
:1072A8003B3221F44033E5E75E070CF002C04F5F44
:1072B8005F4F3D3221F40024041605060CF002C08D
:1072C80041505040333431F4203009F431E240E089
:1072D80050E020E03D3311F0313209F401C09ACF7B
:1072E8003D3321F4AF81B8854D935C935AC00E9419
:1072F800A67D0E94D47420E050E04FEF0E94CE6D2E
:107308000E94FE6C0E94E8740E94EB74E885EA9380
:107318000E94DA46E52FE10FF0E00E94F9720E9420
:107328005F730E94D974303310F03A3308F021C0EB
:107338003053431729F04F3F09F05F5F20E005C045
:10734800A22FAF5FEA2FE3702E2FE52FAF81B8850C
:107358000E94F0740F01E32FA6EBB6E00E94B5740B
:10736800AE0FBF1FE22F0E94F074E491D001EC939E
:10737800432F3B3219F4EE815E1708F002C05F5FBD
:107388004FEF3D3211F4513008F402C051504FEF25
:10739800EE815E1720F4313211F03D3309F401C05B
:1073A800ADCFE32F0E94AD7D299608951A930A93D5
:1073B800A0919A0BECEDEA231E2F00E00D3040F46B
:1073C8000E94F4740E94F874E11711F00F5FF6CF71
:1073D8000E94F474EA0FFB1F0E94D37B0E94E56DA4
:1073E800E02F3DC4AAE9BBE00E94366EAE0FBF1F76
:1073F800EC91E17011F4E3E701C0E9E4EA930E943B
:10740800AE46219608950E94A67D0E94D4740E94DB
:10741800CE6D0E94FE6C0E94E874C8DF5E2F0E9449
:1074280059730E94F9720E945F730E94D9743D32A9
:1074380011F0363311F4503009F401C051503B3289
:1074480011F0333311F45C3008F001C05F5FA09194
:107458009A0BE1E0EA232E2FE52FA8EFB1E00E9476
:10746800B5740E94F874E20FE0939A0B3D3311F063
:10747800313209F401C0CBCFE32F0E94AD7D2696AF
:1074880008950E94A87D0E94D4740E94CE6D0E9427
:10749800FE6C0E94E874AAE9BBE0EC810E941D70B2
:1074A800EC91E17019F4E7E8F9E102C0EBE8F9E1E1
:1074B800FA93EA930E94C5460E9459730E94F97292
:1074C8000E945F730E94D974303310F03A3308F089
:1074D8000FC0AAE9BBE00E9441700F01AAE9BBE016
:1074E800EC810E941D70AC91E1E0EA27D001EC9399
:1074F8003D3311F0313209F401C0C7CFE32F0E94A8
:10750800AF7D259608950E94E66CE1E0EA930E941B
:10751800740F0E947B6C0E947B6C0E9410470E9433
:107528009F6FEAE0EA93E3DEE13209F45FC40E9468
:107538007B6C0E947B6C0E941F6EEFE8F9E10E9451
:10754800E56DE5E9FBE00E94A6705BDEE13209F437
:107558004DC40E947B6C0E947B6C0E941F6EE5E903
:10756800F9E10E94E56DE091970BEF5F0E2FEDB703
:10757800FEB7FA93EA930F93EAE0EA93E8DD0F91F6
:10758800E13209F433C400240216030624F4E02F80
:10759800E150E093970B0E947B6C0E947B6C0E94E9
:1075A8001F6EEEE9F9E10E94E56DECEAFBE00E944E
:1075B800FD7409F41BC40E947B6C0E947B6C0E94C2
:1075C8001F6EE4EAF9E10E94E56DEEEAFBE00E9435
:1075D800FD7409F40BC40E947B6C0E947B6C0E94B2
:1075E8001F6EEAEAF9E10E94E56DE9E9FBE0FA932A
:1075F800EA93E3E60E94057509F4F8C30E947B6CE0
:107608000E947B6C0E941F6EE3EBF9E10E94E56D1E
:10761800FADEE13209F4EAC310E0133010F00C94FA
:10762800CC3B0E947B6C0E947B6C0E941F6EE12FFA
:107638000E946373E9EBF9E10E94E56D0E940A7507
:107648000E941047ADE9BBE00E9495710E948A6DC7
:10765800E0E10E94057509F4C9C3E9E0F0E00E9481
:10766800BC6C0E941047A0EABBE00E9495710E9482
:107678008A6DE0E10E94057509F4B8C30E947B6C2D
:107688000E947B6C0E941F6EE12F0E946373E4ECE2
:10769800F9E10E94E56D1A93F4DEE13209F4A6C31C
:1076A8000E940A750E940E7551F40E944B720E9446
:1076B8001875E2E00E941B7509F498C309C00E947E
:1076C8004B720E941875E0E00E941B7509F48EC386
:1076D8000E947B6C0E947B6C0E941F6EE12F0E94AF
:1076E8006373E6ECF9E10E94E56D0E940A750E9459
:1076F8001047A9EABBE0EE27A10FBE1F2C91332744
:10770800EDB7FEB73197FA93EA933F932F93E0E0F2
:10771800EA9377DD2F913F91E13209F467C3A9EA33
:10772800BBE00E949571EA0FFB1F2083123070F5B1
:107738000E947B6C0E947B6C0E941F6EE12F0E944E
:107748006373EDECF9E10E94E56D0E940A750E94F1
:107758001047A0EBBBE0EE27A10FBE1F2C913327EB
:10776800EDB7FEB73197FA93EA933F932F93E0E092
:10777800EA9347DD2F913F91E13209F437C3A0EB3B
:10778800BBE00E949571EA0FFB1F20831F5F45CF66
:107798002DC30E94A87D10E01A930E94D9730E94FD
:1077A80020750E947B6C0E9410470E94576E0E94B1
:1077B80024750E94D86D0E9426700E94326E0E9425
:1077C8007B6C0E94E06D0E9410470E9434700E94FA
:1077D800436EE7E0F0E0FA93EA930E94E06D0E94BE
:1077E8001047E091AE0BF091AF0B0E94E27A0E9435
:1077F800436E0E947B6C0E94D36D0E941047E4ED9B
:10780800F9E10E94E56DE091970BEF5FEA930E9422
:10781800ED41E7E0F0E0FA93EA930E94D36D0E940D
:107828001047C4DD0E94236EE091990BE03029F0E7
:10783800E091990BEA930E94ED4100E00330D8F5FE
:107848000E947B6CE02FED5FF0E00E94476E0E9483
:107858007872EA930E94ED41EBE2EA930E94AE4609
:107868000E947F72EA930E94ED410E94236E0E945B
:10787800867251F40E948E720E94396E0E943E6E8A
:107888000E94436EE3E709C00E948E720E94396E1F
:107898000E94C47B0E94326EE9E4EA930E94AE46DD
:1078A8000E94236E0E949872EA930E94F2410E94FD
:1078B80028750F5FC3CF0E9475433E2F3B3211F4EA
:1078C800133608F001C01F5F3D3211F4113008F47F
:1078D80001C011503D3439F41A930E94A81913DEDF
:1078E8001A930E94C819313209F056CF7FC20E94FC
:1078F800A87D10E00E943747012F0E947B6C0E94F0
:107908007B6C0E941047E8EDF9E10E94E56D31E0DB
:107918003C3018F51038F8F40E947B6C0E94166D04
:107928000E94476E1A930E94FD190E94576E0E948A
:10793800236EA091330CE3E00E942C75A091340CC7
:10794800E7E00E942C75E0912B06EA93E8E0EA93C1
:107958000E94A74113953F5FDBCF0E948A0E0E94C9
:1079680075433E2F3D34E9F50E944173102F1038BE
:10797800C0F51A930E94FD190E947B6C0E947B6CD3
:107988000E941F6EECEEF9E10E94E56D0E94576EB1
:107998000E9424750E945E6E0E941047EFEEF9E186
:1079A8000E94E56DE3E3FCE0FA93EA93E3E00E94CA
:1079B800057509F41BC20E945E6E0E941F6EE5EFFA
:1079C800F9E10E94E56DE4E3FCE0FA93EA93E7E06D
:1079D8000E94057509F40AC21A930E94311A1F5FA2
:1079E800C6CF313211F0103808F001C083CFFEC184
:1079F8000E94E66C0E9420750E947B6C0E941047D2
:107A0800EBEFF9E10E94E56D10E01530F0F41A9300
:107A18000E943F1A0E947B6C0E941B6F0E94576E47
:107A28000E942475E0912E0C0E943175E091310C72
:107A38000E943175E0912F0C0E943175E091300C55
:107A4800EA930E94F2411F5FE0CF0E9475430E2F18
:107A58000D34E9F50E94417310E01530C0F51A9312
:107A68000E943F1A0E947B6C0E947B6C0E941F6ED2
:107A7800EEE0FAE10E94E56D0E94576E0E942475BF
:107A880030E03430F8F40E945E6E0E941F6E0E944F
:107A9800166D0E94D57AEA56F94F0E94D37B0E9450
:107AA800E56D0E94166D0E94D57AEA56F94F0E943C
:107AB8003575FD013596E4910E94057509F496C166
:107AC8003F5FDFCF1A930E945F1A1F5FC6CF8EC138
:107AD8000E94576CE1E0EA930E94740F00E00732BD
:107AE80010F00C94333E0E94560E0E947B6C0E944C
:107AF8007B6C0E9410470E94FE6C0E9438750E94A1
:107B0800D37B31960E94E56D0E94236E0E94FE6C25
:107B18000E9438753496E491E038A9F40E944B6EBF
:107B28001E2FEDB7FEB7FA93EA931F93E0E1EA93AD
:107B38000EDB1F91E13209F492C0E12FA9E0B0E019
:107B48000E94067C88C0E238A9F40E94AB701E2F00
:107B5800EDB7FEB7FA93EA931F93E0E1EA93F7DAF9
:107B68001F91E13209F47BC0E12FAAE0B0E00E9446
:107B7800067C71C0E138E1F40E94A8741E2FEDB7AD
:107B8800FEB7FA93EA931F93E3E0EA93E0DA1F91D2
:107B9800E13209F464C00E94560E0E94A874E117ED
:107BA80031F0E12FA8E0B0E00E94067CFFCF53C07F
:107BB800E03069F40E94FE6C0E94387532960E948B
:107BC800E96DE1E00E94057509F449C044C0E1305F
:107BD80069F40E94FE6C0E9438750E943575FD019B
:107BE8003596E4910E940575D1F135C0E23061F413
:107BF8000E94FE6C0E94387532960E94E96DEFE093
:107C08000E941B7561F127C0E33071F40E94FE6C7D
:107C18000E9438750E943575FD013596E491EA9306
:107C28004FDAE132E1F017C0E430A9F40E94FE6CAB
:107C38000E94387532960E94D37BE093580CF093DB
:107C4800590C0E94F9720E9438753596E491EA93AE
:107C58004EDBE13221F00E94E4180F5F40CF09911A
:107C680019910895E8810E946373E2E9F9E10E949D
:107C7800E56D0C9497421A930E94417310E01330FB
:107C880010F00C94983E0E947B6C0E947B6C0E94C2
:107C98001F6E1A93E7DFECE0F0E00E94BC6C0E94D4
:107CA80010471A939FDB0E940A750E940E7551F4C3
:107CB8000E944B720E941875E2E00E941B7509F43D
:107CC800FFC209C00E944B720E941875E0E00E9432
:107CD8001B7509F4F5C2123028F50E947B6C0E94CE
:107CE8007B6C0E941F6E1A93BDDFE1E1FAE10E94EE
:107CF800E56DECE0F0E00E94BC6C0E9410470E9429
:107D08002875EAE0F0E00E94BC6C0E941047A0EBE6
:107D1800BBE00E9495710E948A6DE3E60E9405759A
:107D280009F4CEC21F5FABCFCBC20E94A87D10E082
:107D38001A930E94D9730E9420750E947B6C0E943E
:107D480010470E94576E0E9424750E94D86D21E04A
:107D580000E0033080F5E3E0F0E00E942D6D0E9422
:107D6800476E0A937FDF0E94867249F40E948E72E2
:107D78000E94396E0E943E6E0E94436E08C00E94A7
:107D88008E720E94396E0E94C47B0E94326E0A93E2
:107D980029DB2F5F023068F4E7E0F0E00E942D6DE8
:107DA8000E94476E0E9491720E945C6E0E94287524
:107DB8002F5F0F5FCECF0E9475433E2F3B3211F4E9
:107DC800133608F001C01F5F3D3211F4113008F47A
:107DD80001C011503D3439F41A930E94A8194BDFA1
:107DE8001A930E94C819313209F0A2CF0E94AF7DC0
:107DF800249608950E9441730E947B6C0E947B6CBC
:107E08000E941047E7E1FAE10E94E56DE1E0E093A6
:107E18002208E2E2F8E0FA93EA93E0E2EA9397D9DB
:107E2800089522970E94A67D0E9475430E2FE09127
:107E38001B08E03011F00C94C6400132D1F4EAE39B
:107E4800F6E0A091390CB0913A0CEA17FB0761F4FF
:107E5800E7E0E0931808EAE2EA93E0E2FAE10E9438
:107E6800A6700E946964A9C0E0E0E093C0050E9482
:107E78003D750D3331F4E091C005F0E00E941C6DB2
:107E880004910D3441F4EAE2EA93E3E2FAE10E9454
:107E9800A6700E946964063449F4E2E6F6E0E093CD
:107EA800390CF0933A0CE0E0E093C005003311F090
:107EB8000B3229F4E091C005EF5FE093C0050D3265
:107EC80029F4E091C005E150E093C005013329F49D
:107ED80091DFED3311F40E944475033329F48ADFEE
:107EE800ED3311F40E948037063329F4E0E0E09383
:107EF80022080E948037043329F4E0E0E093220846
:107F08000E944475A0912408A13010F40C945D409F
:107F1800023301F56FDFED33E9F40E945175D1F4B6
:107F2800E0912208EA930E94C61B30E0303190F4B9
:107F38000E94166D0E94777059F4E32FE05DEA9372
:107F4800E6E2FAE10E947C70E0E3EA930E948B6427
:107F58003F5FECCF053331F5E0E0E09322080E9463
:107F6800517501F511E01132E8F41A930E94C61B0D
:107F780030E03031A8F40E94166D0E94777071F4D9
:107F8800E32FE05DEA93E6E2FAE1FA93EA93E12F60
:107F9800E05DEA93E0E3EA930E948B643F5FE9CFF8
:107FA8001F5FE1CF013469F4EAE2EA93E9E2FAE11A
:107FB8000E942974E1E0E09318080E94AD7D28969C
:107FC80008950A3409F4B1DE073311F00C945D40CA
:107FD8000E943747E0E0EA930E94BB0EE1E0E0939D
:107FE8001C08E0E0F0E0E0931408F0931508EFE2D5
:107FF800F6E00E94A670E3E7F0E00E9458700E9445
:10800800C568EE83FF830E945A75E8E2F0E00E949B
:108018000E71B9F00E9407130E94C568EE83FF83B2
:10802800A091190CA03021F00E943C34E03009F4F2
:1080380008C00E945074E652F84FAEE0A0830E9438
:108048003B72E5E0F0E00E94986C40E050E00E944E
:108058002E22E03868F00E942E22EF573E2F313052
:1080680010F0313108F004C0E32F0E946271AF01B3
:108078005A934A930E94002040931408509315087D
:108088000091DB05E0E0E093DB05013211F00B32F3
:1080980009F401C0B8CF0B3221F4E1E0EA930E9461
:1080A800BB0E013209F0A3CFE0E0E0931C08E09397
:1080B800DB05A0912408A23011F00C94BF400933CD
:1080C80009F406DD053409F493DC033611F40E9443
:1080D800FE0D083309F45DDB023409F408DC0334CF
:1080E800A9F51091380C0E94374700E0E091370C51
:1080F800E11711F00C3008F01DC00E947B6C0E9443
:10810800FE6C0E94476E1A930E94541F1A9361D105
:108118000E94236EE091280C0E943175E0912B0C8F
:108128000E9431750E941E710E94326E0E94047175
:108138000395DCCF0E948A0ED4D20E2F013221F093
:10814800E091370CE11709F401C0CDCF043499F45C
:108158000E94517581F4A091D30BA03021F4A09115
:10816800D10BA03031F00E94AD730E947B6C0E944D
:10817800AA530E94A21DE0911B08E03011F40E944E
:10818800130F49C0E130D1F4A0912108AB3010F4AD
:10819800013209F405C00E9496160E948A0E0DC08D
:1081A800E0E0E0931E080E945F750E942974E0E0F9
:1081B8000E946475E2E0E0931B082DC0E23059F597
:1081C800013269F4E0E0E0931B080E943747EAE2D5
:1081D800EA93E3E2FAE10E9429740E94130F0B323A
:1081E80011F00D3359F40E945F75FA93EA93E1E3B5
:1081F800EA930E946964E1E00E9464750D3259F4C3
:108208000E945F75FA93EA93E2E3EA930E94696435
:10821800E2E00E946475A0911808A33009F404CE26
:108228000E94AD7D0C94E1451A93E3E0E0931908B0
:108238000E9437470E947B6C0E947B6C0E9410470B
:10824800EFE2FAE10E94E56D0E947B6C0E94E06D0E
:108258000E941047E3E1F6E00E94A670E0E1F0E03A
:108268000E94587010E0E091C90B1E1700F50E949B
:108278004B6EE117D1F0E12FE05DEA93E7E3FAE115
:10828800FA93EA93E0E3EA93E0E00E94837049F40A
:108298000E949571ED5EF94FA1E0A083E12FE05DAA
:1082A80001C0EEE2EA930E94AE461F5FDCCF0E9457
:1082B8003D75E0E0E093C005E0931B080E94130FB2
:1082C80019910895E881E03021F4E4EEF6E00E9487
:1082D8006975A881A13021F4EEEDF6E00E94697578
:1082E800A881A23021F4EAEEF6E00E946975A8811F
:1082F800A33021F4E8EFF6E00E946975A881A43064
:1083080021F4EEEFF6E00E9469750DC11A930A9305
:10831800E0E0E0937D05E0937E0510E0143190F4F1
:1083280000E0033068F4A3E01A9FF001EC57FA4F1D
:10833800DF01EE27A00FBE1FE0E2EC930F5FF1CF45
:108348001F5FECCFC1C31A9311E0E981E11780F0F8
:108358000E949571E255FF4FE491AA81EA2319F032
:10836800E12FE05D01C0E0E2EA93F4D41F5FEDCFB6
:1083780005C51A9311E0E981E11778F00E9495711B
:10838800E255FF4FE491AA81EA2311F0E1E301C02D
:10839800E0E3EA93DFD41F5FEECFF0C40E946E756E
:1083A8000E9473750E947C750E9490750AC10E9494
:1083B8006E750E9494750E949B750FC10E946E7520
:1083C800E1E5FAE10E94A1750E9434740E949B7550
:1083D80004C10E946E75E4E5FAE104C00E946E755E
:1083E800E8E5FAE1FA93EA93EE850E94D66CFE017D
:1083F8000E9490752B9608950E94A87D10E0E1E3F5
:10840800E0933809E89431F8EA930E941164ECE5A6
:10841800FAE10E94197300E0E09182050E17E0F47A
:108428000E94FE6CEC57FA4FE081E03258F4E3E228
:10843800EA930E943A630E94FE6CEC57FA4FE0817F
:10844800E05D05C00E94FE6CEC57FA4FE081EA93AC
:108458000E943A630F5FE0CF0E94A6759F010E94B9
:1084680008163A932A93E8ECF0E0FA93EA930E940C
:10847800D1680E2FA0E031FCA1E0A03011F400304B
:1084880009F001C0ECCF31FE09C0E0E0E0938205BD
:10849800E89431F8E1E00E94AF7DE3C41F5F123039
:1084A80008F4ADCFE0E0E09382050E94AF7DD9C427
:1084B800E0918105E03021F4E881EA930E94D25EE0
:1084C800A0918105A13069F4A0E09299A1E0A130C2
:1084D80021F4A8950E94466FF7CFE881EA930E949D
:1084E8007261A0918105A230F1F4E0918205F0E07B
:1084F800EC57FA4FA881A083E0918205EF5FE093E3
:108508008205E0918305EF5FE0938305A03218F4BC
:10851800EF5FE0938305A0918305A73321F46CDF17
:10852800E0E0E09383052196089508950E94C474BD
:108538000E94C47422D0EBE1EA93BADFE9E6EA9339
:10854800B7DFA0918105A13061F4E8ECF0E00E946A
:10855800B66EE0919A00E069E0939A00E9E1E09351
:108568009900A0918105A23021F446DFE0E0E09374
:108578008305E0E0E09381050895EDE0EA9398DF54
:10858800EAE0EA9395DF08951A9310E0E9811E174F
:1085980028F4EA81EA938CDF1F5FF8CFEFC3EDE29E
:1085A80001C0EDE3EA93E8E2EA93EEDFE6DF08953F
:1085B8000E946E750E9473750E947C750E94A67059
:1085C8000ED02E9608950E946E750E9494750E9492
:1085D800AA75FE010E94A67002D02C9608951A93DF
:1085E8000A9310E0EA81E03011F408E201C00A8140
:1085F800AB81BC81EE27A10FBE1FAC91A03011F05A
:10860800101708F007C0AB81BC810E94AF750E94AB
:10861800B475EECFEA81E03039F0EA811E1720F414
:10862800E0E20E94B475F9CF27C01A930A9310E0CC
:10863800EA81E03011F408E201C00A81E12FAB8140
:10864800BC810E94F074E491E03011F0101708F03A
:1086580009C0E12FAB81BC810E94F074E4910E94B3
:10866800B475ECCFEA81E03039F0EA811E1720F4C6
:10867800E0E20E94B475F9CF198108812596089522
:10868800E091C405A091C305EA17B1F00E94B9753D
:108698000E94396EEC91E093C6050E94B9750E945C
:1086A800AF71E181E093C505A091C4050E94BF7533
:1086B800E093C405E1E00895E0E008950E94C475E0
:1086C800A981A0830E94C4753196A881A083A09136
:1086D800C3050E94BF75E093C305BFC0E091DB05E9
:1086E80008951A93E091DB05E03059F40E940816CA
:1086F8000E94417221F4A091DB05A03009F001C06D
:10870800F5CF1091DB05E0E0E093DB050E944172B4
:1087180009F011E2E12FD6C30E94A87D0E94C56826
:108728008F010E940816EC81FD81E00FF11FFF9375
:10873800EF930E94C568AF91BF91AE1BBF0B9D011F
:108748000024021603061CF40E94417209F001C0BD
:10875800E8CFE0E00E94AF7D269608951A93E9815C
:108768000E94A572A0E0A0830E94CA75108117FF1D
:1087780005C0E12F0E94D175A0E0A08316FF05C0B7
:10878800E12F0E94D875A0E0A0830E94CA75A0E0DE
:10879800A083E9810E949F72A0E0A08318815DC038
:1087A8000E94A87D30E0EE81ADE0EA9FF001E05F35
:1087B800FC4F108116FF17C0E12FEF730E2F0E9498
:1087C800DF7511F03A3008F009C00E94E775DF0143
:1087D8000E94166D0E94ED753F5FF1CF0E94E7750C
:1087E8000E94E374EC9317FF17C0E12FEF730E2F6D
:1087F8000E94DF7511F0343108F009C00E94F3754A
:10880800DF010E94166D0E94ED753F5FF1CF0E9457
:10881800F3750E94E374EC930E94AF7D42C2E88135
:10882800F9810E94E96DEA81FB8132960E94E96D27
:10883800EC81FD8134960E94E96DEE81FF813696C8
:108848000E94E96DE885F9853896E491EA93E9850F
:10885800FA8539960E94FB6C02D022960895A0975B
:108868000E94A67DEDA5FEA5A9A9BAA9EA0FFB1F3E
:10887800AF01E5E0F3E0EE83FF8310E01431C0F5CB
:10888800AE81BF81AC91A03049F1EE81FF81A38117
:10889800B481EFA5F8A9EA17FB0701F5EE81FF817E
:1088A800A181B281E9A9FAA9AE17BF07BCF0EE8190
:1088B800FF81A181B2814A175B0784F00E94F97594
:1088C800AE0FBF1FE9A9FAA9AE17BF073CF00E9477
:1088D800F975AE0FBF1F4A175B070CF402C01A9355
:1088E8003DDFEE81FF813D96EE83FF831F5FC6CF9C
:1088F800E5E0F3E0EE83FF8310E0143110F00C9410
:108908002845AE81BF81EC91E03011F00C942145EF
:10891800EAA5EC93E9A9FAA9AE81BF811196ED9376
:10892800FC93EFA5F8A9AE81BF811396ED93FC9354
:10893800EDA5FEA5AE81BF811596ED93FC93EBA541
:10894800AE81BF811796EC93E0910904A0910F04C2
:10895800EA27AE81BF811896EC93E0911004AE81AE
:10896800BF811996EC93E0911104AE81BF811A96EC
:10897800EC93AE81BF811B960E94976D1C96E0E038
:10898800EC93E887E8A5F9A5309741F00E940476B2
:108998000E940976E4E1EA930E946E69EEA1FFA1C4
:1089A800309751F00E940476E8A5F9A5FA93EA9366
:1089B800E4E1EA930E945A69E0E0EC8F0E940476B1
:1089C8000E9445693E2F3B30C8F000E00E94F375D5
:1089D800E081E03011F0053008F002C00F5FF6CFFB
:1089E8000E94F375E081E03049F40E94F3750E941B
:1089F8000E76E058AE81BF811B96EC93E0E0EA8BDF
:108A08003130C8F000E00E94E775E081E03011F0F5
:108A1800043108F002C00F5FF6CF0E94E775E081CD
:108A2800E03049F40E94E7750E940E76E05CAE8162
:108A3800BF811B96EC93E12F08C0EE81FF813D9624
:108A4800EE83FF831F5F59CFEFEF0E94AD7DE39662
:108A580008951A930A930E9419763097A9F1E09124
:108A68006205E03061F50E94197604900092620573
:108A7800E0916205E03031F4E0E0F0E00E946975D1
:108A8800E0E01AC00E941E760E9419760E94D37BED
:108A9800F595E7958F01D801E0E0F1E00E944B7B66
:108AA800E0938700D801E0E0F1E00E947D7BE0934D
:108AB80086000E941E76E0E4E0938B0005C0E091FA
:108AC8006205E150E09362050991199108950E94A9
:108AD800A87D00E025E033E010E01431B8F5D901B5
:108AE800EC91E03079F111960E94C47B0E942676C1
:108AF80024F5D90113960E94C47BAC81BD81EA1785
:108B0800FB07DCF4F90101801280D90115960E9457
:108B1800C47BE00DF11DAE81BF81AE17BF076CF4B9
:108B2800F90103801480D9011796EC910E944772CD
:108B3800AC81BD81AE17BF070CF004C0E12FEF5F19
:108B48000E2F04C0235F3F4F1F5FC7CF003049F08F
:108B5800E0916305E01721F0A0916305A03009F4C6
:108B680001C022C0A0916405A53079F40A93E1E020
:108B7800EA93A4DD0093630500936505D901EC91A0
:108B8800E0936605E3E0E0936105A0916405AE31EA
:108B980019F4E4E0E0936105A0916105A33018F0B1
:108BA800E5E0E093680507C0E0E0E0936405E09342
:108BB80061050E942B760E94AF7D28960895E0916A
:108BC8006305E03091F0A0916405A93220F4EA939E
:108BD800E2E0EA9373DDA0916405AD3330F0E091F3
:108BE8006305EA93E4E0EA9369DDE0E0E093610578
:108BF800E09364050E942B76E0E0E0936305E09340
:108C08006705089530D182DB0895EA81E0937F05F6
:108C1800E881E0938005E0910A04E061E0930A04AA
:108C280020C10E94A67DA0917F05A43120F4A091C7
:108C38008005A33008F033C0E0917F05F0E0ACE098
:108C4800B0E00E94207B8F01E0918005F0E0A4E174
:108C5800B0E00E94207B9F010E943176ECE0F0E0BA
:108C68000E943676F0E00E94D37A0E94A16CEE81D1
:108C7800E030A9F0E0917F05A3E0EA9FF001EC570E
:108C8800FA4FDF01E09180050E941D704C91552735
:108C98000E9431764A93EFE0EA930E94CE4D0E94FB
:108CA800AD7D27960895E0910A04E07141F0E2E075
:108CB800EA93B7DFE0910A04EF7EE0930A0408958F
:108CC8000E943B76AF3EE0E0BE0744F4A091020369
:108CD800B0910303AF33E1E0BE070CF039C00E9446
:108CE80040760E942F700E94CE4DA0915D05B091F4
:108CF8005E05549734F4A0915F05B0916005139711
:108D08000CF012C0E0915D05F0915E05A3E0B0E0C3
:108D18000E94F87AEC57FA4FA0915F05B091600570
:108D2800EA0FFB1FA981A083E0910D04ACE0EA9F44
:108D3800F0010E943B760E94F0740E944D76E0910B
:108D48005D05F0915E053196E0935D05F0935E0553
:108D58000C94134BE881EA93E0911004EA93B0DF96
:108D68000C94E24A1A9310E00E945276E03031F0F7
:108D78000E945276EA93EEDF1F5FF6CF18812396A2
:108D880008950E9455760E945A76E03021F0083204
:108D9800E0E01E070CF007C00E945A76EA93DADF7B
:108DA8000F5F1F4FF0CF198108815BC00E94557675
:108DB800F801AB81BC810E94617621F0EA810E94B2
:108DC80066760CF009C0F801AB81BC810E946B7615
:108DD800C1DF0F5F1F4FECCF198108810EC30E94BE
:108DE800A87D0E943B760E94707631978F010E9481
:108DF80075760E9431760E947D7633C00E94A87DE8
:108E0800AC810E9484760E2F11270E9475760E94ED
:108E180031760E947D76F1C2EA81FB81E0935D059F
:108E2800F0935E05E881F981E0935F05F0936005B2
:108E3800AA81BB81ECE0F0E00E94207B0E944D7685
:108E4800A881B981E4E1F0E00E94207B06C0EA81B4
:108E5800FB810E944D76E881F981E0930203F0934B
:108E68000303249608950E948C76143120F41A93F3
:108E780075DC1F5FFACF0E947B6C0E947B6C0E949E
:108E88009C6CEFE3F1E00E94A16C10E0153048F40F
:108E9800A5E11A9FF001E051FB4FA0E0A0831F5FFE
:108EA800F5CF10E0143148F4ABE01A9FF001EC5E06
:108EB800FB4FA0E0A0831F5FF5CFE0910A04EF7E8F
:108EC800E0930A04199108950E948C76143100F5F4
:108ED800ADE01A9FF001BF01E85FFC4FDF010E947F
:108EE800C47B0F01DF01EB81FC81AE17BF075CF08B
:108EF800E981FA81E015F10534F0FB01E05FFC4FF0
:108F0800E081E03009F402C01A9328DC1F5FDECF4D
:108F18000E947B6C0E9494760E949C6CA985BA85FD
:108F28000E9499760E94A16C67C2A2970E94A67DB2
:108F3800E9A50E94A5728F01D8011B96EC91E0303B
:108F480009F415C2D8011B96EC91E9A3E07859F011
:108F5800FE013696FA93EA93EBA10E94D175FA9333
:108F6800EA930E942F69E9A1E07459F0FE01369650
:108F7800FA93EA93EBA10E94D875FA93EA930E94B8
:108F88002F69FE013696FA93EA930E944569E8A391
:108F9800E0910D04EB8FE0910E04EA8F0E94FF6EC2
:108FA800D80111962D913C91D80113964D915C9161
:108FB800D80115960E94C47BEEA3FFA3D80117968B
:108FC800EC91F0E0ECA3FDA3D8011896EC91EC8F9E
:108FD800E0910E04A0E10E945B6CEAA3FBA30E944F
:108FE8009E760E9409760E940976ECA1EA930E9477
:108FF800264CD8011996EC91EC8FE03011F4E8E09A
:10900800EC8F0E949E760E94A3765A934A930E9400
:10901800AA760E94AE760E94B5760E94B8760E9423
:109028009E763A932A930E94B876EEA1FFA10E94F9
:10903800BF765A934A930E94A3760E94B876A8A551
:10904800A130B1F43A932A93FA0131960E94B57689
:10905800FA013196FA93EA930E94AA76F9013196B9
:109068000E94C476F9013196FA93EA930E94B87681
:10907800A8A5A230F1F40E94AE7631970E94B57689
:10908800EAA5FBA5E40FF51F3197FA93EA930E942E
:10909800AA76EEA1FFA1E20FF31F31970E94C476D2
:1090A800EAA5FBA5E20FF31F3197FA93EA930E9412
:1090B800B876E8A5E03011F40C948B49D8011996DC
:1090C800EC91EC8FE0910D04ACE00E94C9760E940F
:1090D8004B7BED8FA8A1EA1710F40C94BA48E1E095
:1090E800E0930E04E03021F0ECA1FDA1B5970CF45B
:1090F80002C00E94CF76AAA1BBA1ECA1FDA1EA1BE8
:10910800FB0BDF010E949871EAA3FBA3ABA1AA2382
:109118001AF4E0E0EAA3EBA3A8A10E948476AEA12A
:10912800BFA1F0E00E94D776EE8FA8A5A13021F468
:109138000E94DA760E94DD76A8A5A23031F40E945A
:10914800DA760E94BF760E94E976E0E0E9A30E9401
:10915800EF76AE0FBF1FEC91E03039F00E94EF764A
:109168000E946B760E94F476F2CFD1C0E1E0E093E2
:109178000E04E03031F0ECA1FDA1E734A0E0FA07DD
:109188000CF402C00E94CF76E8A1EF8FEAA1FBA100
:10919800EE0FFF1FACA1BDA1AE1BBF0BE3E0F0E0DB
:1091A8000E944B7BEAA3FBA3ABA1AA2322F4E1E034
:1091B800F0E0EAA3FBA3EF8DE150EF8FEF8DF0E035
:1091C800DE011696AE0FBF1FAC91A03219F0AF8D1D
:1091D800A13008F404C0EF8DE150EF8FEFCFAF8DD1
:1091E8000E948476AE2FEEA1FFA1B0E0EA17FB073C
:1091F80014F3EF8DE03011F4ED8DEF8FAF8DECE0CF
:109208000E94C9760E94D776EE8FA8A5A13021F4D6
:109218000E94DA760E94DD76A8A5A23031F40E9479
:10922800DA760E94BF760E94E976E0E0E9A30E9420
:10923800EF760E94617621F0EF8DA9A1AE1708F0B4
:1092480007C00E94EF760E946B760E94F476EFCFFB
:10925800AF8DE8A1EA1BAE2FED8DEA1768F0AF8D50
:10926800E8A1EA1BACE0EA9FF001A0910D040E947E
:10927800C9760E94D77601C0E0E0EE8FA8A5A1309C
:10928800A1F40E94DA76E20FF31F31960E94367637
:10929800AFE00E945B6CE40FF51FDF01ECA1FDA1BC
:1092A8000E94AF7131960E94B26EA8A5A23089F4CF
:1092B8000E94DA76E20FF31F0E943676AFE00E9432
:1092C8005B6CE40FF51FDF01ECA1FDA10E9418758E
:1092D800BEDD0E94EF76AE0FBF1FAC91A03219F42D
:1092E800E9A1EF5FE9A30E94EF760E94617639F069
:1092F800AF8DE9A1EA1BAE2FED8DEA1708F407C080
:109308000E94EF760E946B760E94F476ECCFD8012B
:109318001C96EC91E03029F10E94FF6E0E949E7627
:1093280096DDF801A485A43698F4EFE0E0931004E4
:10933800F801A485AA3028F0A485AA930E94ED41DB
:1093480006C0D8011C96EC91E05DEA9303DD09C0E4
:10935800ECE0E0931004E2E5EA93FCDCEDE4EA9348
:10936800F9DCEB8DE0930D04EA8DE0930E040E9486
:10937800AD7DAA9608951A9310E0E89427F8143161
:1093880070F40E94DC6EE03011F00E94E36E1F5F03
:10939800A895E12FE37011F40E94FF15F0CFEFE0DC
:1093A800E09310040E94FF150C946B4E1A9310E082
:1093B8001431F8F40E94E86EB1F0A85FBC4F0E9427
:1093C800C47BDF01EB81FC81EA17FB0764F4F00141
:1093D800E85FFC4FDF010E94C47BDF01E981FA816D
:1093E800AE17BF070CF002C00E94E36E1F5FA8957E
:1093F800DFCFEFE0E09310041881259608951A93C3
:1094080010E0143190F40E94E86E31F0FD01E15F44
:10941800FC4FE081E17009F406C01A93E0910A0458
:10942800E170EA9382DD1F5FECCF0C946B4E2C97B2
:109438000E94A67DAD89BE890E9498710E94FC7623
:10944800EB8BFC8BED89FE890E940177EB89FC8907
:10945800E017F107FCF00E9434772E2F33270E9483
:1094680053770E945A770E9461770E9466770E941C
:109478005377F801A98DBA8D0E948A6D0E94617791
:10948800F8010E947077EA8DEA930E94894C0F5F79
:109498001F4FDCCF48C02C970E94A67DAD89BE899E
:1094A800E4E0F0E00E944B7B0E94FC76EB8BFC8BA7
:1094B800ED89FE89EE0FFF1F0E940177EB89FC8979
:1094C800E017F10784F10E943477AE2FED89FE8909
:1094D800B0E0EA0FFB1F9F010E9453770E945A7762
:1094E800E98DFA8DEE0FFF1F0E9470770E94667754
:1094F800ED89FE89EE0FFF1FA98DBA8DAE1BBF0B3C
:10950800BA93AA93F801A98DBA8D0E948A6D0E9418
:109518006177F8010E947077EA8DEA930E94894C7E
:109528000F5F1F4FCBCF0E94AD7D6B960895EA81E8
:10953800F0E0EBBBF5BBF7E1F09365001F98E6E1BF
:10954800E0936500F09365001F9AE881F981EBBB11
:10955800F5BB1F98FFE1F0936500EEE1E09365002D
:10956800F09365001F9A0C94DE4EE2E2EBBBE0E05C
:10957800E5BBE7E1E09365001F98E6E1E09365004D
:10958800E7E1E093650008951F9A0895A091040308
:10959800A23021F4E881A8E3B3E10BC0A091040351
:1095A800A43021F4E881A8E3B3E103C0E881A8E18D
:1095B800B3E1F0E00E94AF710E94D37B2196089539
:1095C800E0910403E23011F4EEE40AC0E43039F427
:1095D800E0E2EA93A981BA810E94707604C0E0E2D1
:1095E800EA93E981FA81FA93EA930E949B4A17C0A9
:1095F800E0910403E23011F4EFE40AC0E43039F4F6
:10960800E1E2EA93A981BA810E94747704C0E1E299
:10961800EA93E981FA81FA93EA930E949B4A229697
:109628000895E0910403E230B9F4E4E4EA930E9477
:109638007977AE0FBF1FFD01FE2FE0E0AF81B8853F
:109648000E948A6D0E949B4AE5E4EA930E94947600
:109658000E949B4AE6E453C0E33089F4E7E3EA93C7
:10966800FF81E0E00F010E947977EA0FFB1F0E945B
:109678007E770E9494760E949B4AE6E340C0E430DD
:1096880049F5E7E3EA93AF81B8850E947076DF0178
:10969800EB81FC81AE1BBF0BFD01FE2FE0E00F014B
:1096A800AF81B8850E9470760E947E77AD81BE81B9
:1096B8000E947477DF01E981FA81AE1BBF0BBA9370
:1096C800AA930E949B4AE6E3EA93AD81BE810E9479
:1096D80074771CC0E0E5EA930E94EB740E949B4AF1
:1096E800E1E5EA930E9479770E948A6D0E949B4A7D
:1096F800E2E5EA930E9494760E949B4AE3E5EA93A6
:10970800E981FA81AD81BE81EA0FFB1FFA93EA93E2
:109718000E949B4A28960895E0910403E33029F4B7
:10972800E3E0EA93E0E1F1E00BC0E43029F4E3E0A0
:10973800EA93E0E2F1E004C0E3E0EA93E0E3F0E179
:10974800FA93EA930E949B4A0895E0910403E33058
:1097580029F4E3E0EA93E1E2F1E00BC0E43029F414
:10976800E3E0EA93E1E1F1E004C0E3E0EA93E8E34F
:10977800F0E1FA93EA930E949B4A08951A930A9398
:10978800EFE10E948777EBE10E948777EFE10E9483
:109798008777E8EFFFEFE0935A0CF0935B0CE491C6
:1097A800EF3F39F0E0915A0CF0915B0C0490009275
:1097B8000403E6EBF3E18F01A0910403A23019F44E
:1097C800E8E9F3E18F01A0910403A43019F4E8E576
:1097D800F3E18F01F801E491ED3F39F4F801319696
:1097E8000E94E96D0E94A57A19C0EE3F71F4F80154
:1097F80031960E94D37BDF01E0910403F0E0EA1781
:10980800FB0711F00D5F1F4F09C0F801E491EA93BF
:10981800F80131960E94E96D0E949B4A0D5F1F4F27
:10982800F801E491EF3FB1F60E94746CE1E0E09337
:109838000E04E0930D04E4E1E09313046DDF099155
:10984800199108950E948B77AE85AA2362F0AD85A1
:10985800BE85A03FE0E0BE0734F4AB85BC85AF33DE
:10986800E1E0BE070CF050C00E949377AE0FBF1F17
:10987800A03FE0E0BE0734F0AD85BE850E9470765B
:10988800E987FA87EF81F885AB85BC85AE0FBF1FE6
:10989800A034E1E0BE0734F0AB85BC850E94747744
:1098A800EF83F8870E94F46D0E94F46D0E94F46DB6
:1098B8000E94F46DB6DE0E94F46D0E949877498587
:1098C80054DE0BBB15BB2EE13FE100E010E0EF8159
:1098D800F885E017F10764F050E0451730F0209361
:1098E8006500309365005F5FF8CF0F5F1F4FEFCFC4
:1098F8004BDE0E947B6C0E947B6C0E949C6CEFE3A9
:10990800F1E0FA93EA938DDEC9C00E948B770E943A
:109918009377EA17FB0741F0EF81F885AB85BC85A3
:10992800EA17FB0709F03EC00E94A0771CF00E94CE
:10993800A77784F42D853E85ED85FE85E987FA872E
:109948002D873E872B853C85EB85FC85EF83F88743
:109958002B873C870E94F46D0E9498770E9493772A
:10996800EA17FB0749F4F1DEEB85FC85ED87FE87F6
:10997800EF81F885E987FA87F8DD0BBB15BB2EE187
:109988003FE10D851E85E985FA85E017F1073CF072
:1099980020936500309365000F5F1F4FF4CFF4DD0F
:1099A800BBDE7CC000930B0410930C040E94AE77BE
:1099B8000E94B577FF93EF930E94B9770E94B5771D
:1099C800AF91BF91EA17FB0780F10E94A777B4F423
:1099D80020E030E00E94BC77E217F30774F00E94A1
:1099E800AE770E94C3770E94BC770E94C8770E9416
:1099F800D17758D02F5F3F4FEDCF16C020E030E031
:109A08000E94B977E217F3077CF00E94AE770E94B4
:109A1800C3770E94B9770E94C877F9010E94D87766
:109A280041D02F5F3F4FECCF39C00E94A077DCF4C4
:109A380020E030E00E94DC77E217F3079CF00E94F8
:109A4800B9770E94C3770E94DC77D0010E944B7BD4
:109A5800AF010E94D177FA010E94D87723D02F5FF7
:109A68003F4FE8CF1BC020E030E00E94AE77E217FE
:109A7800F307A4F00E94B9770E94C3770E94AE77DB
:109A8800D0010E944B7BAF01F9010E94D877FA01FF
:109A98000E94D87707D02F5F3F4FE7CF0E94AD7D58
:109AA8002F960895EA81FB81FA93EA9389DD0E9453
:109AB800E3779EDDE2E2EA93E0910B04F0910C0477
:109AC800FA93EA930E949B4A249608950E94A67DE1
:109AD80000910D0410E0E0910E041E1710F00C9494
:109AE800CD4DE885F985FA93EA9382DD2C853D858D
:109AF8004A855B85022E032A11F40C94C54D37FF65
:109B080036C05A934A935CDDE2E2EBBBE0E0E5BB8A
:109B1800E7E1E09365001F98F6E1F0936500E093B4
:109B28006500EE81EBBBEF81E5BBEFE1FEE1E09381
:109B38006500F0936500E093650001FF04C0F093B1
:109B48006500E093650036FF11C0F0936500E0936F
:109B5800650001FF06C0F0936500E09365004F5F64
:109B68005F4F220F331F4F5F5F4FEDCF1F9A220FBA
:109B7800331F01FF02C04F5F5F4F4F5F5F4F0C9471
:109B88007E4DE885F9853196E887F9871F5F0C9443
:109B98006F4D38C022970E94A67DE885EA930E94FF
:109BA800CA4AEE83FF83E985A8E1EA9FF001E85EEF
:109BB800F84F8F0130E0383028F5F801E4915E2F36
:109BC8000F5F1F4FF801E4914E2F407F0E94E87706
:109BD8000E94ED77EA87FB87F801E4914E2F440F46
:109BE800440F440F440F0F5F1F4FF801E4915E2F9D
:109BF8000F5F1F4F0E94E8770E94ED77EA87FB8787
:109C08003F5FD9CF0E94AD7D2E96089524970E947C
:109C1800A67DEA85EA930E94CA4AEE83FF8300E0A4
:109C280010E0EB850E946676D4F5EF85F889E88721
:109C3800F98720E030E0EC850E94FA772CF5E98975
:109C4800FA89449155273196E98BFA8B5A934A93AE
:109C5800EA85FB85FA93EA93E989FA89FA93EA9304
:109C6800EC85FD85FA93EA930E946A4DE0910D0414
:109C7800EE0FEE0FEE0FA885B9850E94F074E88705
:109C8800F9872F5F3F4FD7CFE0910E04AD85BE8592
:109C98000E94F074ED87FE870F5F1F4FC2CF0E94AE
:109CA800AD7D639608951A93EFEF0E946E72E0936C
:109CB800390910E00E949571E05CF54FE081EF3FB3
:109CC80031F00E9495710E94FF771F5FF3CF1991C1
:109CD80008951A930A930091CF0BAA81A53411F421
:109CE800E0E066C0AA81A23539F4A0913508A13018
:109CF80019F40E94027809F405C00E94FA1CE0E0F9
:109D0800E0933508AA81AB3411F0A33599F4E02F1C
:109D1800E470E43011F414E001C013E0E02FE270C5
:109D2800E23009F41C5FE02FE170E13009F41F5FB5
:109D3800E12F3EC0AA81A13511F0A13799F4E02F97
:109D4800E470E43011F417E001C016E0E02FE2708F
:109D5800E23009F41C5FE02FE170E13009F41F5F85
:109D6800E12F26C0AA81A33421F0A13411F0A23436
:109D780041F413E0E02FE170E13009F41F5FE12FB7
:109D880017C0AA81A73741F417E0E02FE170E1304E
:109D980009F41F5FE12F0CC0AA81A03441F415E03B
:109DA800E02FE170E13009F41F5FE12F01C0EFEF10
:109DB800198108812396089524970E94A67D2091F1
:109DC800CF0BA0914009A53411F00C94B24FE0E0FC
:109DD800E09335080E946772E0E0E0935D0BE09144
:109DE800D30BE030B9F5E0911008A0911108EA17FB
:109DF80039F00E940878ED55F84FE081E13009F01C
:109E080029C0E7E7EA930E943A630E940878E85578
:109E1800F84F0E94B4710E94A76D0E949A630E9435
:109E28000878EC55F84FDF010E94C47B0E94A76DAB
:109E38000E949A630E940878E755F84F0E940E78AE
:109E4800E2E0E09335080E940878ED55F84FA2E06B
:109E5800A08329DFE0913508E03011F00C94B24F6F
:109E68000E94027811F40C948B4F0E94EF1CE1E0E1
:109E7800E0933508E22FE870E83081F40E94137807
:109E8800E8EEF3E00E944B7BDF010E949C7D14F416
:109E9800E1E301C0E0E3EA930E943A63E22FE07451
:109EA800E03411F413E001C012E0E091230CF0E07B
:109EB8000E94C76D0E949A63E22FE470E43049F46F
:109EC8000E941378E0E1F7E20E947D7BAF0114E085
:109ED80006C00E9413780E94A073AF0113E0E22F1E
:109EE800E071E03111F4415050405A934A930E9476
:109EF800CE6D0E949A63E22FE072E03211F414E012
:109F080001C013E0E091260CF091270C17C018E06F
:109F1800E22FE470E43009F41F5FE22FE870E830C4
:109F280009F41F5FE22FE072E03209F41F5FE22FAD
:109F3800E074E03409F41F5FE0E0F0E0FA93EA939C
:109F48000E94CE6D0E949A63E22FE170E13029F4FD
:109F5800E0915D0BEA930E943A63A5DEA091400967
:109F6800A73729F4E2E0E0933508E03009F474C03B
:109F78000E9467720E9418780E941D731E2F0E940B
:109F88003873AF01E1E0EA930E94C8620E2FE091B6
:109F98001008A0911108EA1739F00E940878ED55C9
:109FA800F84FE081E23009F054C00E940878EC557F
:109FB800F84FDF010E94C47B4E175F0711F00C9425
:109FC80029500E940878E655F84F008011800E94B9
:109FD8004B6E0E94FC71EA17FB0771F10E9408782A
:109FE800E655F84FDF010E94C47B0E941E780E944C
:109FF8000878E655F84FDF010E94C47BEC59F44F0E
:10A008000E9426780E942A780E942E780E94CE6D9F
:10A018000E943178E3E6FAE10E941973003029F0D2
:10A028005A934A930E94716302C00E9437780E9433
:10A038003B780E942C6409C0003039F00E943F78B8
:10A0480020F40E9410740E94F026E1E1F8E00E94DA
:10A058004678E0E0E0933508A0914009A33421F464
:10A068000E943C34E03009F40BC00E9467720E94E1
:10A0780018780E94AD730E947B6C68D30E94A21D61
:10A08800A0914009A13411F0A23421F40E94677212
:10A098000E941878A0914009A03421F40E943C3411
:10A0A800E03009F420C00E941D73E887F987E2E0D8
:10A0B800EA930E94C8621E2F0E944A780E94FA18EA
:10A0C8000E9450740E945078E152F84F10830E9409
:10A0D8005074E652F84FA7E0A0830E943B720E949A
:10A0E80067720E941878A0914009AB3439F0A33503
:10A0F80029F0A13519F0A13709F076C00E943C3447
:10A10800E03011F40C94F2500E9467720E94577864
:10A11800E1E4F9E00E943373E22FE270E23029F4BF
:10A12800E4E0EA930E94C86202C0E1E0F0E0E88758
:10A13800F987A0914009A13511F0A13721F40E94B7
:10A1480038731E2F02C01091E50BE22FE470E43043
:10A1580011F4E4E001C0E3E0EA930E94C862AF01B1
:10A16800A0914009A33511F0A13731F4E885F985AC
:10A178000E94BF7AE887F9870E943F7820F0A09173
:10A18800D30BA13011F51A935A934A93EB85FC85AA
:10A19800FA93EA930E94C11D0E94B577EE83FF836C
:10A1A800AE81BF810E949C7D84F40E946772E6E6BE
:10A1B800EA930E943A63EE81FF813197EE83FF8331
:10A1C800AE81BF810E949C7D94F31A935A934A935F
:10A1D800EB85FC850E94F07266DD06C00E94AD73B7
:10A1E8000E947B6C0E94C11D0E94AD7D2A96089535
:10A1F8000E945B78E89422F80E942F74E2E7EA93C1
:10A208000E943A63E0913B08EA930E943A63EFE0C8
:10A21800EA930E943A63A0913808AA3219F41A9373
:10A228006AD31AC0A0913B080E949571EC59F44F6B
:10A23800E081EA1721F4E0913B08E03349F40E94F9
:10A24800196DAC59B44FE0913B08EC931A9353D372
:10A2580022FC02C00E942C64C5C20E945B78E09177
:10A268003B08E053AE2F0E949571EB58F44FE08104
:10A27800EA1741F51A933FD3A0913608A23019F492
:10A288000E94637809F402C00E946978A091360898
:10A29800A33019F40E94637809F402C00E94697817
:10A2A800E0E0E0933608E0935E0C0E949571EB586D
:10A2B800F44FBF01E081EF5FAE2FEAE00E947A7BA6
:10A2C800DB01EC938FC2E881E03019F40E94377803
:10A2D80006C0E881E8500E94AD740E94716321961F
:10A2E80008950E94A67D25FC2DC20E94637811F472
:10A2F8000C94F8520E946C78E752F84F9F01D901EC
:10A308001196EC91E43071F50E9472780E9475788C
:10A318000E947C78F901A681A03021F4A281B38142
:10A32800109709F007C0E6E6FAE10E9419730E9447
:10A338003B7815C00E942E780E9483780E9431785D
:10A34800E9E6FAE10E9419730E9487780E948D78E5
:10A35800F901A085B185BA93AA930E9471630E94FE
:10A368009378F0C1E730C9F40E9472780E9475783A
:10A378000E947C78ECE6FAE10E9419730E948778C3
:10A388000E943178EFE6FAE10E9419730E948378FF
:10A398000E9471630E949378D5C1E93089F40E94C4
:10A3A80072780E9475780E947C78E2E7FAE10E9450
:10A3B80019730E949A780E9431780E949378C2C1DA
:10A3C800E63029F5EAE2EA930E941164E5E7FAE14A
:10A3D8000E941973D901EC910E949D78E091CD0BF0
:10A3E8000E949D78EBE4EA930E943A630E94837886
:10A3F8000E947163E4E5EA930E943A630E948778B9
:10A408000E9471630E942C640E9469789BC1E530A8
:10A41800E1F40E9401740E941E78D901EC91EA933C
:10A428000E943A630E942A780E942E780E948378BC
:10A438000E943178E3E6FAE10E9419730E94877856
:10A448000E9471630E9493787DC1E83039F50E94BB
:10A4580072780E9475780E947C78E8E7FAE10E9499
:10A468001973F901A681AA930E940D74309719F007
:10A478000E94267004C0D9011696EC91F0E0FA9378
:10A48800EA930E9471630E943B780E942C64D90170
:10A498001196E0E0EC930E94697854C1E130C9F567
:10A4A800A0911908A53029F4E091CD0BE65F1E2F85
:10A4B80001C011E0E12F0E94A1780E9495710E94CD
:10A4C800A6780E942A780E942E780E9483780E949B
:10A4D8003178EBE7FAE10E9419730E9487780E94AD
:10A4E8008D78D9011796EC910E94AD740E94716322
:10A4F800A0911908A53041F40E94A978A481B581DA
:10A50800BA93AA930E94DB630E94A6750E94AF7853
:10A5180019C1E330B1F40E940174F0960E94BA7830
:10A528000E9401740E94A6780E942A78EEE7FAE158
:10A538000E9419730E9487780E94BE780E94AF78A3
:10A5480001C1EB3069F50E94C1780E94C4780E946D
:10A558002A78E1E8FAE10E941973F901A681AA9321
:10A56800B2DE0E94A978A781AA93ADDE0E94A978DD
:10A57800A085B185BA93AA930E948D780E948778A6
:10A588000E948D78F901A481B581BA93AA930E949B
:10A598008D780E949A780E94BE780E94AF78D2C0C7
:10A5A800EC3089F40E94C1780E94C4780E942A780D
:10A5B800E4E8FAE10E9419730E949A780E94BE7832
:10A5C8000E94AF78BFC0EE3079F40E94C1780E9433
:10A5D800C4780E942A78E7E8FAE10E9419730E9479
:10A5E800A6750E94AF78AEC00E94027861F0A09173
:10A5F8003608A03041F4A091D20BA13021F40E947A
:10A608004B6EE13009F427C0A091850BA03059F0BA
:10A61800E091870BF091880BFA93EA93E8EEF3E068
:10A628000E94B773C1F4E1E30E94BA78E091760B17
:10A638000E949D780E942A780E944B6EEA930FD15F
:10A64800E09336080E94A675E0935C0CF0935D0CCD
:10A65800E0E0E093850BA0913608A03059F0E09136
:10A668005C0CF0915D0CFA93EA93E4E6F0E00E944A
:10A67800B77309F025C0A0913608A23019F40E94DA
:10A68800637809F402C00E946978A0913608A33063
:10A6980019F40E94637809F410C0A0915E0CA330ED
:10A6A80030F00E946978E0E0E0935E0C06C00E94FA
:10A6B8006C78E652F84FA8E0A083E0E0E093360813
:10A6C800A091860BA130F1F5E091380CA091370CE0
:10A6D800EA1799F1EAE20E94BA78E091740B0E94B5
:10A6E8009D780E942A78E091380CEA930E94541FC2
:10A6F8000E942E78E091280C0E94AD740E94317857
:10A70800EAE8FAE10E9419730E941E71FA93EA932B
:10A718000E948D780E9498740E94C8780E942C64C8
:10A72800E091380CEA930E94991DE091380CEA9365
:10A738000E94681DE093380C05C0E0E0E093860BAA
:10A74800689420F80E94AD7D269608951A930A937E
:10A758000E943C34E030D9F00E945074E752F84F20
:10A768008F01EC81FD81D8011296ED93FC93EA816B
:10A77800FB81D8011896ED93FC93EE81D8011696CB
:10A78800EC93D8011196E4E0EC930E943B72198196
:10A79800088127960895E091420BEA930E943A6354
:10A7A800E091430BEA930E943A630895F4DF0E9414
:10A7B800E3770E94CB780E94CB780E94317899C0C9
:10A7C8001A930E9456621E2F103021F0E12FE1509B
:10A7D800E093400BE0DFE091400BEF5F0E94AD7427
:10A7E8000E943178199108950E94A87D31E00E9455
:10A7F800D27828F00E942773AC91A43308F02AC0BD
:10A8080030E00E942773EC91E270E6951E2F0E94BB
:10A818002773EC91E1700E2FA0915A0B1A1729F4A7
:10A82800E1E0EA27E0935A0B31E0A0915B0B0A17AD
:10A8380029F0E1E0EA27E0935B0B31E0E0915B0B64
:10A84800EE0FE05DA0915A0BEA0FEA930E943A637B
:10A858000E942074E32F0E94AF7D249608951A93D6
:10A8680010E00E94027811F40C9479540E94EF1CB5
:10A87800EEE8FAE10E941973E091230C0E94AD748E
:10A888000E943178E1E9FAE10E941973E091260CFF
:10A89800F091270C0E94C8780E941378A031E7E253
:10A8A800BE074CF4E4E9FAE10E941973E091240C24
:10A8B800F091250C13C0E7E9FAE10E941973E981C8
:10A8C8000E943B700E941378EA0FFB1F0E94DC7005
:10A8D800E091240CF091250CE051F742FA93EA93A9
:10A8E8000E9471630E943B7811E00E94D678E12FA4
:10A8F80018812296089524970E94A67D0E94D678F2
:10A908000E94FF61E13010F40C945357E091420B20
:10A91800EB3441F4E091430BE33219F40E945662A0
:10A928001E2FBAC2E435A9F4E091430BE33221F4B7
:10A938000E945662EE83FF83E091430BEF3441F4AB
:10A948000E9456621E2F1A930E94EB740E94FA18F6
:10A95800A3C2E23411F00C94F255E091430BE132BA
:10A9680051F4AA85AF3F29F40E94AD730E947B6C15
:10A97800EDDE0E94A21DE091430BE134E1F40E9458
:10A9880056621E2F113071F4A0913608A13019F4C7
:10A998000E94027809F402C00E94FA1CE0E0E093E9
:10A9A800850B09C0E1E0E093850B0E94C568E09340
:10A9B800870BF093880BE091430BE534A9F4EAE99F
:10A9C800FAE10E9419730E94D71CF3973CF00E9489
:10A9D80056620E94DC700E94DD7801C0E0E3EA93D1
:10A9E8000E943A630E943B78E091430BE634D9F425
:10A9F8000E94E97819F40E945662AF01E885F9854A
:10AA08000E942B700E2F033620F0A091D30BA1309B
:10AA180051F40E94F5780E94C11DAA85AF3F19F430
:10AA28000E94F57893DEE091430BE23511F00C9427
:10AA3800AF550E94E97819F40E945662AF0130E0E0
:10AA4800A091D30BA03021F40E944B6EE13009F0A5
:10AA580027C00E944234E03011F10E94E472EC55A4
:10AA6800F84FA885B985A083B1830E94E472E655A2
:10AA7800F84FDF01EA850E9437720E94E472E855B8
:10AA8800F84F10830E94E472E755F84F40830E9404
:10AA9800E472ED55F84FA1E0A0830E94EA7259C014
:10AAA8000E943C34E23010F40C94AD550E944A7870
:10AAB8000E94CE1E3E2F3F3F29F00E94F170A4173E
:10AAC800B5070CF412C00E949874E41BF50B0E94A1
:10AAD800FF700E94C17219F4E0E0E093280C3A93E9
:10AAE8000E945B1F689420F803C0E0E0E887E987CC
:10AAF8000E945074E752F84FDF01EA85F0E0EC5904
:10AB0800F44FE081EC930E9450740E945078EF510A
:10AB1800F84FDF01EA850E9437720E945074E152B3
:10AB2800F84F10830E945074E652F84FA5E0A083B6
:10AB38000E943B72E885F985309759F00E944A785F
:10AB4800FA010E94BF7A0E94F0720E94F5780E9472
:10AB5800491D689422F8E091430BE335F1F50E9412
:10AB68005662E887F9870E946C78DF01E652F84F51
:10AB7800E081E23081F4FD01EF51F84F008011804F
:10AB88000E944B6E0E94FC71EA17FB0721F4A0910A
:10AB98003608A23009F01FC00E946C78E552F84FC1
:10ABA800DF010E94C47BDF01E885F985EA17FB070E
:10ABB80079F40E946C78DF01ED51F84FE081EA9357
:10ABC800FD01E752F84FE081EA930E94F02603C0A6
:10ABD800E7E0E0932406689422F85EC1E43411F0BB
:10ABE8000C945B56E091430BE33559F4EDE9FAE137
:10ABF8000E9419730E94F75E0E949D78E1E0E0933D
:10AC08003909E091430BE03511F00C945A560E9433
:10AC1800F978E03011F40C945A5620E00E94FD783F
:10AC280040F00E942773AC91A23219F00E9401797A
:10AC380009F43CC0E22FE03061F40E942773AC9124
:10AC4800A33211F421E004C00E9405790E94D25E6B
:10AC58002AC0E13051F40E942773AC91A43211F458
:10AC680022E001C020E010E01EC0E23011F0E33025
:10AC7800D1F40E9405790E949D68EF3F99F0E12F79
:10AC8800E295E07FEF930E9405790E949D68AF915D
:10AC9800EA0F1E2F2F5F243021F41A930E94D25EF0
:10ACA80020E001C020E00E942074B8CFF5C0E33452
:10ACB80011F00C94C356E091430BE534B9F4EAE97A
:10ACC800FAE10E9419730E94D71CF3974CF00E9476
:10ACD8005662E05FF84D0E94DC700E94DD7801C08A
:10ACE800E0E3EA930E943A630E943B78E091430BC9
:10ACF800E634A9F441E050E00E9456620E2F0E940B
:10AD08000979E13019F40E945662AF011A930E9442
:10AD1800FE6CE05FF84D0E94C4760E94C11DE09170
:10AD2800430BE33591F40E940D790E942170E831BC
:10AD380031F4E091890BEA930E94A91806C0E885CE
:10AD4800EA93EFEFEA930E94F026E091430BE13497
:10AD5800A9F4E0EAFAE10E9419730E940D79EA93D6
:10AD68000E94A8190E942F26E03011F0E1E301C0EB
:10AD7800E0E3EA930E943A630E943B788DC0E6358F
:10AD880011F00C942857E091430BE33411F00C9424
:10AD980027570E9456621E2F113010F40C94275723
:10ADA800A0911908A13091F50E940979E03021F0AD
:10ADB800A091A2061A1709F028C011500E945662E5
:10ADC800AF011A930E94C2213E2F0E9467730E940E
:10ADD800AF710F010E9467730E94396E0E94147947
:10ADE8000E940979E03071F00E945662AF010E941A
:10ADF8007B730E94AF710F010E947B730E94396EB2
:10AE08000E9414791A930E9491121DC01630D8F42A
:10AE18001150A12FEAE00E942A7BA3E2EA9FF001E9
:10AE2800E855F94FBF01A12FEAE00E947A7BF0E0D4
:10AE3800BB01AAE0B0E00E94F87ADB01AE0FBF1FA9
:10AE480014960E94467128C0E93431F5E091430B0D
:10AE5800E03551F40E9456621E2FE0E0EA931A93FF
:10AE68000E947B19E0932E06E091430BEC34A1F489
:10AE78000E941A62E09328060E940979E03021F0C6
:10AE88000E941A62E09329060E940979E03021F0B5
:10AE98000E941A62E0932A060E94BE6131CD0E9488
:10AEA800AD7D2B960895A091580BA03521F4A09163
:10AEB800590BA33608F005C0E091590BEA930E949C
:10AEC800C819A091580BA33521F4A091590BAA30A9
:10AED80008F005C0E091590BEA930E94F319A0917C
:10AEE800580BAB3421F4A091590BA03808F005C0D9
:10AEF800E091590BEA930E94311AA091580BA6359C
:10AF080021F4A091590BA03108F005C0E091590B2C
:10AF1800EA930E945F1AA091580BA43511F40E947D
:10AF2800E418A4D60895E3EAF6E0FA93EA93E091E8
:10AF3800420BEA93E0E8F0E00E94587008950E94FE
:10AF48001C79A0E0A083E091400BE093590BE091BD
:10AF5800420BE093580B08950E94A67D0E94FF6162
:10AF6800E13010F40C94AE5AE091580BA091420BCA
:10AF7800EA1709F098DFE091420BE33239F5E091E6
:10AF8800430BEC3431F4CFDFE4E0E09318080E947F
:10AF98002279E091430BE435C1F4C5DFE091610CFF
:10AFA800E03029F0EF77A9E0B0E00E94067CE0915C
:10AFB800620CE03029F0EF77AAE0B0E00E94067C4E
:10AFC8000E942279E7E0E093180802C0EB34E1F52B
:10AFD800E091430BE13211F4A6DF35C0E53211F4FC
:10AFE80062DF31C0E33299F40E94287921F00E948F
:10AFF80033790E94FD190E941C79E081EB3429F411
:10B00800E0E0E093330CE093340C99DF1CC0E134AA
:10B01800D1F40E9456629F012093330C0E94397923
:10B0280091F00E9456629F01A091330CF901E270E1
:10B03800F070EA2BE093330C0E94397921F00E94DA
:10B048005662E093340C83C2E33581F5E091430BFB
:10B05800E13211F468DF29C0E33299F40E942879BB
:10B0680021F00E9433790E94D7190E941C79E0814F
:10B07800E33529F4E091400BEA930E94EA1B5FDF75
:10B0880014C0EE3491F40E94D07410E01A3068F4C1
:10B09800A3EBBBE0EE27A10FBE1F0E949571EC5BEE
:10B0A800F44FE081EC931F5FF1CF51C2E63511F008
:10B0B8000C94A658E091430BE13211F434DF41C0FF
:10B0C800E33299F40E94287921F00E9433790E9492
:10B0D8003F1A0E941C79E081E63529F4E091400B83
:10B0E800EA930E94721A2BDF2CC0E63531F40E94D5
:10B0F80056629F0120932F0C24C0E53471F40E94FE
:10B1080056629F0120932E0C0E94397929F00E94E3
:10B1180056629F012093310C14C0E43591F440E04D
:10B1280050E00E9456629F01022E032A11F042E06D
:10B1380050E00E94397919F00E945662AF0140939D
:10B14800300C05C2E43511F00C946059E091430BC2
:10B15800E33231F40E9456623197E093400BABC062
:10B16800E03511F00C945F5910E00E94FD7850F022
:10B178000E942773AC91AD3329F00E94017911F038
:10B188001E3008F005C00E9495710E943F79EDCFEE
:10B198000E9495710E944879EDE30E944D7911F063
:10B1A8000C945F59E4E5E093580B10E00E94BA70E4
:10B1B8003496E491EF3F11F40C945F590E94527950
:10B1C8000E94BA700E94E96D0E941D69E03011F07A
:10B1D8000C945D590E94BA703496E491E03851F4A9
:10B1E8000E945662E058FF4FE093610CE0E8E0935C
:10B1F800620C5FC0E23839F40E945662E058FF4F93
:10B20800E093620C56C0E13839F40E945662A8E017
:10B21800B0E00E94067C4DC0E03011F0E13051F4FE
:10B228000E94B070FF93EF930E945662AF91BF9156
:10B23800EC933FC0E23059F40E94B070FF93EF9353
:10B248000E945662AF91BF91ED93FC9332C0E330F8
:10B2580051F40E94B070FF93EF930E943562AF9152
:10B26800BF91EC9326C0E43021F50E94BA70359660
:10B27800E491EA930E941A630E94B070E0935F0C15
:10B28800F093600C00E00E94BA703596E4910E17B6
:10B2980080F40E94FE6CEC5BF44FE081A0915F0C9F
:10B2A800B091600CEC93AFE5BCE00E94D66E0F5FE6
:10B2B800EACF1F5F7BCF4BC1E03511F00C94AB5A3E
:10B2C800E091430BE33299F40E94287921F00E941F
:10B2D80033790E94A8190E941C79E081E03529F48D
:10B2E800E091400BEA930E94FF1B29DE30C1E13256
:10B2F80011F419DE2CC1E134D1F40E9456621E2FDC
:10B3080000E00D3098F40E94F474EA0FFB1F3396A6
:10B31800E491E11749F40E94F4740E94F874A09132
:10B328009A0BEA2BE0939A0B0F5FEBCF10C1E6352F
:10B3380059F5E0E0E093410BADE9BBE00E94577995
:10B34800FF93EF930E945662AF91BF91EC93EBE2AB
:10B35800EA930E94CE61E03059F0A0EABBE00E9477
:10B368005779FF93EF930E945662AF91BF91EC9388
:10B378000E945A79A091410BA33018F40E943979A0
:10B3880009F401C0D9CFE3C0ED34D1F4E0E0E09393
:10B39800410BA9EABBE00E945779FF93EF930E9403
:10B3A8005662AF91BF91EC930E945A79A091410BDC
:10B3B800A33018F40E94397909F401C0EACFC7C054
:10B3C800E735D1F4E0E0E093410BA0EBBBE00E944D
:10B3D8005779FF93EF930E945662AF91BF91EC9318
:10B3E8000E945A79A091410BA23018F40E94397931
:10B3F80009F401C0EACFABC0E434D9F5E0E0E0934A
:10B40800410B0E9456629F01E2E0EA930E94DB61D1
:10B41800AF01E3E70E944D7969F40E946079BF01AA
:10B42800D901E4E6F0E00E94207BE40FF51FDB0180
:10B43800ED93FC93E9E40E944D7979F40E946079D8
:10B4480020833183AAE9BBE00E9457790F010E944B
:10B458006679EC91E160D001EC930E945A79A09151
:10B46800410BA33018F40E94397909F401C0C9CFFF
:10B478006EC0EE3499F40E94D07410E01A3068F46B
:10B48800AAE8BBE0EE27A10FBE1F0E949571EC5BF6
:10B49800F44FE081EC931F5FF1CF59C0E33449F4D6
:10B4A8000E94F9780E945662E093950BF093960BF0
:10B4B8004EC0E33589F40E9456629F0100240216AB
:10B4C800030624F42B30E0E03E070CF004C0F90139
:10B4D8003197E093970B3BC0E53529F40E945662FB
:10B4E800E093990B34C0EF3491F40E9456621E2FFA
:10B4F800ECE2EA930E94CE61E12FE295E07FEF93C0
:10B508000E945662AF91EA0FE093980B20C0E03595
:10B51800F1F4E0E0E093410BACEABBE00E946C7907
:10B528000E94AF71FF93EF93E2E0EA930E94DF621B
:10B53800AF91BF91ED93FC930E945A79A091410B72
:10B54800A23018F40E94397909F401C0E5CF0E94AD
:10B55800BE6104CDE0E0E093430A0E94AD7D2696EB
:10B5680008950E94A87D0E94FF61E13010F40C94B8
:10B578006B5DE091420BE332A9F4E091430BE035B7
:10B5880019F4E3EAFAE109C0E83419F4E4ECFAE161
:10B5980004C0E33531F4EFEDFAE1FA93EA930E943F
:10B5A8004B6392C2E43511F00C94745BE091430B49
:10B5B800E43229F4E7E2F0E00E94707990C0E332C7
:10B5C80011F4FED88CC0E03511F00C94735BE3D80D
:10B5D800A091400BA73210F00C94735B0E94747911
:10B5E8000E94E96D0E944B63EDE3EA930E943A637F
:10B5F8000E9474793496E491E03839F40E944B6ED5
:10B608000E94AD740E9471636AC0E23839F40E94E6
:10B61800AB700E94AD740E94716361C0E13839F467
:10B628000E94A8740E94AD740E94716358C0E030F3
:10B6380011F0E13061F40E94747932960E94D37B54
:10B648000E94B471FA93EA930E94716348C0E23091
:10B6580059F40E94747932960E94D37BDF010E94CC
:10B668001B740E9471633BC0E33051F40E947479EB
:10B6780032960E94D37BE081EA930E947E632FC0BA
:10B68800E43069F50E94747932960E94D37BE09386
:10B698005F0CF093600C10E00E9474793596E49189
:10B6A8001E1790F40E949571EC5BF44F0F01A09166
:10B6B8005F0CB091600CEC91D001EC93AFE5BCE06D
:10B6C8000E94D66E1F5FE8CF0E9474793596E49188
:10B6D800F0E00E9448790E9452790E94C863F4C140
:10B6E800E33579F5E091400BEA930E94D719E09190
:10B6F800430BE43229F4EAE0F0E00E94707920C0BC
:10B70800E33211F45DD81CC0EE34D1F444D810E013
:10B718001A3068F40E949571EC5BF44F0F01A3EBAB
:10B72800BBE00E94AF75D001EC931F5FF1CFE0E062
:10B73800E0934E0B0E9452790E94C8630E943B78A6
:10B74800C3C1E635D9F5E091400BEA930E943F1A50
:10B75800E091430BE43229F4E5E0F0E00E947079CF
:10B768002CC0E33211F42CD828C0E53451F413D896
:10B77800E0912E0C0E94AD740E947879E091310C12
:10B7880019C0E63529F40E94CF53E0912F0C12C05E
:10B79800E43599F40E94CF53E091300CE03011F079
:10B7A800E1E301C0E0E3EA930E943A630E947E79F4
:10B7B800E091300CF0E00E94C87886C1E03511F0C5
:10B7C8000C94355DE091400BEA930E94A819E09132
:10B7D800430BE43229F4E3E6F0E00E94707940C1BB
:10B7E800E33219F40E94E4533BC1E13411F00C94A4
:10B7F8003F5C0E94CF5312E0A0919A0BECEDEA2334
:10B808003E2F00E00D3078F40E94F4740E94F87422
:10B81800E31739F40E94F474EA0FFB1F339614916E
:10B8280002C00F5FEFCF0E94CE6D0E943178E09189
:10B83800980BE03089F0EAEFFAE10E9419730E9450
:10B84800AD6D0E94AD740E947879E091980BEF700D
:10B858000E94AD740E943178E091990BE03051F06C
:10B86800EDEFFAE10E941973E091990B0E94AD7413
:10B878000E943178F5C0E43479F50E948279A0916C
:10B88800410BA33040F5E091410BE03011F00E94EC
:10B898007E790E946679EC91E17061F4A3EABBE0DD
:10B8A8000E946C790E94396E0E941B740E94DB63AF
:10B8B800E3E70BC0A3EABBE00E946C790E94396EF3
:10B8C8000E941B740E947163E9E4EA930E943A6340
:10B8D8000E945A79D4CFC0C0ED34C9F40E9482794D
:10B8E800A091410BA33090F4E091410BE03011F0AE
:10B8F8000E947E79A9EABBE00E948879EC910E94B7
:10B90800AD740E9471630E945A79EACFA5C0E735E9
:10B91800C9F40E948279A091410BA23090F4E09181
:10B92800410BE03011F00E947E79A0EBBBE00E9451
:10B938008879EC910E94AD740E9471630E945A79D3
:10B94800EACF8AC0E63531F50E948279A091410B91
:10B95800A330F8F4E091410BE03011F00E947E79B9
:10B96800ADE9BBE00E948879EC910E94AD740E9419
:10B978007163EBE2EA930E943A63A0EABBE00E949B
:10B988008879EC910E94AD740E9471630E945A7983
:10B99800DDCF62C0EE34D1F40E94CF5310E01A30EC
:10B9A80068F40E949571EC5BF44F0F01AAE8BBE0C4
:10B9B8000E94AF75D001EC931F5FF1CFE0E0E093F8
:10B9C8004E0B0E9452790E94C86346C0E33499F432
:10B9D8000E94CF530E945279E5E0FBE1FA93EA9383
:10B9E8000E9426700E9434740E94AA750E9452799F
:10B9F8000E94C86331C0E035A9F40E94CF53E0919A
:10BA0800AC0BF091AD0BFA93EA930E94DB630E94B2
:10BA18007E79E091AE0BF091AF0BFA93EA930E9416
:10BA2800DB631AC0E33531F40E94CF53E091970BE2
:10BA3800EF5F0DC0EF34A1F40E94CF530E94AD6DAB
:10BA48000E94AD740E947879E091980BEF70F0E055
:10BA5800FA93EA930E947163EBE3EA930E943A63D4
:10BA680033C0EB3489F5E091400BEA930E94FD194D
:10BA7800E091430BE43229F4E0E8F0E00E947079A9
:10BA880023C0E33219F40E94E4531EC0E134E1F408
:10BA98000E94CF53A091330CE1E0EA230E94AD74D9
:10BAA8000E947879A091330CE3E0EA230E94AD74F8
:10BAB8000E947879E091340C0E94AD740E94716301
:10BAC800E8E0FBE10E9419730E94BE614CCD0E9420
:10BAD800D6780E94AF7D249608951A930E946772C3
:10BAE800E0E4F9E00E9433730E94D6780E948C79D2
:10BAF800E181E43471F40E948C7902800E944B6EDB
:10BB0800E05DE01529F00E948C79E281EA3209F4BF
:10BB180001C057C00E9491790E948C79E1810E94EE
:10BB280095790E948C79E2810E9495790E94277309
:10BB38001C910E948C7933960E943373E12FE23175
:10BB480031F40E949B79E6E0EC9306DA3AC0E131E1
:10BB580031F40E949B79E2E1EC9303DD32C0EF30CF
:10BB6800A9F40E949B79EEE0EC930E94F853E1302F
:10BB780039F4A0913508A03019F00E94027809F430
:10BB880002C00E94FA1C0E94A1791BC0EE30C9F4C1
:10BB98000E949B79EFE0EC930E94F853E13089F41E
:10BBA800A0913508A03019F00E94027809F402C06B
:10BBB8000E94FA1CE0E0E0933508EFEFEA930E9458
:10BBC8007F5463C21A930E942F740E948870EAE718
:10BBD800EA930E943A630E94277311971C91E12F00
:10BBE800E23131F4E6E0EA930E943A63B5D937C00E
:10BBF800E13131F4E2E1EA930E943A63B2DC2FC00A
:10BC0800EF3099F40E942A780E94F853E13039F411
:10BC1800A0913508A03019F00E94027809F402C0FA
:10BC28000E94FA1C0E94A1791AC0EE30C1F4EFE01C
:10BC3800EA930E943A630E94F853E13081F4A0919C
:10BC48003508A03019F00E94027809F402C00E9459
:10BC5800FA1CE0E0E0933508EA930E947F54A09133
:10BC68003808AA3211F00E942C640FC2EFEFE0935B
:10BC7800580BE093590B0895AC81A03310F0AA3308
:10BC880008F006C00E94A879E0530E94B079CCC49D
:10BC9800AC81A13410F0A73408F006C00E94A8793E
:10BCA800E7530E94B079C0C4A881B981E0E0EC9361
:10BCB800BBC4AA93EA93FA93EFB7EA931A930A9349
:10BCC8001BB10CB1E0919B0CF0E0E759F34F0083F6
:10BCD800A0919B0CAF5FA0939B0CA23319F4E0E0FA
:10BCE800E0939B0C09911991F3C21A93E0919C0C73
:10BCF800A0919B0CEA17D1F3F0E0E759F34F1081BC
:10BD0800A0919C0CAF5FA0939C0CA23319F4E0E0C7
:10BD1800E0939C0CB9C1A0919B0CAE5CE0919C0C8B
:10BD2800AE1BE2E30E947A7B08950A921A92FA9275
:10BD38006A937A938A939A93AA93BA93EA93FA9313
:10BD4800EFB7EA930E94B57949F0A0913909A0307C
:10BD580021F00E94CA0DE13009F401C011C0E09140
:10BD6800020DF0E0E356F34FE081ECB9A091020D2B
:10BD7800AF5FA093020DA43619F4E0E0E093020D42
:10BD8800E991EFBFF991E991B991A99199918991B7
:10BD980079916991F9901990099018951A930E94D0
:10BDA800B57959F45D9B09C0A0913909A13021F4F6
:10BDB8000E94CA0DE03009F013C01091010D0E94D5
:10BDC8009571E356F34FA981A0831F5F143609F4D8
:10BDD80010E0E091020DE117E1F31093010D02C0AC
:10BDE800E981ECB9A1C20E94B57921F40E94CA0D7B
:10BDF800E13009F001C016C350C10E94A87D8BDF55
:10BE0800E03011F40C94FF5F70DF1E2FA091660CD8
:10BE1800A53618F0E0E0E0933A0930913A09E0914C
:10BE28003A09E03011F00C94665FA091E40BA13060
:10BE380021F0A091E40BA23031F4E12FEF77E093E9
:10BE48004009EBE4CEC01A3521F4E1E0E0933A0969
:10BE5800CAC0123049F4E4E1E0933A09E0E0E09323
:10BE68003B09E0933D09BFC0A091E40BA33069F4FE
:10BE7800173729F01A3310F4103308F402C0E7E03A
:10BE880001C0E0E0E0933C0905C01A930E946D4EA2
:10BE9800E0933C09A0913C09AF3F99F01093400909
:10BEA800E1E0E0933B0910933D09E0913C09E03063
:10BEB80011F4E5E404C0EAE0E0933A09E0E0E09335
:10BEC8003F0991C0E13069F4103039F4E2E0E093C1
:10BED8003A09E0E0E0933F0903C0E0E0E0933A0963
:10BEE80082C0E23059F410933C0910933D09E0E018
:10BEF800E0933B09E3E0E0933A0975C0E330F1F4DD
:10BF08000E94BB790E94C179EA0F0E94CB79A9F4FB
:10BF1800E0913D09E03071F4E4E0E0933A09E09102
:10BF28003B090E94D46F0E94D4790E94BB79A0E09B
:10BF3800A08303C0E0E0E0933A0955C0E43049F437
:10BF48001D3019F4EAE5E0933F09E0E0E0933A098F
:10BF58004AC0EA3079F40E94BB790E94C179EA2785
:10BF68000E94CB7931F4E0E0E0933A09E5E4E0930C
:10BF78003F0939C0E431B9F40E94BB791083E12F3D
:10BF8800A0913D09EA27E0933D09E0913B09EF5F65
:10BF9800E0933B09E0E0E093650C133019F4E5E128
:10BFA800E0933A0920C0E53111F0E63159F41A93CB
:10BFB800E5E6FCE0FA93EA93EAE3F9E0FA93EA9318
:10BFC8005BDE11C0E73179F4E0E0E0933A0917311C
:10BFD80031F4E091650CA0913D09EA1709F003C01E
:10BFE800E3E4E0933F09A0913A093A1719F0E0E039
:10BFF800E093660C04CF0E94AF7D70C4AA93BA93F5
:10C00800EA93FA93EFB7EA931A930A9310919B0075
:10C0180000919C00E12FEC71A9F4E091CB0DF09117
:10C02800CC0DED5FF24F0083ABECBDE00E94D66E05
:10C03800E83CA0E0FA0731F4E0E0F0E0E093CB0D53
:10C04800F093CC0D09911991E991EFBFF991E9911C
:10C05800B991A99118951A930E94D9790E94DE790D
:10C06800D9F30E94D979ED5FF24F1081ADECBDE0B4
:10C078000E94D66EE83CA0E0FA0731F4E0E0F0E078
:10C08800E093CD0DF093CE0DE12F199108950E9404
:10C09800D9790E94DE7909F0C5C1E0E008950E94CF
:10C0A800A87DF5DFE03021F0A091640CA03009F004
:10C0B800E5C0D1DF1E2FA091D70DA53618F0E0E01E
:10C0C800E093D10D3091D10DE091D10DE03059F4CC
:10C0D800113019F4E4E0E093D10D1A3519F4EAE0CF
:10C0E800E093D10DC3C0E430C1F4E0E0E093D10D9A
:10C0F8001A3229F00E944B6EE05DE11769F4109343
:10C1080038081093D20DE5E0E093D10DE0E0E0931C
:10C11800640CE1E0E093D40DA9C0E530A9F4E0E0B7
:10C12800E093D10D0E944B6EE05DE11761F00E9433
:10C13800E5790E94EE79E091D40DEF5FE093D40D9C
:10C14800E6E0E093D10D92C0E63091F4E091D40D91
:10C158000E94EE790E94E579EF5FE093D40DE0E06C
:10C16800E093D50D133019F4E7E0E093D10D7EC0CC
:10C17800E73011F0E83059F41A93E5EDFDE0FA9351
:10C18800EA93E1EDFDE0FA93EA9376DD6FC0E930DA
:10C1980081F4E0E0E093D10D173131F4E091D50D51
:10C1A800A091D20DEA1709F003C0E4E5E093640C0E
:10C1B8005DC0EA3041F4103011F4EBE001C0E0E07A
:10C1C800E093D10D53C0EB3071F4E0E0E093D40D6F
:10C1D8001093D30D1093D20DECE0E093D10DE0E075
:10C1E800E093640C43C0EC30A1F5E091D40DF0E08D
:10C1F800E05CF64F10830E94E579EF5FE093D40D81
:10C20800E091D30DE150E093D30DA091D30DA03070
:10C2180021F4A091D20DA03009F00EC0EDE0E0931A
:10C22800D10DE091D40D0E94D46F0E94D479E09191
:10C23800D40DF0E00E94D479A091D30DA03021F460
:10C24800A091D20DA03009F403C0E0E0E093D10D35
:10C258000DC0ED3059F4E0E0E093D10D1D3031F41C
:10C26800EAE5E093640CEFEFE093630CE091D10D05
:10C27800E31719F0E0E0E093D70D13CF0E94AF7DEC
:10C288002DC3AA93EA93FA93EFB7EA93E091D90EF4
:10C29800A091D80EEA1791F0E0913708E03019F034
:10C2A800E89426F80AC00E94F379F0E0E030A1E0B3
:10C2B800FA0719F4E0E0E093D90E03C0E89425F8F2
:10C2C80026F8E091630CE03019F0E0E0E093D10D3E
:10C2D800E991EFBFF991E991A99118951A93E09125
:10C2E800D90EA091D80EEA1721F4E0919B00E072D4
:10C2F800C1F4E091D80EF0E0E852F24FA981A08392
:10C308001091D80E1F5F0E94196DA030E1E0BE07A2
:10C3180009F410E0E091D90EE117E1F31093D80E7B
:10C3280003C0E981E0939C00188122960895E0E01B
:10C33800E093D90EA091D80EA13020F00E94F37995
:10C34800689426F80895AA93BA93EA93EFB7EA9304
:10C35800E091630CE03041F4E0E0E093D90E0E94F4
:10C368004B6EEF5FE0933708E991EFBFE991B99120
:10C37800A99118950E94FD7818F00E94017909F496
:10C3880003C00E942074F6CF0E94017911F40E9424
:10C39800207408950E942773AC91E881EA1729F464
:10C3A8000E9420743197E1E070C1E0E06EC10E9404
:10C3B800017AEEE20E944D79E9F420E030E0EC8168
:10C3C8000E94FA77BCF4D8010E94DE748F010E94A3
:10C3D800D27818F00E94067A08F009C00E942773E4
:10C3E800EC910E94A5730E0F1F1F0E9420742F5FEF
:10C3F8003F4FE5CF16C10E94FD7828F00E948C7946
:10C40800E181E03208F410C00E942773EC91E093B8
:10C41800420B0E9420740E942773EC91E093430B17
:10C428000E942074E1E008950C94FF660E945576FE
:10C438000E9405790E949D68EF3F89F0F8010E94EB
:10C44800D37AFF93EF930E9405790E949D68AF917C
:10C45800BF910E94F0748F010E942074E9CFF80107
:10C468001EC01A930A9310E00E9427730C910B3395
:10C4780011F0003208F412C0013310F0093308F04B
:10C4880007C0E02F0E94A573E255FF4FE4911E2BD1
:10C498000E9420740E9427730C91E9CFE12F099123
:10C4A800199108950E94017A0E942773AC91AD32C8
:10C4B80021F40E94207431E001C030E00E94D2785B
:10C4C80018F00E94067A08F009C0D8010E94DE74AC
:10C4D8000E940A7A8F010E942074F0CF303021F434
:10C4E800F8010E94AF7DFAC1F8010E94BF7A0E944C
:10C4F800AF7DF4C124971A93E0E0E983EA83EB83E4
:10C50800EC830E942773AC91AD3221F40E94207411
:10C5180011E001C010E00E94D27818F00E94067A5B
:10C5280008F022C0A981BA818B819C81EAE0F0E001
:10C5380060E070E00E94257B7F936F93FF93EF93F9
:10C548000E942773EC91E053AF91BF918F919F9117
:10C55800FF27662777270E94B57AE983FA836B83DA
:10C568007C830E942074D7CF103031F4E981FA819E
:10C578006B817C81188158C0E981FA816B817C814B
:10C588000E94C37A188150C00E94A87D20E030E044
:10C5980000E010E0EC810E9466765CF4D9010E940C
:10C5A800DE740E940A7A9F010E9420740F5F1F4F59
:10C5B800F1CFF90137C00E94017A20E030E00E94F3
:10C5C800D27818F00E94067A08F013C0AC81A13026
:10C5D80030F0D8010E94DE740E940A7A8F0131E09F
:10C5E800213018F0AC81A13008F403C0EC81E1508F
:10C5F800EC830E942773AC91AE3211F422E031E053
:10C60800313011F40E9420743130C1F2AC81A13074
:10C6180040F0D8010E94DE748F01EC81E150EC8378
:10C62800F5CFF8010E94AF7D259608951A9310E082
:10C638000E94F978E030A1F00E94FD7858F00E943D
:10C648002773AC91A23231F00E94017919F0E98187
:10C658001E1708F005C00E9495710E943F79ECCF23
:10C668000E9495710E9448790C945B67E8810E944A
:10C678009579E881A0915C0BEA0FE0935C0BE88167
:10C68800A0915D0BEA27E0935D0B219608951A931C
:10C6980010E0E12FA981BA810E94F074E491E030A2
:10C6A80051F0E12FA981BA810E94F074E491EA93D4
:10C6B800DDDF1F5FEECFAEC01A9310E00E949571C8
:10C6C8000E94107A41F00E949571EC5BF44F0E9431
:10C6D80026781F5FF3CF0C94FA660E9452790E9465
:10C6E800157AEC81FD810E9434740E94AA75E4DFFA
:10C6F8000C945C671A93ECE3EA93B8DF11E0193005
:10C7080080F40E949571E255FF4FE491A981EA23D4
:10C7180019F0E12FE05D01C0E0E2EA93A7DF1F5FB7
:10C72800EECFEEE3EA93A2DF0C945B671A930E94C4
:10C7380052790E94157AEF81F8850E9434740E941C
:10C74800AA7510E00E9495710E94107A11F01F5F7F
:10C75800F9CFE981FA810E94196DAE17BF0724F459
:10C768000E9437781F5FF5CFA7DF18810C941B69EB
:10C778000E9452790E94157AEC81FD816E817F8139
:10C788000E94817499DFAAC01A93E2E2EA936EDFED
:10C7980010E00E945276E03031F00E945276EA931F
:10C7A80065DF1F5FF6CFE2E2EA9360DF33C01A93DA
:10C7B8000E945279E6E1FBE1FA93EA93AD81BE81EA
:10C7C800E4E6F0E00E944B7B0E943474A985BA85A8
:10C7D800E4E6F0E00E947D7B0E94347488E00E94C9
:10C7E800716B2C9610E00E9495710E94107A91F05E
:10C7F8000E949571EC5BF44FE081E03211F4E0E3C4
:10C8080005C00E949571EC5BF44FE081EA932EDF3E
:10C818001F5FE9CF18812396089525FE06C0E5E03D
:10C82800F0E00E94B66EA895F8CFE8EDFDE0E09341
:10C838005E0BF0935F0BE1E00E946E72E0935C0B7D
:10C848000E941A7A0E944B6E0E949D780C94866909
:10C858001A930A93E091630CE03011F00C94CE68BF
:10C86800E3E0EA9303DFE0915C0BE295EF70EA9373
:10C878000E94B4681E2FE0915C0BEF70EA930E944F
:10C88800B4680E2F1A93F2DE0A93F0DEE7E1EA931A
:10C89800EDDEE8EDFDE0A0915E0BB0915F0B0E942C
:10C8A800E77BEA1BE093D80E689425F80C94CE68D1
:10C8B800EE81EA93B2DFEC81FD810E9419730E9438
:10C8C8001E7A56DFC5DF0C94AD69EB81EA93A5DFCC
:10C8D8000E949071DCDE0E941A7ABADF24960895CD
:10C8E800ED81EA939ADFEB81FC810E941973EA815A
:10C8F800EA93BCDEE981E03011F0EA93B7DEE88123
:10C90800E03011F00E941A7AA3DF269608950E945B
:10C91800A67D10E0EDE1FBE1A885B985EA17FB07E4
:10C9280019F444E150E002C048EC50E0EA85E09395
:10C938003809E89431F8EA93E985FA85FA93EA9395
:10C94800EA85EA93EA85EA93E0E0EA93C9DF0E9480
:10C95800C5689F010E9408160E949E760E94D168B1
:10C968000E2F31FC02C0003009F001C0F3CF31FEB8
:10C9780004C0E89431F8E1E004C01F5F1230B0F25F
:10C98800E0E00E94AD7D2B9608951A930A93E091FA
:10C99800400AE03011F40C94CE68E0E0E0933909E5
:10C9A800E2E0EA93FBD910E003E00E9495710E944F
:10C9B800257A61F00E9495710E94FF770E94957117
:10C9C800E05CF54FE0810E271F5FEFCFE3E0EA93CD
:10C9D800E5D9E02FE295EF700E942A7AE02FEF70F8
:10C9E8000E942A7AE7E1EA93D9D90C94CE681A937F
:10C9F8000A93E091400AE03011F40C94CE680E944A
:10CA0800AB70E03021F0E091420AEA3209F405C047
:10CA18000E94AB70E05DE093420AE0E0E0933909E0
:10CA2800EAE5EA93BBD9E0E0EA93B8D910E00E94BE
:10CA380095710E94257A11F01F5FF9CF1F5F012FB2
:10CA48000A93ACD910E00E9495710E94257A61F092
:10CA58000E9495710E94FF770E949571E05CF54FE6
:10CA6800E0810E0F1F5FEFCFE02FE195EA9396D993
:10CA7800EDE0EA9393D90C94CE681A930A93F8944C
:10CA8800E0E0E0933708E091D90EE093D80E78946F
:10CA9800E091400AE03011F40C94CE68EAE5EA939C
:10CAA8001DDCE0E0EA931ADC10E00E9495710E9418
:10CAB800257A11F01F5FF9CF1F5F012F0A930EDC53
:10CAC80010E00E9495710E94257A79F00E94957174
:10CAD800E05CF54FE081EA9301DC0E949571E05C2F
:10CAE800F54FE0810E0F1F5FECCFE02FE195EA9341
:10CAF800F5DBEDE0EA93F2DB0C94CE68E881EA938B
:10CB08008CDEEAE5EA93B2DDE0914009EA93AEDD16
:10CB18000E942773EC91E03031F00E940579A6DD80
:10CB28000E942074F5CF94DE0C9486691A930E94B3
:10CB38006772E0913B08EA9399DDE4E4EA9396DDB5
:10CB4800E0913908EA9392DD14E00E949571E85C5F
:10CB5800F74FE081E43040F00E949571E85CF74FB0
:10CB68000E9426781F5FF1CFE0E0EA937FDD3FDF88
:10CB78003DC11A930A9341D9E0913F09E03011F47D
:10CB88000C943A66A0913F09AA3541F4A0913B095B
:10CB9800A33020F0E0914109E43409F04BC00E9431
:10CBA800AB70E03021F0E0914209EA32C1F40E9412
:10CBB8004B6EE05DA0914209EA1721F0E09142092D
:10CBC800EA3221F40E94715D12DF08C0E3E4F9E063
:10CBD8000E943373E09142090E94307A2BC00E9470
:10CBE800AB70E05DA0914209EA1721F50E944B6EF7
:10CBF8001E2FE0914309ED3421F4E0914409E3321A
:10CC080009F007C0E5E4F9E00E9433734BDC1E2FFE
:10CC1800B1DB0E944B6EE11729F0E12FE05D0E9425
:10CC2800307A08C00E944B6EE05DE09342090E9492
:10CC3800715DDDDEA0913F09A53449F4A091E40BB4
:10CC4800A33019F40E94762B02C00E94E04EA091F6
:10CC58003F09A33411F40E942E2BA0913F09AB3455
:10CC680011F40E94292BE0E0E0933F09A091E40B26
:10CC7800A33011F40E94762BE0E00C94CE680FDA12
:10CC8800A091640CA43529F4A0E025FCA1E0A03013
:10CC980009F03AC0E0913A08E03581F4E0913B08A8
:10CCA800EA93E6E0EA930E946243A0913B08A03829
:10CCB80020F0E0913B08E093650523C0E03721F4BC
:10CCC800E0E0E09365051DC0EA3519F40E94E65DD1
:10CCD80018C0EA3711F42ADF14C0E23519F40E94AB
:10CCE800FC500FC0E23719F40E9431510AC00E946B
:10CCF800FA30E0913908A0913809EA1711F46894DC
:10CD080031F8E0E0E093640CA091640CAA3531F4AA
:10CD18000E94715DB2DEE0E0E093640C6CC0A0910B
:10CD2800670CA13050F0E091670CE150E093670C7C
:10CD3800E03019F4E1E0E093680CA0E025FCA1E004
:10CD4800A13049F4A0E026FCA1E0A03021F4A09194
:10CD58003708A03009F001C0EADAE0913708E0307E
:10CD680019F0E150E09337080895E091D70DEF5F8F
:10CD7800E093D70DE091660CEF5FE093660CE091CD
:10CD8800630CE03019F0E150E093630C0895A09132
:10CD9800E40BA13021F0A091E40BA23029F4E3E0E8
:10CDA800E0939000E8E3E9B90895E0E00E943B6C65
:10CDB800E1B3E360E1BB85E38A95F1F7E1B3EC7F8A
:10CDC800E1BBE4E4E09374000E94526C08951A9366
:10CDD80014EAE4EA0E94377A41F40E943C7A183057
:10CDE80011F0103111F4E0E001C0E2E0199108956A
:10CDF800E4E9E0937400E0E008951A93E981E160C2
:10CE08000E94417A31F40E943C7A103411F4E0E037
:10CE18004EC04CC01A93E9810E94417A31F40E94B5
:10CE28003C7A183111F4E0E042C040C01A93E9811D
:10CE38000E94417A31F40E943C7A183211F4E0E001
:10CE480036C034C01A93E981E03011F0E4EC01C037
:10CE5800E4E80E94377A79F40E943C7AE091730002
:10CE6800AA81BB81EC93103511F0183521F4E0E06C
:10CE780018810C94036CE1E018810C94036C1A93EC
:10CE8800E981E093740010E0E0917400E07811F417
:10CE9800163908F005C08BE18A95F1F71F5FF4CFCA
:10CEA800E0917400E07811F0E0E001C0E1E0188161
:10CEB800229608950E94A87D3D810C8120E087DF9D
:10CEC800E03011F5EE810E94616FF1F43A93AEDF24
:10CED800E030D1F40E94457AB9F479DFE030A1F46A
:10CEE800EE810E94496C81F4EDB7FEB7FA93EA939C
:10CEF8001F930E944E6C1F91E03031F479DFE12FCF
:10CF08000E94AF7D0C94AD6950DFD9CF0E94A87DF7
:10CF180030E00E811D815BDFE03099F4EF810E94E3
:10CF2800616F79F40E94457A61F41A937FDFE030EB
:10CF380041F4EC81EA937ADFE03019F459DFE0E05C
:10CF480002C033DFE8CF0E94AF7D2896089522976C
:10CF58000E94A67D50E02B853A85A89538DFE03001
:10CF680011F00C940D68EE850E94616F11F00C941D
:10CF78000D682A935BDFE03011F00C940D683A934A
:10CF880055DFE03011F00C940D6821DFE03011F02E
:10CF98000C940D68EE850E94496CD9F5E0E0EE83AB
:10CFA800EF83EC85FD8531970E94267649F4EDB72D
:10CFB800FEB7FA93EA931F930E944E6C1F9109C023
:10CFC800EDB7FEB7FA93EA931F93E1E0EA933ADFED
:10CFD8001F910E2FEE81FF81A885B985EA0FFB1FEF
:10CFE8001083EE81FF813196EE83FF83003039F4A0
:10CFF800EC85FD85AE81BF81AE17BF0708F001C083
:10D00800D0CFEC85FD850E94267619F4F1DEE0E0AC
:10D0180002C0CBDEA3CF0E94AD7D2F9608956897FE
:10D028000E94A67D20E0E0E0EC8FED8F31E0A8952E
:10D03800E9A1FAA1662777270E947D7CEA87FB870A
:10D048006C877D87EE8D0E944A7A0E940A700E9442
:10D058000F70AA85BB858C859D850E94537DEA8BC0
:10D06800FB8B6C8B7D8B0E94D77BFE017296FA93AB
:10D07800EA930E94056CEE8BFF8B688F798F0E9474
:10D08800507A0E94447CAF010E94507AAE8DBB2733
:10D09800882799270E94DE7B0E94637ADE015A96D0
:10D0A8000E94447CED93FC930AA119A190DEE03024
:10D0B800D1F5EDA10E94616FB1F50E94457A99F50D
:10D0C8001A93B4DEE03079F5303051F14F5F5F4F9D
:10D0D800EC8DFD8D3196EC8FFD8FAC8DBD8D11974C
:10D0E800EBA1FCA1EA17FB0711F430E018C0EC8DA6
:10D0F800FD8D3197AF8DB8A10E946B7697DEEE8DCE
:10D10800DA01F0E0EA17FB0751F472DEEA8DFB8DD5
:10D11800A9A1BAA1EA0FFB1FE9A3FAA389CFD4CF2B
:10D1280067DEE0E002C041DEC1CF0E94AD7DA69679
:10D138000895A881A03310F0AA3308F004C0E8814C
:10D14800E0530C948669A881A13410F0A73408F044
:10D1580004C0E881E7530C948669EFEF0C94866964
:10D16800A881AA3020F4E881E05D0C948669A88142
:10D17800AA3020F0E881E95C0C948669E8E50C9413
:10D1880086691A930A93F8940091620B1091630BC5
:10D198007894F8010991199108951A930A93F1DF87
:10D1A8008F01EA81FB81AC81BD81EA0FFB1FE01B87
:10D1B800F10BDF010E949C7D2CF4E0E019810881CD
:10D1C8000C94316CE1E0198108810C94316CECE825
:10D1D800F4E1FA93EA93E8E2F0E0FA93EA930E9422
:10D1E800D36DE4E1EA93EDE2EA93EFE0EA930E947B
:10D1F8000A4E0895089599818881009641F0BD816D
:10D20800AC81FB81EA8105900D920197E1F7FD81E0
:10D21800EC810C94316CB981A881109631F0FC81B5
:10D22800EB816A8161931197E9F7EB81FC8125967F
:10D238000895E991F991A991B9911D90059001146A
:10D2480021F40020D1F7EE2708951018E1F3E1E06A
:10D2580008F4E2500895E991F991A991B991CD01A5
:10D2680061916D936623E1F7FC010895E991F991C5
:10D27800A991B991CD0105900D920020E1F7FC012B
:10D288000895A991B991EE27FF276D91662311F0B2
:10D298003196FBCF0895AA27BB27E991F99105900C
:10D2A800002011F01196FBCFFD0108957991E991C5
:10D2B800F991A991B991CD01772351F07A956191AE
:10D2C8006D936623C9F7772319F07A956D93FBCF91
:10D2D800FC0108956991E991F991A991B991CD015C
:10D2E800662351F06A9505900D920020C9F76623D0
:10D2F80019F06A950D92FBCFFC0108955D9BFECF56
:10D30800E881ECB9219608951A930A93AC81BD81FE
:10D318000E94C47B3097C1F0AA81BB810E94C47B64
:10D328008F01309749F00230E0E01E0760F0F80105
:10D3380031978F01ED93FC93AC81BD810E94D66E2D
:10D348003197AE81A08303C0EE81EA93D7DF1981BC
:10D358000881279608952C970E94A67D10E0E88DF5
:10D36800F98D3196E88FF98F3197E4912E2FE030BF
:10D3780011F40C946D6BE12FE03039F4253211F47F
:10D3880011E002C00E94687AA3C1E130C1F42532DD
:10D3980019F40E94687A9BC112E0E0E0E98B00E092
:10D3A8002D3211F401E094C12B3219F4EBE2E98B30
:10D3B8008FC1203219F4E0E2E98B8AC102C0E23061
:10D3C80039F450E013E0203311F4006881C102C041
:10D3D800E330A1F4203310F02A3308F009C0A52F58
:10D3E800EAE0EA9FF0015E2FE22FE0535E0F70C182
:10D3F80040E02E3211F414E06BC110C0E430A1F407
:10D40800203310F02A3308F009C0A42FEAE0EA9F7D
:10D41800F0014E2FE22FE0534E0F5AC12C3619F46B
:10D42800026015E055C104C0E53011F00C946C6B36
:10D43800E22FE33649F40E94737AEE89FF89A481CA
:10D44800AA930E94797A43C1E33741F40E94737A20
:10D458000E94837A0E9445691E2F0AC0E037A1F412
:10D468000E94737A0E94837A0E944F691E2F086077
:10D478000F77403011F0411708F001C0142F40E039
:10D48800E0E0E88B30E076C0E43611F0E93611F4DC
:10D49800046002C0E537A1F4EAE0E88B01FF08C0A8
:10D4A800E0E0FAEC6AE97BE30E949A6E1AE023C096
:10D4B800E0E1F7E260E070E00E949A6E15E01BC0C0
:10D4C800E83511F4086004C0E83711F00C946B6B70
:10D4D800E0E1E88B01FF08C0E0E0F0E060E070E127
:10D4E8000E949A6E18E007C0E0E0F0E160E070E0AA
:10D4F8000E949A6E14E0403011F00F7701C041E0AD
:10D5080001FF08C00E94737AAE89BF8914960E94F1
:10D51800C87B13C002FF08C00E94737AAE89BF8916
:10D5280014960E943E6E09C00E94737AAE89BF8924
:10D5380014960E94C47B66277727EC87FD876E8741
:10D548007F8702FF16C0AF85AA2362F4EC85FD85AC
:10D558006E857F850E94C37AEC87FD876E877F87FB
:10D56800EDE2E98BE989E03019F01F5F4F5F01C0F8
:10D578000B7F342F00FD14C0151710F4351708F071
:10D588000FC007FF08C002FF04C00B7F2989115094
:10D5980001C020E301C020E20E94687A5150ECCF1C
:10D5A8001417B0F4006102FF0AC00B7FE989EA93FF
:10D5B8000E94797A503009F0515011504150E0E3FF
:10D5C800EA930E94797A503009F051504150E8CFDF
:10D5D800312FE889E030D1F43030B9F003FF08C0CA
:10D5E800EE81FF813196EE83FF833197E49105C088
:10D5F800AE81BF81ED91AE83BF83EA930E94797AB1
:10D60800503009F051503150E7CF57C00E948B7A03
:10D618000E94507B2E2F2A3030F003FF02C0295C75
:10D6280001C0295A01C0205D04FD25C0213360F4E2
:10D63800A885B9858A859B85A130E0E0BE07E0E032
:10D648008E07E0E09E0709F40BC0431740F4531718
:10D6580010F000FF01C014C020E207FF0CC020E357
:10D66800006102FF08C00B7FE989EA930E94797A7A
:10D67800503009F051500E94687A503009F05150EA
:10D6880031500E948B7A0E948B7BEC87FD876E87D6
:10D698007F87E889A885B9858A859B85FF276627BE
:10D6A80077270E94507B0E949A6EE885F9856A85E3
:10D6B8007B850E94987D09F0A9CF00FF08C05030F3
:10D6C80031F05150E0E2EA930E94797AF8CF10E005
:10D6D80046CE0E94AD7D6A960895FF92F82E229755
:10D6E8001A930A93DE010E94B17A8D01DE01169623
:10D6F8000E94B17A0E94C47BEA83FB83DE01149600
:10D708000E94B17A0E941B741A930A93FE013696FE
:10D718000E94BC6C20DEAA81BB81E0E0EC931981F9
:10D7280008812496FF900895A991B991EE270024C5
:10D7380060E8E894162E169407941E2A1EF0A01589
:10D74800B10518F0A019B109E62BB7FBAA0FBB1F4A
:10D75800669580F708957B816A81F981E88177FB76
:10D76800770F67FD7160972F9E5781F078F0983199
:10D7780090F4AA27BB27882708948795B795A7957B
:10D788009A95D1F7EA23FB23682305C0E894772705
:10D79800EE27FF2766276F77769508F4606877F994
:10D7A800A991B99189919991EA17FB0768077907B7
:10D7B80097FB08950E941E7A0E94947A19F40E9499
:10D7C8009B7A1DC0E6F7A881B9818A819B81E0E038
:10D7D800F0E060E87FE30E94637A11C00E941E7A3D
:10D7E8000E94947A19F40E949B7A09C0E6F30E9479
:10D7F8009B7AA0E0B0E080E89FE30E94B77C249683
:10D8080008950E94A07A0E94987D39F4A881B98170
:10D818000E945C700E94CE7B20C0AA81BB818C8153
:10D828009D810E94A07D34F40E94A07A0E94D77B3B
:10D83800C1DF05C00E94A07A0E94D77BCFDFA881F4
:10D84800B9810E94CE7BA881B9810E94C87BAA8138
:10D85800BB818C819D810E94637A26960895E99107
:10D86800F99130971AF4E095F09531960895E09380
:10D878007100E0E0E0937400E2B3E360E2BB089576
:10D8880088EC90E00197F1F70895EA930E94016708
:10D89800E0300895E0E0EA930C94266780E991E08F
:10D8A8000197F1F708951A930A930C943747EA9F62
:10D8B800F001F0E00895FA93EA93A02FB0E00895FC
:10D8C800ECE3F0E00E94207B0895ECE3F0E0FA93AB
:10D8D800EA930895E2E3F3E0FA93EA930C9413448D
:10D8E800E0E0E0930F04EFE0E09310040895E0E037
:10D8F800F0E0FA93EA930895FA93EA93E8E2F0E005
:10D90800FA93EA93E0E0EA930C94264CE0915905E7
:10D91800F0915A05FA93EA930895E0915B05F09126
:10D928005C05FA93EA930895FA93EA930C9490436A
:10D93800EFEEF0E0FA93EA930895FA93EA93E0E0C1
:10D94800EA930C94264CFA93EA930C941344E12F2F
:10D95800A8E3B2E0F0E00E94D77AEA0FFB1F08952F
:10D96800A12FB0E0ADCFFA93EA93E2E3F0E0089597
:10D97800FA93EA93BCCFE0911004E0930F04089562
:10D988000E94610E0C94BF49E32FF0E0E85BFD4F65
:10D99800E4910895EA930E94770EFE013696FA9371
:10D9A800EA930895FF27662777270E94D77B84E0AC
:10D9B8000E94716B28960895FE017196FA93EA9376
:10D9C8000C9433440E94A87D0C943747E8E0F0E0BB
:10D9D800FA93EA930895E4E0F0E0FA93EA9308955D
:10D9E800FA93EA93E8E3F0E0FA93EA9308950E9441
:10D9F800D37BBECFE02FF0E00895A091390CB09111
:10DA08003A0CBD01A3E0B0E00E94F87AE60FF71FD8
:10DA1800E491E0300895E091C005EE0FEE0FEF5F5E
:10DA28003E2F0895E32FF0E00895A12FB0E0089568
:10DA3800A091390CB0913A0CBD01A3E0B0E00E946E
:10DA4800F87AE60FF71F08950E94D57AE85AFD4F35
:10DA58000895FA93EA93E22FF0E008950E94A67DD4
:10DA6800A09119080895E091C20BF0E00895AFE382
:10DA7800B1E00E944B7B089530911E08E1E0E093ED
:10DA88000D04E2E0E0930E043A930E94A819E09195
:10DA9800980BE295EF70E0930F04E091980BEF700C
:10DAA800E09310040895FA93EA93E52FF0E0FA93CF
:10DAB800EA930895E7E3F0E0FA93EA930895E22FF2
:10DAC800E450F0E0FA93EA930895FA93EA93F7CFD3
:10DAD800E32FE058EA930BCFEAE8FBE0FA93EA93E6
:10DAE8000C9433443A930E94A819A0918A0BAD3242
:10DAF8000895E091980BE295EF70E0930F04E091A0
:10DB0800980BEF700895E52FF0E00895EA0FFB1FDA
:10DB1800FA93EA930895EF5EFC4FBF01E081E05865
:10DB2800DB01EC930895E0E0EC93AE81BF810895AA
:10DB3800E3E0F0E0FA93EA930895E52FE450F0E08B
:10DB4800FA93EA930895FA93EA93F2CFE550F0E056
:10DB58000895E091980BE295EF700895EA1BA2E50D
:10DB6800B7E0F0E00E94D77A0895F0E0EE0FFF1FCB
:10DB7800E25DFD4F0895ACE2B2E0F0E0EE0FFF1F6A
:10DB8800EA0FFB1F0895FA93EA93E12FF0E0FA9366
:10DB9800EA930895E12FF0E0FA93EA930895E2E01A
:10DBA800F0E0FA93EA930895EAE8FBE0FA93EA933F
:10DBB800EAE0EA930C94DA46E1E0F0E0FA93EA93BB
:10DBC8000895FA93EA930C94C5460E94D37BFA937E
:10DBD800EA930895ABE0EA9FF001E252FA4F089504
:10DBE800ED85FE85FA93EA9308951A930A933BCF3D
:10DBF8001A930A93E0E0EA930E94264CDDCFE1E015
:10DC0800E0933B0C0E94C568E0933C0CF0933D0CFC
:10DC18000895BD01AAE0B0E00E94F87AE60FF71F68
:10DC28000895FA93EA93EAE0EA930C94DA46E1E07D
:10DC3800E0930E045CCE0E9410470C94F346E0E299
:10DC4800EA930C94AE46A6E4B7E0E881F0E0EE0F64
:10DC5800FF1FAE0FBF1F0E94C47B0895FA93EA937B
:10DC68000C94DB41E881F0E00895EE0FFF1FAE0F42
:10DC7800BF1F08950E94C47B0E94E27A08950E9403
:10DC8800D77B0C94D241FA93EA930C941047A9E0FD
:10DC9800B0E00E94F27B0895A7E11A9FF001EF5CC3
:10DCA800F94FE0810895E12FEF5FEA930C94ED417D
:10DCB800F0E0D4CFE8E0F0E05BCEEA93E6E0EA9368
:10DCC8000E94BD4183CEE0916D05F0916E050895E7
:10DCD800E0916905F0916A050895AE0FBF1FE3E072
:10DCE800F0E00E944B7B0895FA93EA931A930A9303
:10DCF8000C948D13FA93EA933A932A930C948D1308
:10DD0800A0917105B09172050895A0917305B09125
:10DD180074050895A0E0B0E00E94EE7B08950E948B
:10DD2800E77BEA1BFB0B0E94E27A0895E887F987F4
:10DD38006A877B870895A885B9858A859B85EFEED4
:10DD4800F0E060E070E008950E94E27A0E94757B3E
:10DD58000895A4E0B0E00E94EE7B0895FA93EA9358
:10DD68000C942B47FA93EA930C94A57AA9E01A9F8E
:10DD7800F001E858FC4F089537960E94D37BDF01E5
:10DD88000E94C47B08950A921A92FA926A937A932F
:10DD98008A939A93AA93BA93EA93FA93EFB7EA937A
:10DDA8001A930895ED91FD913196FE93EE9308959F
:10DDB800ADE01A9FF001EB5FFC4FE08108951A93E4
:10DDC800E1E0EA930C949947ADE01A9FF001DF0176
:10DDD800EB5FFC4FE081E0300895E2E0EA930C94B9
:10DDE8009947FA93EA93E4E6F0E0FA93EA930E94FB
:10DDF800D168E0300895E1E0E0930D04E0930E046B
:10DE08000895E0912908F0912A0860912B087091F3
:10DE18002C080895E0912108E150A3EAB6E0F0E06B
:10DE28000E94D77AAE0FBF1F0E94C87B0895E12FCA
:10DE3800EF5FF0E028CFE0912208EA93E0911E0816
:10DE4800EA930E947B1AA0911D0CB0911E0C1097AA
:10DE58000895A0911F0CB091200C8091210C9091F5
:10DE6800220C0E94A07D0895E0911D0CF0911E0CDB
:10DE78000895E0911F0CF091200C6091210C709195
:10DE8800220C0895E2E3F0E06DCF1A93E0EAEA93FA
:10DE9800EA81F0E0E050F84FFA93EA930E945E6757
:10DEA8001E2F0895E0EAEA93EA81F0E0E050F84F87
:10DEB800FA93EA931A930C948A67EA930E940E677E
:10DEC800E0300895E0EAEA93EDE5F0E0FA93EA93AA
:10DED800E0E0FFE0FA93EA93EEEBFBE00895FA93B3
:10DEE800EA93E0E2EA930C941368E0EAEA93E981A2
:10DEF800FA81E050FC4FFA93EA930895EA81F0E042
:10DF0800A8E2B0E00E94207B0895E0EAEA9347CEB9
:10DF1800FA93EA930C94AB67FA93EA930C945E67CE
:10DF2800E0EAEA93E8E2F0E0FA93EA931A930A93B4
:10DF3800EAE8FBE00895EAE8FBE0FA93EA9308953B
:10DF4800EDE2EA93EAE0F0E0FA93EA930E940F69BF
:10DF5800E0E00895EA81F0E0ABE0B0E00E94207BC9
:10DF6800E050F24F8F01AA81AA300895E0EAEA93BF
:10DF7800EBE0F0E0FA93EA931A930A93E2EBFBE002
:10DF88000895E3EBFBE0FA93EA930895EA81F0E061
:10DF9800EE0FFF1FE050F04F8F01AA81A0380895BF
:10DFA800E150F0E00895EA81F0E00E94D77AE05865
:10DFB800F14F8F01AA81A5300895EEE2FCE0FA93B3
:10DFC800EA93E0E0EA9307CDEBE1FCE0FA93EA9309
:10DFD800E0E0EA93FBCC0E94207BDF01EA85F0E0D9
:10DFE800AE0FBF1FE8E0F0E00E94207BE050F04D4C
:10DFF8008F01E0EAEA93EACC1A930A93EBE1FCE09A
:10E0080087CFAE81BF81888599850895EE83FF8388
:10E01800688779870895EE81FF81688579850895F5
:10E02800E0931F0CF093200C6093210C7093220C4A
:10E038000895F0E0AE0FBF1F0895EA930E94A81953
:10E048000C944620E091950BF091960B0895FA9365
:10E05800EA930C944719ED81EA93ED81EA930895C8
:10E06800E091AC0BF091AD0B0E94E27A0895F0E0DC
:10E07800A4E6B0E00E94207B0895EC81F0E0EA0F6E
:10E08800FB1F0895E0912708F09128080895E09370
:10E09800260CF093270C0C94DD1CE3EAF6E0FA93C7
:10E0A800EA93E0E0EA930895FA93EA930C940F69EF
:10E0B800E0E0F0E060E070E00895E0932908F09374
:10E0C8002A0860932B0870932C080895E091970B09
:10E0D800A3EAB6E0F0E00E94D77A0895AE0FBF1F1A
:10E0E8000E94C87B0895ED5EF94FE081E130089504
:10E0F800FA93EA93E0912208E05DEA930895EA939F
:10E108000E948B64E1300895ECE3F8E0E093600B43
:10E11800F093610B0895E12FA3EAB6E0F0E00E94C6
:10E12800D77A08950E94FF68A881AF5FEAE00E944D
:10E138002A7BE05D0895A881AF5FEAE00E947A7BC0
:10E14800E05D0895FA93EA93E0E0EA930895AAE07F
:10E15800B0E00E94F27B0895E12FF0E00E94D57AAA
:10E16800E854FF4F32960E94D37B0895E12FF0E0E8
:10E178000E94D57AE854FF4F08953696E491D90164
:10E18800EC930895E0EAEA93E5E0F0E0FA93EA9385
:10E198000895EA930E94CE1CFA93EA93E3E2FCE026
:10E1A8000895FA93EA93EFEFEA93E5E0F0E07CCF85
:10E1B800E093240CF093250C08950E94E77BEA1B5A
:10E1C800FB0B0895A091290CB0912A0C0895E0E06A
:10E1D800E093370CE093380C0895A0912B0CB09184
:10E1E8002C0C0895E0912B0CF0912C0CAC81BD8186
:10E1F800EA0FFB1F0895E0932B0CF0932C0C089565
:10E208001A930E94681D1E2F0895E093290CF0931D
:10E218002A0C0895FA93EA930E94D168E030089591
:10E22800ABE01A9FF001E452FA4F08951A930E9446
:10E23800541FD3CFE091290CF0912A0C0895EA934A
:10E248000E94541F0E94F11EE0300895EB81EA936A
:10E258000E948F1DFA93EA93E8E2FCE00895E0E05B
:10E26800E0934B0CE0934A0C08951A930A93E091BB
:10E278001208ABE0EA9FF001E752F84F8F01D8018E
:10E2880011960895E0E0F0E0ED93FC930895EA819B
:10E29800D801EC93E2E1F8E0FA93EA930E94303473
:10E2A800198108810895E12FACE8B0E0F0E0EE0FA5
:10E2B800FF1FEA0FFB1F0E94D37B0895ACE8B0E074
:10E2C800F0E0EE0FFF1FEA0FFB1F0E94D37B0895BB
:10E2D800A0911608B0911708EA2BFB2BE0931608BB
:10E2E800F09317080895E150A7E1EA9FF001089517
:10E2F800A7E10A9FF001E15DF94FAF010895A3E29C
:10E308001A9FF001ED55F94F0895EC93EC81E15017
:10E31800ADE0EA9FF0010895E981FA81FA93EA9362
:10E328000895E12FF0E00895E2E0F0E00E944B7BD1
:10E338000895AAE9BBE0E0911A080895ADE9BBE0A9
:10E34800E0911A0876CEA0EABBE0E0911A0871CEF7
:10E35800A6E4B7E0D8CBEE0FFF1FEA0FFB1F089526
:10E36800E081F0E00895A7E11A9FF001E15DF94F1F
:10E37800EE83FF83AE81BF810895EE81FF81A48182
:10E38800AA930C948D200D901C90AE81BF8112969B
:10E39800EC91F0E0E00DF11DDB01ED93FC930895A5
:10E3A800ED91FD913197FE93EE9308950E942322FB
:10E3B8000E2EAA85BB85EC91E0150895A3E20A9F6D
:10E3C800F001E855F94F0895E0911208ABE0EA9F93
:10E3D800F001E752F84FEC87FD87AC85BD851196B3
:10E3E80008951296EC91AC85BD851696EC93089528
:10E3F800D001F0E00895A885B98518960E94C47BDD
:10E408000895AC85BD85EC93E2E1F8E0FA93EA93D0
:10E418000C943034E885F985A281AA9308950A936B
:10E428000E947D20E0300895AA85BB85EC91EA938F
:10E43800E3E0EA930C946243AA85BB85E0E0EC93A1
:10E44800E2E0E09324060895BF0100801180AE81C8
:10E45800BF811296EC910895DB01ED93FC93AE8198
:10E46800BF81129660CBF0E0ED93FC930895E2E152
:10E47800F8E0FA93EA930C943034E0911908A091EB
:10E488001808EA170895F0E0E00DF11D0895A3EAD1
:10E49800BBE047CFADE9BBE0EE27A10FBE1FEC9173
:10E4A8000895A0EABBE0EE27A10FBE1FEC910895E6
:10E4B800BD01AAE0B0E00E94F87ADB010895E0818E
:10E4C800EA930C94D25EE0E4FAE0E0935E0BF093FA
:10E4D8005F0B0895EA930E943A63E0E00895EA9397
:10E4E8000E943A630C94C964ADE9BBE0EE27A00F23
:10E4F800BE1FEC910895A0EABBE0EE27A00FBE1F57
:10E50800EC910895AAE9BBE0EE27A00FBE1FEC919D
:10E51800E1700895A3EABBE06DCAA0EBBBE0EE276B
:10E52800A00FBE1FEC910895A9EABBE0EE27A00F4B
:10E53800BE1FEC910895ADE0EA9FF001E15FFC4F4A
:10E548000895ADE0EA9FF001EB5FFC4F0895ABE062
:10E558000A9FF001E452FA4F0895ABE00A9FF001D8
:10E56800EE51FA4F0895FA93EA930C94BB35FA9357
:10E57800EA930E94D4433A9330CCE0912B0CF0916B
:10E588002C0C30970895AFEFBFEFA083B1830895A7
:10E598000E94C568E093500CF093510C0895FA93CB
:10E5A800EA93E0E0F0E80895E0911208ABE0EA9F12
:10E5B800F001E752F84FFA93EA930E948A2957CF5D
:10E5C800E0911008ABE0EA9FF0010895E0E1F8E07F
:10E5D800FA93EA930C943034FA93EA930C94AA537E
:10E5E800E88DABE0EA9FF0010895FA93EA9302CA36
:10E5F800E0E1EA93E0912506EA930E947B191E2F39
:10E60800089540DDFA93EA930895FA93EA930C94F7
:10E618001F1FE0932506E0E0E0934D0CE1E3E09353
:10E628004E0C0E94C92A0C94A826FA93EA930C94DB
:10E638004B63E1E4F9E0E093600BF093610BE3E0F6
:10E64800EA930C94C862A091600BB091610B089595
:10E658000E94C568E093450CF093460C0895E0933A
:10E66800600BF093610B0895E3E0EA930C94C862A1
:10E67800E0932708F093280808950E943747E0E0C0
:10E68800EA930C94740FE0E0F0E0E0932508F0932F
:10E698002608E2E0E0930E040895E091130456CAB8
:10E6A800E0912508F0912608D9CAE0915D05F0911E
:10E6B8005E0531970895FA93EA930C940946EF5C46
:10E6C800EA930C94AE46A6E0B7E0ACC9A3EABBE077
:10E6D800E0911A08F0E03FCE0E94C47BD001ED9390
:10E6E800FC9327CEF0E0EA0FFB1F0F0122CEA6E431
:10E6F800B7E098C9E7E0E0931808EA93E0E0EA9306
:10E70800F6C8EA930E9466410E9475431E2F089539
:10E71800EAE2EA93EDE2F9E115CD0E94752CE1E019
:10E72800EA930C945D2C1F771A930C94A819A09166
:10E738002508B09126080895E8EEF3E00E947D7B55
:10E748000895E053F0E00895A0E024FCA1E0A03093
:10E758000895E0E0EA93CBC8E0913308F0913408DB
:10E76800FA93EA930895FA93EA930E94D168E13004
:10E7780008950E94C568E0933308F093340808951B
:10E78800E0E0E0934A0C0895D2DFEA17FB0708950A
:10E79800E0931808E0E0E093300808950E94696467
:10E7A8000E94DE2DE093240808950E94A8190C9475
:10E7B8003747E0911908EA93E0E0EA930E94882D30
:10E7C8000C943C290E9475431E2F1A930E940E2E0A
:10E7D800103808951A93E091C605EA930895E091D8
:10E7E800890BEA930E94B318E03008950E94C56827
:10E7F800E093520CF093530C0895D90118960E9497
:10E80800C47B0895E4E6F0E060E070E00E94757B68
:10E8180008950E94A81916CC0A93E091C605EA93B8
:10E828000895E0912F08EA930A930C94EB1A0E943A
:10E83800C47BFA93EA930895A0E6BBE0B3CAE091DB
:10E848003C08E053E09322080895FA93EA93E0E342
:10E85800EA930C946964E0913908EA930C94116482
:10E868000E94E27A0E94D77B08950E94BC63EBE382
:10E87800EA930C943A63E89423F8E0E0F0E0F8DED9
:10E888000A93E1E0EA930C94882D0A93E1E0EA9375
:10E898000E94882DE1E00895E0911208ABE0EA9F1C
:10E8A800F0010895A881B981EC91EF5FEC93089588
:10E8B800ABE00A9FF001E352FA4F0895A083ABE062
:10E8C8000A9FF0010895ABE00A9FF001E152FA4F68
:10E8D8000895EDE5F9E1FA93EA93EA85ABE0EA9F5A
:10E8E800F0010895AC81BD81EE27A00FBE1F0895E9
:10E8F800E02FAC81BD81F0E008950E94D77B84E0D1
:10E908000E94716B28960895EE27A30FBE1FEC9105
:10E91800D001EC930895A2E5B7E084C80E94D77AA5
:10E92800EA0FFB1FAF010895E0912B0CF0912C0C1E
:10E938000895E32FA0911E08EA0F0895ADE02A9FDD
:10E94800F001E35FFC4F0895A8E0B0E00E94F27B7D
:10E958000895F0E0FA93EA9308950E94E7420C9430
:10E96800C142F0E00E94D77A08950E94D77B0E94A6
:10E97800DC420C94C1420E94E742E1E8F9E1E2CBB3
:10E988000E94C1420C94C14220E030E0E12FE05DDA
:10E99800EA93E4E8F9E1ACCBEAE0EA930C941A6371
:10E9A80010915D0500915F0508950E9475433E2F03
:10E9B8000C945746EAE0F0E00E94207B0895DF01BE
:10E9C800EE27A30FBE1F0895FA93EA9334C9EF8187
:10E9D800F885FA93EA930895F0E0EA0FFB1F08958B
:10E9E800E02FA8EFB1E0BDCFEA0FFB1F3296E4910C
:10E9F8000895FA93EA93E2E0EA930E940539E13236
:10EA08000895EA930E94AB38E1320895E6E0F0E019
:10EA18000C94BC6C0E941047AAE9BBE0EE27A10F3A
:10EA2800BE1FEC91E1700895EE0FFF1F6FC8EA93C7
:10EA38000E940539E13208950E948A0E0C947B6C7D
:10EA4800EAE3EA930C94AE46E3E7EA930C94AE4605
:10EA5800EA23EA930E94F241F2C8EA930E94F24143
:10EA6800EEC8DF013296B1C80E94D57AE854FF4F4C
:10EA78000895EAE3F6E0E093390CF0933A0C089530
:10EA88000E944A1BE0E0E09321080E9496160E942B
:10EA98008A0EE1E0E0931B0808950E9437470E9420
:10EAA80024110E9475430E2F0D330895EE81FF81C6
:10EAB800FA93EA930895EAE2EA93ECE2FAE1089518
:10EAC800EA930E94E6160C948A0EE093C105F0932F
:10EAD800C20508952A97FE01FA93EA930895E4E49B
:10EAE800FAE1FA93EA93AE85BF85888999898ACE37
:10EAF8000E94D77BAA89BB898C899D89E4E6F0E0CE
:10EB080060E070E00E948F7B0E94D77B88E00E94C3
:10EB1800716B2C96FE010895FA93EA930C94B6460D
:10EB2800EDE4FAE1FA93EA93EE85FF8599CE84E065
:10EB38000E94716B2896FE01EFCFFA93EA93EE8557
:10EB4800FF8508950E942C640C94C56884E00E9497
:10EB5800716B28960895EE27A10FBE1FEC910895BA
:10EB6800EA930E945C421F5F0895E091C405A7ECF8
:10EB7800B5E0F0E00895AF5FEAE00E947A7B08957F
:10EB8800E091C305A7ECB5E0F0E0E5CBE981ADE0A5
:10EB9800EA9FF001E05FFC4F0895EF73A5E1EA9F5B
:10EBA800F001E051FB4F0895EF73ABE0EA9FF001ED
:10EBB800EC5EFB4F0895AC81BD81EE27A30FBE1F0D
:10EBC800AC91A0300895ABE00A9FF001EC5EFB4FDA
:10EBD8000895EA0FFB1F0F01AC81BD8195CEA5E119
:10EBE8000A9FF001E051FB4F0895EE81FF810180FB
:10EBF8001280AE81BF8115960E94C47BD001089512
:10EC0800FE013896FA93EA930895EAA5FBA5FA93CC
:10EC1800EA930895FA93EA93FE013A96FA93EA93EF
:10EC28000E942F6930E0E02F0895E091C105F0912E
:10EC3800C2050895A1ECB5E0ED91FD913296FE93E1
:10EC4800EE930895AE81BF81EA17FB070895E0E0CF
:10EC5800E0936505E093660508951A930A933A933D
:10EC68002A930895FA93EA93E0910E040895A091E7
:10EC78000003B09101030895E0910003F0910103AE
:10EC8800FA93EA93E0910203F0910303FA93EA936B
:10EC98000895E0930003F09301030895A981BA81D0
:10ECA8005ACF1A930A9300E010E00895F801AA8158
:10ECB800BB81EA0FFB1FE4910895AE0FBF1FAC9113
:10ECC800A0300895D801F0E0AE17BF070895AE0F41
:10ECD800BF1FEC91EA930895EFEEF0E0EA1BFB0BFF
:10ECE8000895A0910E04E4E1EA9FF0012E2F332746
:10ECF800C3CFE0E0EA930E94264C0E94AF7D0895BE
:10ED0800ECE0EA9FF001A0910D04EA9FF00108955C
:10ED18001A93E1E0E0930E04E0930D0410E00895E7
:10ED2800ED81FE81FA93EA930895EF81F885EA1B55
:10ED3800FB0B08953A932A935A934A930895EAA5A8
:10ED4800FBA5E20FF31FFA93EA930895ECA1EA9367
:10ED58000C94894C3A932A93EEA1FFA1E40FF51F76
:10ED68000895FA93EA93EBCFEAA5FBA5E40FF51F04
:10ED7800FA93EA93EBCFE20FF31FFA93EA9308951D
:10ED8800FA93EA935A934A930895EA9FF001AEA141
:10ED9800BFA1F0E00895E2E0E0930E04E0E2F0E0C5
:10EDA800EAA3FBA30895AE1BBF0BBECAEE8DF0E02D
:10EDB8000895E20FF31F3196FA93EA93ECA1FDA1AF
:10EDC800E40FF51F31960C94B26EECA1FDA1E40F8F
:10EDD800F51F0C94B26EE9A1F0E0DE0116960895D5
:10EDE800ED8DEA930E946446E9A1EF5FE9A30895D7
:10EDF800ED8BFE8BAB89BC8997CAA98DBA8DEA0FBA
:10EE0800FB1FE98FFA8FEB89FC89AF89B88DEA0F70
:10EE1800FB1FEF8BF88FED89FE89AD89BE890E94B3
:10EE2800207B0E94E27A0E947D7CEE87FF87688BB8
:10EE3800798BEB89FC89AB89BC890E94207B0E9475
:10EE4800E27A0E947D7CAE85BF85888999890E9477
:10EE5800537DEA87FB876C877D8700E010E0089583
:10EE6800F8010E94E27A0E947D7CD0D8D4D8C9D813
:10EE78000E94057DAA85BB858C859D850E94057DA0
:10EE8800AE85BF85888999890E94E17B0E94B07C04
:10EE98000E94467CAF015A934A930C94986BE98D73
:10EEA800FA8DE21BF30BFA93EA930895E98DFA8D34
:10EEB800E01BF10BFA93EA930895F901AD8DBE8D2D
:10EEC8000C948A6DED8DFE8DE01BF10BFA93EA939D
:10EED800EA8DEA930C94894CAD8DBE8D0C948A6DA5
:10EEE800EFE3F1E0EA1BFB0B0895EB81FC81AF81B6
:10EEF800B8850895E00DF11DFA93EA930E949B4AA4
:10EF0800E5E3EA930895E09365000C94466F0E9448
:10EF1800A67DEE81EA930E94CA4A8F010895E98589
:10EF2800FA85AD85BE8508950E94E44AEB85FC8587
:10EF3800FA93EA930C94FC4AED85FE85A985BA8577
:10EF4800AE17BF070895EB85FC85AF81B885AE176E
:10EF5800BF070895AD85BE85E985FA85EA1BFB0BD9
:10EF68000895FA93EA930C94336CAB85BC85DDCE97
:10EF7800AF81B885EB85FC85EA1BFB0B0895D901A9
:10EF88000E94207B0F010895D0010E944B7BAF01A6
:10EF9800FA01AD85BE850C948A6DED85FE85E21B70
:10EFA800F30BFA93EA930895AD85BE850C948A6DA8
:10EFB800A985BA85ED85FE85EA1BFB0B0895E881D6
:10EFC800F981FA93EA9308955A934A93EE85FF8557
:10EFD800B4CDFA93EA93EC85FD85FA93EA930E94FF
:10EFE8006A4DE0910E04AA85BB85F6CCD901F0E004
:10EFF800AE17BF070895E05CF54F61CAE091360C83
:10F00800A091350CEA170895E0911108ABE0EA9F4A
:10F01800F0010895E081E05DEA930C943A63A091D1
:10F02800240CB091250C0895E2E5EA930E943A6316
:10F038000C94574EF096EA930E941164E2E7EA9323
:10F048000C943A63E081EA930C943A63EEE0EA9315
:10F058000C943A63E0E6FAE1E8CA0E947163EBE3D4
:10F06800EA930C943A63E0E3EA930C943A63EBE393
:10F07800EA930C943A635A934A930E9447190E2FC5
:10F0880003360895FA93EA930C9430341A93E98579
:10F09800FA85FA93EA930895E552F84FA885B98559
:10F0A800A083B183F9CBE2E5EA930C943A631A930F
:10F0B800E0913908E0531E2FEDE3F8E0D0CAE09163
:10F0C8001208A0911308EA170895E3E1F8E0DACFEF
:10F0D800E0911308ABE0EA9FF0010895A091740B4A
:10F0E8004ACDE093740BEAE2EA930E941164DBCF05
:10F0F800E091740BE05AEA930E943A63A7CFD901D2
:10F108001696EC9126CCF901A281B381BA93AA9301
:10F1180008950E947163EAE3EA930C943A63D90173
:10F128001196E0E0EC930E942C64CFCFD901EC91CA
:10F1380010CCE05DEA930C943A63E05DEA930E9498
:10F148001164B1CFEB58F44F65CFEAE3EA930E941C
:10F158003A63F9010895E0935C0CF0935D0CE2E0EA
:10F16800E0933608D9011196EC930895EA930E942A
:10F17800116499CF0E947163E5CCE091190CDDCF41
:10F18800E091190CF0E0DECFFA93EA9366CF0E9483
:10F198007163ECE2EA930E943A6311CF54DAAC91BE
:10F1A800A0330895A0915E0BB0915F0BE0E0EC9363
:10F1B8000895EE81FF81E093260CF093270C1093BD
:10F1C800230C0E94DD1CE1E3089541E050E00E9419
:10F1D8005662E887F987EAE3EA930E94CE61E13054
:10F1E80008951A93E985FA85CBCDE2E2EA930C9467
:10F1F800CE6129DAAC91A032089525DAAC91AB330F
:10F20800089521DAEC91EA930895EAE3EA930C94DD
:10F21800CE610E9456623197E887F987E88508959C
:10F228000E94C47BE40FF51FD001ED93FC93089571
:10F23800E091400BF0E0ED55F94F0895E0E0E093E0
:10F24800610CE093620C08950E9456623197E09336
:10F25800400BE091590BA091400BEA1708950E94CA
:10F268005757E091400BEA930895ECE2EA930E9425
:10F27800CE61E0300895EC5BF44F0F01E4D9EC91D6
:10F28800D001EC931F5FD8CAEC5BF44FA0E0A083D9
:10F298000895EA930E94CE61E1300895E4E4FBE02A
:10F2A800FA93EA930895E091410B96CBE091410BD4
:10F2B800EF5FE093410B0895A3EABBE0E091410BB7
:10F2C800F0E049C8AAE9BBE0E091410B0C941D703D
:10F2D800E091410BF0E00895FA93EA930C94DA5325
:10F2E800E091400BF0E0C0CB0E947163ECE2EA933E
:10F2F8000C943A63ECE2EA930C943A630E94CF537D
:10F30800E0E0E093410B0895E091410B0C941D70EF
:10F31800E091600BF091610B0895AEE5BBE00C94B1
:10F32800D66EA0915E0BB0915F0BEC93F6CFA091D7
:10F338005E0BB0915F0B13970895E0E0EA930E948B
:10F348003354E09335080895AA81BB81EC91E29586
:10F35800E07FAE2FEC810895EA0FAA81BB81EC9380
:10F36800A1CAE091020DA091010DEA170895E0915C
:10F378003B09F0E0E05CF64F08951083E0913B090B
:10F38800EF5FE0933B09E12FA0913D090895E093D9
:10F398003D09E0913C09E150E0933C09E0300895D3
:10F3A800E05CF64FA0E0A0830895E091CD0DF091C8
:10F3B800CE0D0895A091CB0DB091CC0DEA17FB07A7
:10F3C8000895E12FA091D20DEA0FE093D20DE091BC
:10F3D800D40D0895F0E0E85CF74F10830895E091AC
:10F3E800D90EF0E0E852F24FE081E0939C00E09102
:10F3F800D90EEF5FE093D90E08950E94A87D00E032
:10F4080010E0089520D9AC91AA3308950F011BD9B3
:10F41800EC91E0530C944772EC5BF44FE081E030E0
:10F428000895EEE0FBE1FA93EA930895E881EA9300
:10F438000C943A63E881F9816A817B810E94D77BC9
:10F448000895E05CF54FE081E0300895EA930E946A
:10F45800B468EA930C94D25EEA930E948265EAE566
:10F46800E0933E090895EA930E944367E0300895C7
:10F47800E0917100E87F1E2F0895E0937300E4E89F
:10F48800F2CF0A930E941A67E0300895FF27662793
:10F4980077270E947D7C0895EE8DAE85BF8588898B
:10F4A8009989F4DF0E94057DA9A1BAA18827992727
:10F4B8000E94DE7B0E94E17B0E94B07C08950E943E
:10F4C800E17B0E94B07C08952A93ED89FE89FA9326
:10F4D800EA93FE017596FA93EA930C948869EE898B
:10F4E800FF893497EE8BFF8B0895ED89FE89FA9397
:10F4F800EA93FE017596FA93EA930C948869AE89AB
:10F50800BF8914960E94C47BEE83FF83CFCAE88527
:10F51800F9856A857B85AC85BD858E859F8508952F
:10F528000E94AF6BE883F9836A837B830895E8813F
:10F53800F9816A817B810895EA81FB816C817D81F3
:10F548000895E991F991309639F080EA9FE00197A2
:10F55800F1F7A8953197C9F708950024AF0DB01DAC
:10F568000895EA0FFB1F681F791F0895EA1BFB0B1C
:10F57800680B790B0895F195E195F0400895F095A1
:10F5880060957095E195FF4F6F4F7F4F0895EE237B
:10F598000E2EEA2F19F0EE0F0A94E9F70895EE0FF0
:10F5A800FF1FEE0FFF1FEE0FFF1FEE0FFF1F089547
:10F5B800FE2FFF0FFF0B6F2F7F2F08956F2F660F02
:10F5C800660B762F0895BA2FBB0FBB0B8B2F9B2F83
:10F5D80008958B2F880F880B982F0895EA17FB073B
:10F5E800E1E00CF0EE270895FA9FF02DEB9FF00D67
:10F5F800EA9FE02DF10D08957A9F702D6B9F700D95
:10F60800F89F700DE99F700D6A9F602D710DFB9F2B
:10F61800600D711DE89F600D711D8827FA9FF02D00
:10F62800610D781FEB9FF00D611D781FEA9FE02D9B
:10F63800F10D681F781F089582D0D6DF0EF49BDF86
:10F6480008958BD0D9DF0EF49ADF0895002498E04E
:10F65800AA0F001C0E1A10F40E0E01C0A1609A9594
:10F66800B9F7EA2FA02D08950024112490E1AA0FDC
:10F67800BB1F001C111C0E1A1F0A18F40E0E1F1EA9
:10F6880001C0A1609A9599F7FD01D001089557D05E
:10F69800EBDF0EF470DF08953F934F935F930024E0
:10F6A80011244427552730E2AA0FBB1F881F991F32
:10F6B800001C111C441F551F0E1A1F0A460B570B1E
:10F6C80028F40E0E1F1E461F571F01C0A1603A9551
:10F6D80059F7FD01BC01D001CA015F914F913F91DB
:10F6E80008953BD0D9DF0EF44ADF0895AFDFEA2F43
:10F6F8000895E894B7FF04C0A095B0951196689452
:10F70800F7FD39DFB1DFFD010EF435DF0895C4DF01
:10F71800FD01BC010895E89497FF09C0A095B09534
:10F7280080959095AF5FBF4F8F4F9F4F689477FD3F
:10F7380026DFB2DFFD01BC010EF421DF0895E89455
:10F74800F7FF02C018DF6894B7FF06C0A095B09510
:10F75800119600F8039400FA0895E89477FF02C020
:10F768000EDF689497FF0BC00024A095B095809594
:10F7780090951196801D901D00F8039400FA089545
:10F78800ED91FC9111970895ED91FD916D917C910A
:10F7980013970895ED93FD936D937C9308950590C9
:10F7A800F491E02D08957A936A93FA93EA93089571
:10F7B800689401C0E89401D09DD0182E862F612D41
:10F7C800192E972F712D1B2EBF2FF12D1A2EAE2F0C
:10F7D800E12D0895119602D0FE2F1197E199FECFE1
:10F7E800FF93FFB7F894AEBBBFBBE09AEDB3FFBF82
:10F7F800FF91089507D01196EF93EF2F03D0EF9163
:10F8080011970895E19B02C0A895FCCF9FB7F89483
:10F81800AEBBBFBBE09A8DB3E81719F0EDBBE29A17
:10F82800E19A9FBF0895552342F4503811F4E0FF40
:10F8380004C03196691F791F6BF050E8572711F4FF
:10F848005F93CDC05F3F31F0660F000C5795679509
:10F85800752F08955F9300200AF0CDC0C6C050E808
:10F86800192E1522880F991F9527550F879550E84F
:10F87800072E0522660F771F7527550F6795089580
:10F88800689401C0E8945F93F2DF703818F07F3F06
:10F8980008F4A5C056E1571BAAF4519558300EF448
:10F8A800593030F0EFEFFFEF6FEF7FE777F91AC0CD
:10F8B80077275523B9F0EE0FFF1F661F771F5A955C
:10F8C800D1F710C07727583028F0EF2FF62F672F81
:10F8D8005850F9CF552331F076956795F795E79508
:10F8E8005A95D1F700200AF44ADE5F91089568948A
:10F8F80001C0E894309760407040B1F0002426F0D1
:10F90800772312F400943BDE172E7EE1112032F0AB
:10F918007A95EE0FFF1F661F111CF9CFEF2FF62FF8
:10F92800612D5F938ADF5F9108954F93AF01FD01C9
:10F93800DA01AB01BC01CA01402D012C142E4F91F4
:10F948000895EA0FFB1F681F0895E095F0956095EC
:10F95800EF5FFF4F6F4F08955F9381DF903871F12C
:10F9680050E8152604C05F937ADF903839F1703873
:10F9780021F1572F591B13F112F4D7DFFACF583161
:10F9880018F0AA27BB278827583028F0AB2FB82FA4
:10F9980088275850F9CF552329F08695B795A7950C
:10F9A8005A95D9F7502D512562F0CBDF38F4679579
:10F9B800F795E795739513F41EC0B7DF3EDF5F91A7
:10F9C8000895EA1BFB0B680B51F010F40094BDDF9F
:10F9D8006623A2F3EE0FFF1F661F7A95CBF7EE277B
:10F9E800FF27662777275F910895EFEFFFEF6FE70F
:10F9F8007FEF5F910895EFEFFFEF6FE77FE75F918C
:10FA080008955F932CDF703851F3903841F3012447
:10FA18000894791F23F41CF300203AF3ECCF0F92DB
:10FA28001F932F933F934F93112722279927689F5E
:10FA3800A0018F9F302D410D591F6B9F300D411D27
:10FA4800591F8E9F27D0BF9F25D06A9F23D0BE9F66
:10FA58001DD0AF9F1BD0AE9F110D291F391F491F05
:10FA6800591FE32FF42F652F522F4F913F912F915C
:10FA78001F910F9066232AF0550FEE1FFF1F661F78
:10FA880002C073954BF2CFDE5F910895100D211DD2
:10FA9800391F02C0200D311D491F591F08955F935A
:10FAA800DEDE703821F411200AF49FCFA4CF9038FD
:10FAB80009F495CF01240894970B1BF4D4F3002084
:10FAC800F3CF792F1F932F933F934F93112411272F
:10FAD800222733274427552790E2AE17BF0786070A
:10FAE800410730F0AE1BBF0B860B410B089401C0D9
:10FAF8008894551F221F331F111CAA1FBB1F881F64
:10FB0800441F9A9551F7F901612D4F913F912F911B
:10FB18001F91662332F0550FEE1FFF1F661F7A955F
:10FB280043F281DE5F9108953097604070400895F8
:10FB380000240A160B06089500240A160B06080668
:10FB4800090608955A934A933A932A931A930A9363
:10FB580008955D814C813B812A811981088108952E
:00000001FF
